:100000000C9436050C9455050C9455050C94550527
:100010000C9455050C9455050C9455050C945505F8
:100020000C9455050C9455050C9455050C945505E8
:100030000C9455050C9455050C9455050C94CEA9BB
:100040000C9455050C9455050C9455050C945505C8
:100050000C9455050C9455050C9455050C945505B8
:100060000C9455050C94CE8E0C94FC8E0C94550576
:100070000C9455050C9455050C9455050C94550598
:100080000C9455050C9455050C9455050C94550588
:100090000C94CA100C9455050C94F6100C9455054C
:1000A0000C9455050C9455050C9455050C94550568
:1000B0000C9455050C9455050C9455050C94550558
:1000C0000C9455050C9455050C9455050C94550548
:1000D0000C9455050C9455050C9455050C94550538
:1000E0000C9455050C94DB110C94E5110C94D11172
:1000F0000C947B110C94A6110C94EF110C945011DC
:100100000C9403120C94AE160C94C1160C94550565
:100110000C9455050C9455050C940D120C94F91182
:100120006E616E00696E6600202073747430383A18
:1001300030343A3030202E2E2E2E20536574207409
:10014000696D65202848483A4D4D3A535320666FF3
:10015000726D61742900202073747531323735391E
:100160003930383538202E2E205365742074696D4F
:10017000652F646174652028556E69782074696DF7
:100180006520666F726D6174290D0A00202065205C
:100190002E2E2E2E2E2E2E2E2E2E2E2E2E2E204576
:1001A0007261736520454550524F4D2C206C6F6134
:1001B000642064656661756C7420636F6E66696740
:1001C00075726174696F6E0D0A0047656E657261C4
:1001D0006C20436F6E6669673A0D0A0020206D201F
:1001E000706F6C6C203630202E2E2E2E2E2E20532B
:1001F000657420696E74657276616C2062657477CF
:1002000065656E20636865636B696E6720666F72F3
:1002100020757064617465730D0A0020206D207470
:100220007072203435202E20536574207365636FFF
:100230006E647320666F72205450726F67206F7502
:10024000747075740D0A00202020202020202020AA
:10025000202020616E6420656E64732061742030FC
:10026000373A35393A35390D0A0020202020202030
:1002700020202020202020696E64657820322E20E6
:10028000507269636520697320302E34352C2073D9
:1002900074617274732061742030303A30303A30B7
:1002A000300D0A0020202020202020202020202087
:1002B0004164642F4F766572777269746520656E4C
:1002C00074727920746F2070726963696E6720742C
:1002D00061626C652C20656E7472790D0A002020B5
:1002E000702061646420322030303A30303A30304F
:1002F0002030373A35393A353920302E34350D0A29
:10030000002020702064656C2032202E2044656C13
:1003100065746520656E74727920322066726F6D27
:10032000207072696365207461626C650D0A00203B
:10033000207020696E666F202E205072696E7420C6
:1003400070726963696E6720696E666F2026206D22
:10035000657465722073657474696E67730D0A0045
:1003600050726963696E67206F72204D65746572A3
:100370002053747566663A0D0A002020736D632061
:100380002E2E2E2E2E20536574206D6F64652074E2
:100390006F20636F6F7264696E61746F720D0A0013
:1003A0002020736D72202E2E2E2E2E205365742049
:1003B0006D6F646520746F20726F757465722F6540
:1003C0006E646E6F64650D0A002020736331352002
:1003D0002E2E2E2E20536574206368616E6E656C20
:1003E00020746F2069653A2031350D0A0020207392
:1003F0007042414444202E2E205365742050414EBB
:10040000494420746F2069653A2030784241414464
:100410000D0A003830322E31352E3420436F6D6D89
:10042000616E64733A0D0A0020206970202E2E2E12
:100430002E2E2E205072696E742066756C6C2049C9
:1004400050204D656E750D0A00495020436F6D6D4B
:10045000616E64733A0D0A00202064202E2E2E2E29
:100460002E2E2E2044756D7020726164696F20728B
:1004700065676973746572730D0A00202069202E08
:100480002E2E2E2E2E2E20496E666F0D0A004465EC
:1004900062756767696E673A0D0A00556E6B6E6F1D
:1004A000776E206D6574657220636F6D6D616E642B
:1004B0000D0A00556E6B6E6F776E206D65746572F8
:1004C00020636F6D6D616E640D0A00706F6C6C203F
:1004D0007261746520746F6F20736D616C6C0D0AAE
:1004E0000053657420706F6C6C20726174650D0A26
:1004F000007450726F6720746F6F20736D616C6C45
:100500000D0A00536574207450726F670D0A005510
:100510006E6B6E6F776E2070726963696E672063B1
:100520006F6D6D616E640D0A00556E6B6E6F776E48
:100530002070726963696E6720636F6D6D616E64B0
:100540000D0A000D0A4572726F7220616464696E53
:100550006720656E7472790D0A007450726F67209F
:10056000287365636F6E6473293A2000506F6C6C5A
:10057000696E6720706572696F6420287365636FA8
:100580006E6473293A2000556E6B6E6F776E20276C
:100590007365742720636F6D6D616E643F0D0A0093
:1005A000496E76616C69642074696D65206F706551
:1005B000726174696F6E0D0A006E6F6465207479E4
:1005C0007065206368616E6765642E205265626F96
:1005D0006F74206E6F77202E2E2E0D0A006E6F64C2
:1005E000652074797065206368616E6765642E208C
:1005F0005265626F6F74206E6F77202E2E2E0D0A5B
:10060000002C207265736574206E6F646520746FB2
:100610002074616B65206566666563742E0D0A0043
:1006200053657474696E67206368616E6E656C20D3
:10063000746F20000D0A53657474696E6720504111
:100640004E494420746F20000D0A5A49503E00451F
:100650004550524F4D20496E76616C69642E204C96
:100660006F6164696E672064656661756C74730D93
:100670000A00454550524F4D2056616C69640D0A81
:100680000003020201010000FFFEFDFCFBF9F7F48C
:10069000EFB1253D22A821802C00000000CC3300C2
:1006A000007430A52F00001C3800009F3931340041
:1006B000003425442500000A25232500000000EC15
:1006C000240000000000004A249C2400008A243AF0
:1006D000246C2400002B247B24010401010102016D
:1006E00001010101010101010104010802010101EF
:1006F00001020101020102010102010202010101E4
:10070000012201110104010401010101080202009A
:100710000110010808485454502F312E3120323036
:1007200030204F4B0D0A436F6E74656E742D5479F3
:1007300070653A206170706C69636174696F6E2FC7
:100740006578690D0A0D0A003C3F786D6C2076656E
:100750007273696F6E3D92312E309220656E636FB9
:1007600064696E673D925554462D38923F3E0D0A9E
:10077000003C54696D6520786D6C6E733D926874B1
:1007800074707B737D3A2F2F7265662F7665729237
:100790003E0D0A3C556E6978546D3E003C2F556EF7
:1007A0006978546D3E0D0A3C2F54696D653E0D0A03
:1007B000003C54617269666650726F66696C6520B0
:1007C000786D6C6E733D92687474707B737D3A2F94
:1007D0002F7265662F766572923E0D0A003C545466
:1007E0004920687265663D222F70722F302F746623
:1007F000662F0022202F3E0D0A003C2F54617269A3
:10080000666650726F66696C65203E0D0A003C5446
:10081000544920786D6C6E733D92687474707B736C
:100820007D3A2F2F7265662F766572923E0D0A3CD7
:10083000737461727454696D653E003C2F7374610A
:10084000727454696D653E0D0A3C656E6454696D41
:10085000653E003C2F656E6454696D653E0D0A3C33
:100860004368617267653E3C66697865643E3C76C4
:10087000616C3E003C2F76616C3E0D0A3C637572E4
:100880003E5553443C2F6375723E0D0A3C2F6669FA
:100890007865643E0D0A3C2F4368617267653E0DC2
:1008A0000A3C2F5454493E0D0A003C41637469765A
:1008B0006554617269666620786D6C6E733D9268EE
:1008C0007474707B737D3A2F2F7265662F76657214
:1008D000923E003C2F41637469766554617269668B
:1008E000663E000D0A0020202020202020207C00D1
:1008F000202020202A2020207C00496E646578205A
:100900007C20416374697665207C202020537461CB
:10091000727420207C20202020456E642020207CC2
:100920002056616C7565200D0A00494E46494E49B6
:1009300054594E414ECDCCCC3D0AD7233C17B7D1AC
:100940003877CC2B329595E6241FB14F0A00002052
:10095000410000C84200401C4620BCBE4CCA1B0ED1
:100960005AAEC59D7400407A10F35A00A0724E181A
:10097000090010A5D4E80000E87648170000E40B51
:1009800054020000CA9A3B000000E1F50500008017
:10099000969800000040420F000000A08601000071
:1009A00000102700000000E80300000000640000C1
:1009B0000000000A00000000000100000000002C00
:1009C00076D888DC674F0823DFC1DFAE59E1B1B7C5
:1009D00096E5E3E453C63AE651997696E8E6C28492
:1009E00026EB898C9B62ED407C6FFCEFBC9C9F40AA
:1009F000F2BAA56FA5F490055A2AF75C936B6CF9CF
:100A0000676DC11BFCE0E40D47FEF520E6B500D0A4
:100A1000ED902E0300943577050080841E080000B9
:100A2000204E0A000000C80C333333330F986E1287
:100A3000831141EF8D2114893BE65516CFFEE6DB8D
:100A400018D1844B381BF77C1D901DA4BBE42420D7
:100A50003284725E228100C9F124ECA1E53D276356
:100A600064696E6F70737578585B000011241FBE47
:100A7000CFEFD1E4DEBFCDBF16E1A0E0B2E0E4E607
:100A8000F3E801E00BBF02C007900D92A430B1075C
:100A9000D9F719E3A4E0B6E101C01D92AF37B10761
:100AA000E1F70E94600D0C94D8690C940000089541
:100AB000089508956F927F928F929F92AF92BF9206
:100AC000CF92DF92EF92FF920F931F93DF93CF931A
:100AD000CDB7DEB7EC970FB6F894DEBF0FBECDBF33
:100AE00080E00E94CA9400D000D000D0EDB7FEB7DD
:100AF00031964E010894811C911CADB7BEB7129679
:100B00009C928E92119780E092E0938382838091F1
:100B1000A4079091A507958384830E9495BDEDB7A6
:100B2000FEB736960FB6F894FEBF0FBEEDBF82E05B
:100B3000B4010E94388F80E197E20E9419138091DE
:100B4000C01B882319F42EE032E002C022E132E01B
:100B500000D000D000D0EDB7FEB731968E010F5F08
:100B60001F4FADB7BEB712961C930E93119785E138
:100B700092E093838283358324830E9495BDEDB7F1
:100B8000FEB736960FB6F894FEBF0FBEEDBF83E0FA
:100B9000B4010E94388FC80162E272E00E9434BC46
:100BA000D8010D900020E9F77D010894E108F108D3
:100BB00080E197E20E941913CC24DD2429E2622E01
:100BC00022E0722E58018E01095F1F4F00D000D025
:100BD00000D0EDB7FEB73196ADB7BEB71296FC9216
:100BE000EE92119773826282D601A45DB64D8C910C
:100BF000848315820E9495BDE2E0F0E0EE0EFF1EB8
:100C00008DB79EB706960FB6F8949EBF0FBE8DBFE8
:100C100097E0C91661F4D7011C9284E0B4010E94E8
:100C2000388FC5016EE272E00E9434BC78010894EE
:100C3000C11CD11CB0E1CB16D10441F6F7011082E2
:100C400085E0B4010E94388F8E010F5F1F4FC801ED
:100C500065E372E00E9434BCD8010D900020E9F7F2
:100C60007D010894E108F1089CE3C92E99E2D92E90
:100C7000870189E2A82E82E0B82E00D000D000D0F3
:100C8000EDB7FEB73196ADB7BEB712961C930E9373
:100C90001197B382A282D6018D916D018483158252
:100CA0000E9495BD0E5F1F4FEDB7FEB736960FB68B
:100CB000F894FEBF0FBEEDBFF4E4CF16F9E2DF06F5
:100CC000E1F6D70150961C9280E197E20E94191339
:100CD00086E0B4010E94388F83E040E452E46FE084
:100CE00070E020E030E00EE816E0EE24FF240E94E1
:100CF0002D15EC960FB6F894DEBF0FBECDBFCF9189
:100D0000DF911F910F91FF90EF90DF90CF90BF90F8
:100D1000AF909F908F907F906F900895EF92FF9289
:100D20000F931F93DF93CF93CDB7DEB7EC970FB63A
:100D3000F894DEBF0FBECDBF80E00E94589281E0E4
:100D40000E94589282E00E94589280E00E9467912F
:100D50002DB73EB7285030400FB6F8943EBF0FBEB7
:100D60002DBFEDB7FEB731968E010F5F1F4FADB7A8
:100D7000BEB712961C930E9311972CE332E0338387
:100D8000228364837583868397830E9495BD2DB7E4
:100D90003EB7285F3F4F0FB6F8943EBF0FBE2DBF42
:100DA00087E0B8010E94388F81E00E946791ADB75B
:100DB000BEB718970FB6F894BEBF0FBEADBFEDB764
:100DC000FEB7319612961C930E93119726E432E0EB
:100DD0003383228364837583868397830E9495BDC2
:100DE0002DB73EB7285F3F4F0FB6F8943EBF0FBEFA
:100DF0002DBF88E0B8010E94388F82E00E94679181
:100E0000ADB7BEB718970FB6F894BEBF0FBEADBF53
:100E1000EDB7FEB7319612961C930E93119720E50D
:100E200032E03383228364837583868397830E94B1
:100E300095BD2DB73EB7285F3F4F0FB6F8943EBF24
:100E40000FBE2DBF89E0B8010E94388F83E040E4D7
:100E500052E46FE070E020E030E00AE515E0EE24B7
:100E6000FF240E942D15EC960FB6F894DEBF0FBE3E
:100E7000CDBFCF91DF911F910F91FF90EF9008951B
:100E8000AF92BF92CF92DF92EF92FF920F931F9398
:100E9000CF93DF938AE592E00E9460BDC3E2D6E083
:100EA00043E8E42E43E0F42E37E6A32E32E0B32EDF
:100EB000E881F981108100D000D000D0EDB7FEB7F5
:100EC0003196ADB7BEB71296BC92AE921197F3822F
:100ED000E282148315820E9424BD07E08DB79EB77D
:100EE00006960FB6F8949EBF0FBE8DBFC12EDD24AF
:100EF000C601002E02C0959587950A94E2F780FD01
:100F000003C080E390E002C081E390E06091793912
:100F100070917A390E94F8BC015050F785E792E051
:100F20000E9460BD2296A0E1B0E0EA0EFB1EB6E092
:100F3000C737DB0709F0BCCF85E792E00E9460BDB0
:100F4000DF91CF911F910F91FF90EF90DF90CF90A5
:100F5000BF90AF9008953F924F925F926F927F92B1
:100F60008F929F92AF92BF92CF92DF92EF92FF92B9
:100F70000F931F93DF93CF93CDB7DEB7A2970FB632
:100F8000F894DEBF0FBECDBF809104169091051678
:100F90000197909305168093041601969F70892BF4
:100FA00011F46A9A629A789480E090E00E94C40FEB
:100FB000182F8F3F09F46CC58B3121F080910616F4
:100FC0008823D1F180915538882329F080E090E082
:100FD0000E94EB9F5DC580910616882311F481E085
:100FE00005C0813031F41B3521F582E0809306166F
:100FF0004FC58230F1F410920616113409F048C53D
:1010000000D000D086E792E0ADB7BEB712969C93B1
:101010008E93119787E096E114969C938E93139785
:101020000E9424BD1092CF160F900F900F900F903A
:101030002FC5109206162CC58091CF16883C50F40F
:101040006091793970917A39812F992787FD909530
:101050000E94F8BC8091CF16883C08F019C51D305D
:1010600019F01A3009F0FFC4E82FF0E0E053F94E10
:101070001082982F9F5F9093CF16809155388823C8
:1010800049F080ED96E10E94EB9F1092D0161092ED
:10109000CF168ACF8091D0168C3609F468C28D366F
:1010A00084F4843609F408C1853624F48C3409F0BC
:1010B000CEC36FC2853609F480C2893609F0C7C332
:1010C00013C0823709F450C283373CF48D3609F4DB
:1010D00055C3803709F0BBC376C2833709F4EFC02C
:1010E000843709F0B4C3A9C08091D116803729F4A0
:1010F00080ED96E10E946EA09FC400D089E792E047
:10110000EDB7FEB7928381830E9424BD8DB79EB751
:1011100008970FB6F8949EBF0FBE8DBFEDB7FEB710
:10112000319680E892E0ADB7BEB712969C938E934D
:1011300011978091692690916A26A0916B26B091B3
:101140006C2682839383A483B583809165269091D6
:101150006626A0916726B091682686839783A0872C
:10116000B1870E9424BD0F900F900F900F90EDB7A4
:10117000FEB731968AE992E0ADB7BEB712969C935E
:101180008E9311978091A307828313828091A40785
:101190009091A507958384830E9424BDEDB7FEB787
:1011A00036960FB6F894FEBF0FBEEDBF8091810357
:1011B00090918203892B51F400D086EB92E0ADB779
:1011C000BEB712969C938E93119707C000D08AECFD
:1011D00092E0EDB7FEB7928381830E9424BD0F9009
:1011E0000F90CE010196BE016C5F7F4FAE014E5F46
:1011F0005F4F0E9490A98DB79EB708970FB6F894DD
:101200009EBF0FBE8DBFEDB7FEB7319682EE92E066
:10121000ADB7BEB712969C938E9311978981828346
:1012200013828C81848315828A81868317820E942F
:1012300024BDEDB7FEB7389626C22091A4073091A1
:10124000A507FE0138968BE0DF011D928A95E9F72C
:1012500082E088873A872987933048F480ED96E1C9
:101260006AEF72E00E9434BC85E08093CF168091D3
:101270008103909182034091CF16BE01685F7F4F3A
:10128000892B51F485E090E09C878B87415082E068
:1012900021ED36E100E205C0415082E021ED36E16A
:1012A00003E2EE24E394E5E0CE2EAA24A39488245E
:1012B00083940E94563CC0C30E944007BDC38091E6
:1012C000D1168D3609F48FC08E363CF4833609F47E
:1012D00041C08B3609F038C16BC0833709F4C8C0F0
:1012E000843709F4FDC0803709F02EC182ED96E104
:1012F0000E94A38B9B838A8300D084E396E0EDB7A2
:10130000FEB7928381830E9436BD00D08FEF92E0BA
:10131000ADB7BEB712969C938E9311978A819B812D
:1013200014969C938E9313970E9424BD0F900F9058
:101330000F900F908E010E5F1F4F80E5B8010E9445
:10134000D73C80E50E94913B8EE090E062E070E047
:10135000A801C3C01A8282ED96E10E949EBA8A83D8
:1013600080E190E061E070E0AE014E5F5F4F0E946F
:101370001C1200D080E296E0EDB7FEB79283818325
:101380000E9436BD00D0EDB7FEB7319686E093E0FF
:10139000ADB7BEB712969C938E9311978A818283C4
:1013A00013820E9424BD0F900F9081E096E04AC204
:1013B00002ED16E163E1E62EF12CEC0EFD1EC801F4
:1013C0000E94438BD7018D937D010E5F1F4FB6E1C5
:1013D000023F1B07A1F784E190E060E170E0AE01FD
:1013E0004D5E5F4F7AC08091D216823771F481E0F2
:1013F00090E0909382038093810300D08DED95E07F
:10140000EDB7FEB7928381830FC08336C1F410928B
:1014100082031092810300D089EB95E0ADB7BEB78F
:1014200012969C938E9311970E9436BD0F900F9049
:1014300081E190E062E070E041E853E04EC002EDEF
:1014400016E15CE3E52E59E2F52EC8010E94438BBC
:10145000F70181937F010E5F1F4FF6E1023E1F07E8
:10146000A1F784E290E068E070E04CE359E235C017
:101470008091D216813321F581E08093C01B8DE5E8
:1014800060EC7BE10E94D73C87E760EC7BE10E9447
:10149000D73C80E860EC7BE10E94D73C82E860ECBE
:1014A0007BE10E94D73C0E94083D0E94083D81E8F4
:1014B0006CE279E20E94D73C83E86CE379E205C0F4
:1014C0001092C01B8DE560EC7BE10E94D73C83E16C
:1014D00090E061E070E040EC5BE10E941C12ACC265
:1014E0008091D2168437C9F40E943FA95B016C0138
:1014F00020E831E541E050E00E946DB67B018C01AF
:1015000083ED96E10E9406AA6A0D7B1D8C1D9D1D30
:101510006E197F09800B910B10C0853789F483ED1C
:1015200096E160E070E04AE050E00E9488B9611501
:1015300071058105910509F47FC20E9433A97CC21F
:1015400000D080EA95E074C100D087E895E0EDB75F
:10155000FEB7928381830E9436BD0F900F9080E08A
:1015600090E00E945A0568C20E948E0665C24EB184
:101570002091D116332727FD30952053304081E04C
:1015800090E002C0880F991F2A95E2F78C71842B96
:1015900012C04EB12091D116332727FD309520532C
:1015A000304081E090E002C0880F991F2A95E2F751
:1015B0008C71809584238EB93FC286ED90E06FEFE9
:1015C0000E9421C139C282ED96E169E073E00E9478
:1015D000ECBBFC01009709F4CDC08081843609F48E
:1015E00058C0803721F0813609F0C0C06CC00E941D
:1015F000C0AA8091810390918203892BF9F000D0D9
:101600008CE695E0ADB7BEB712969C938E9311977A
:101610000E9436BD0F900F900E9449A800D000D0C4
:101620002DE033E0EDB7FEB73283218394838383CB
:101630000E9424BD0F900F900F900F9000D08AE56C
:1016400095E0ADB7BEB712969C938E9311970E940A
:1016500036BD0F900F900E944EA800D000D000D051
:1016600022E133E0EDB7FEB732832183ADB7BEB7D9
:1016700013966D937D938D939C9316970E9424BD32
:10168000EDB7FEB736960FB6F894FEBF0FBEEDBFAE
:10169000D3C180E090E069E073E00E94ECBB0E945F
:1016A0009EBA182F0E9468A800D000D0EDB7FEB7F0
:1016B000319688E193E0ADB7BEB712969C938E93B6
:1016C0001197128340C080E090E069E073E00E94CF
:1016D000ECBB0E949EBA382E80E090E069E073E097
:1016E0000E94ECBB0E9406AA2B013C0180E090E026
:1016F00069E073E00E94ECBB0E9406AA4B015C010A
:1017000080E090E069E073E00E94ECBB60E070E094
:101710000E941AB86B017C01832DB301A2019501CF
:1017200084010E9479A88823E9F400D000D0EDB7A5
:10173000FEB731968BE293E0ADB7BEB712969C939D
:101740008E931197328213820E9424BD0F900F90C6
:101750000F900F900E9457A8AC018EE490E062E8D1
:1017600070E0BBCE00D083E495E06CC000D089E28D
:1017700095E05EC000D08FE095E064C082ED96E118
:1017800069E073E00E94ECBBFC01009709F457C0CC
:101790008081803759F1843721F0893609F045C0BE
:1017A0004BC180E090E069E073E00E94ECBB60E038
:1017B00070E04AE050E00E9488B96C837D838E839C
:1017C0009F830E9438A8882369F080ED90E064E050
:1017D00070E0AE014C5F5F4F0E941C1200D083E0AE
:1017E00095E026C000D081EF94E02CC080E090E02E
:1017F00069E073E00E94ECBB0E949EBA8A839B83DF
:101800000E942DA8882369F084ED90E062E070E0EA
:10181000AE014E5F5F4F0E941C1200D081EE94E03B
:1018200007C000D08BEC94E00DC000D083EB94E0B7
:10183000ADB7BEB712969C938E931197F9C000D0A6
:101840008BE994E0EDB7FEB792838183F1C000D0BD
:10185000EEE8F4E0ADB7BEB71296FC93EE931197A5
:101860000E9436BDEBE7F4E0ADB7BEB71296FC932D
:10187000EE9311970E9436BDE8E5F4E0ADB7BEB730
:101880001296FC93EE9311970E9436BDE9E4F4E0C2
:10189000ADB7BEB71296FC93EE9311970E9436BD7A
:1018A000E8E2F4E0ADB7BEB71296FC93EE93119761
:1018B0000E9436BDE3E1F4E0ADB7BEB71296FC93EB
:1018C000EE9311970E9436BDEDEEF3E0ADB7BEB7D3
:1018D0001296FC93EE9311970E9436BDE9ECF3E06B
:1018E000ADB7BEB71296FC93EE9311970E9436BD2A
:1018F000E0EAF3E0ADB7BEB71296FC93EE93119712
:101900000E9436BDEAE7F3E0ADB7BEB71296FC938E
:10191000EE9311970E9436BDE0E6F3E0ADB7BEB797
:101920001296FC93EE9311970E9436BDEFE2F3E01E
:10193000ADB7BEB71296FC93EE9311970E9436BDD9
:10194000E1E0F3E0ADB7BEB71296FC93EE931197CA
:101950000E9436BDEEEDF2E0ADB7BEB71296FC9335
:10196000EE9311970E9436BDE4EAF2E0ADB7BEB740
:101970001296FC93EE9311970E9436BDEAE6F2E0D0
:10198000ADB7BEB71296FC93EE9311970E9436BD89
:10199000E7E4F2E0ADB7BEB71296FC93EE93119771
:1019A0000E9436BDEBE1F2E0ADB7BEB71296FC93F4
:1019B000EE9311970E9436BD0F900F908091810396
:1019C00090918203892B69F000D0ECEDF1E0ADB786
:1019D000BEB71296FC93EE9311970E9436BD0F90FE
:1019E0000F9000D0EAECF1E0ADB7BEB71296FC93D1
:1019F000EE9311970E9436BDECE8F1E0ADB7BEB7AB
:101A00001296FC93EE9311970E9436BDE6E5F1E045
:101A1000ADB7BEB71296FC93EE9311970E9436BDF8
:101A2000E8E2F1E0ADB7BEB71296FC93EE931197E2
:101A30000E9436BD0F900F901092D0161092CF16C4
:101A400080915538882309F0AFCA00D0EEE3F3E067
:101A5000ADB7BEB71296FC93EE9311970E9424BDCA
:101A60000F900F90A1CA183051F4882309F49CCA32
:101A7000E82FF0E0E053F94E1082815006C0E82FC5
:101A8000F0E0E053F94E10838F5F8093CF168CCA3D
:101A9000A2960FB6F894DEBF0FBECDBFCF91DF91F7
:101AA0001F910F91FF90EF90DF90CF90BF90AF907C
:101AB0009F908F907F906F905F904F903F90089590
:101AC000CF92DF92EF92FF920F931F93DF93CF930A
:101AD000CDB7DEB72E970FB6F894DEBF0FBECDBFE1
:101AE0000E941E3D882311F00E9417120E94D616F4
:101AF000789481E00E943511882311F00E9417121A
:101B00000E94C98D8AB1806D8AB98BB1806C8BB906
:101B10005C988CE364E070E045E453E00E942A8E18
:101B200080E395E70E94191380E395E70E9419135B
:101B300080E395E70E9419130E944D9086EF9FE085
:101B40006DED7FE00E94ACBC00D000D000D0EDB7BE
:101B5000FEB731968AE493E0ADB7BEB712969C9378
:101B60008E9311978CE693E09383828388E793E0CA
:101B7000958384830E9424BDEDB7FEB736960FB6D9
:101B8000F894FEBF0FBEEDBF86ED90E00E9419C134
:101B9000893A09F0A4C000D082E796E0ADB7BEB79D
:101BA00012969C938E9311970E9436BD0F900F90C2
:101BB00080E090E060E170E041E050E023EA37E04F
:101BC0000E944E1280E090E061E170E042E050E05F
:101BD00021E833E00E944E1280E090E06EE070E079
:101BE00042E050E024EA37E00E944E1280E090E0AC
:101BF00068E070E046E050E02EE636E20E944E12C9
:101C000080E090E063E170E041E050E020EC3BE1F7
:101C10000E944E1280E090E064E170E040E150E00C
:101C20002CE239E20E944E1280E090E064E270E023
:101C300048E050E02CE339E20E944E1280E090E050
:101C40006CE470E042E050E02EEB3BE10E944E126B
:101C500080E090E06CE370E040E150E023E538E0A4
:101C60000E944E1280E090E06CE270E040E150E0B3
:101C700023E638E00E944E1280E090E060ED70E0D4
:101C800044E050E09E012D5F3F4F0E944E126B8159
:101C90007C818D819E810E9438A880E090E064ED77
:101CA00070E042E050E09E012F5F3F4F0E944E12D5
:101CB00089819A810E942DA880918103909182034D
:101CC000892B09F036C10E9457A89C0180E090E062
:101CD0006EE470E042E850E00E944E122AC100D04B
:101CE0008FE496E0EDB7FEB7928381830E9436BD04
:101CF00098E19093A3070F900F9080916D26882311
:101D000099F490936E2680EF80936F268FE98093ED
:101D1000702685EE809371260E940AB88093722601
:101D20000E940AB8809373268E01095F1F4F88E0D6
:101D3000D8011D928A95E9F781E08F8382E0888738
:101D400083E0898784E08A8785E08B8786E08C87BB
:101D500087E08D8781E090E060E070E048E050E04F
:101D600098010E944E1280E090E068E070E0A801C7
:101D70000E941C1280E190E061E070E043EA57E0CD
:101D80000E941C1280E090E061E170E042E050E0CF
:101D900021E833E00E944E128091810390918203EA
:101DA000029730F081E090E090938203809381036A
:101DB0008EE090E062E070E044EA57E00E941C127E
:101DC0008CE490E062E070E04EEB5BE10E941C125C
:101DD00088E090E066E070E04EE656E20E941C1259
:101DE0008CE390E060E170E043E558E00E941C1253
:101DF0008CE290E060E170E043E658E00E941C1243
:101E000083E190E061E070E040EC5BE10E941C1235
:101E10008091810390918203892B09F054C080E066
:101E200040E050E060E070E008E710E020E030E0E3
:101E30000F2EF0E0CF2EF0E0DF2EF0ECEF2EFFE3E0
:101E4000FF2EF02D0E9479A881E049E750E060E084
:101E500070E000EF10E020E030E00F2EFDECCF2E20
:101E6000FCECDF2EFCE4EF2EFEE3FF2EF02D0E94B3
:101E700079A882E041EF50E060E070E008E611E010
:101E800020E030E00F2EFDECCF2EFCECDF2EFCE44A
:101E9000EF2EFDE3FF2EF02D0E9479A883E049E6A6
:101EA00051E060E070E00FE711E521E030E00F2E37
:101EB000F0E0CF2EF0E0DF2EF0E0EF2EFFE3FF2E7C
:101EC000F02D0E9479A80E9457A8AC018EE490E002
:101ED00062E870E00E941C128CE390E0A0E0B0E0A9
:101EE0008B839C83AD83BE838CE390E09A8389834C
:101EF00080ED90E064E070E0AE014D5F5F4F0E94C6
:101F00001C1284ED90E062E070E0AE014F5F5F4F25
:101F10000E941C1289819A810E942DA86B817C816C
:101F20008D819E810E9438A886ED90E069EA0E942A
:101F300021C10E94228B81E00E94B13B80918103EC
:101F400090918203892B21F48EE696E20E94878A83
:101F500000D088E496E0EDB7FEB7928381830E94BB
:101F600036BD8EB18C618EB98DB18C618DB90F90FB
:101F70000F900E94A8AE0E94083D0E94AB070E94ED
:101F80004D900E9417ADF7CFDF93CF930F92CDB74F
:101F9000DEB781E0BE016F5F7F4F41E00E942311F9
:101FA000813019F02FEF3FEF03C08981282F30E0F7
:101FB000C9010F90CF91DF9108950F931F93DF9385
:101FC000CF930F92CDB7DEB78E010F5F1F4F81E029
:101FD000B80141E00E9423118823C9F3898190E070
:101FE0000F90CF91DF911F910F9108950F931F9341
:101FF000DF93CF930F92CDB7DEB789838A3071F428
:102000008DE089838E010F5F1F4F81E0B80141E0B1
:102010000E942C118823C9F38AE089838E010F5F07
:102020001F4F81E0B80141E00E942C118823C9F3C1
:1020300080E090E00F90CF91DF911F910F91089574
:102040009B01AC016050774F824C9F4FF2E0660FCE
:10205000771F881F991FFA95D1F7E3E0220F331FEE
:10206000441F551FEA95D1F70E946DB621503040AC
:102070003093CD002093CC0082E08093C80086E0AE
:102080008093CA0088ED8093C9000895DC01809197
:10209000C9008F7B8093C9002091BA268091BB260E
:1020A000821730F0275F922F981B892F295005C087
:1020B0002150922F981B892F2F5F482F681708F403
:1020C000462F342F12C09091BB26E92FF0E0EA553D
:1020D000F94D8C918083993019F41092BB2603C07E
:1020E0009F5F9093BB2631501196332361F7809107
:1020F000BE26882351F4E22FF0E0EA55F94D8081A5
:102100008093CE0081E08093BE268091C9008064D8
:102110008093C900842F0895DC012091BF262223DB
:1021200011F480E008958091C9008F778093C900F1
:102130002A3058F08091BD268093BC268AE0809397
:10214000BF266A3020F02AE003C0261708F0262FA9
:10215000322F17C0E091BC26F0E0EA55F94D828598
:102160008C939091BC269F5F9093BC268091BF2654
:1021700081508093BF269A3011F41092BC2611969C
:102180003150332339F78091C90080688093C900AA
:10219000822F08951F920F920FB60F920BB60F92D7
:1021A00011248F939F93EF93FF939091BD2680917D
:1021B000BF268F5F8093BF268091CE00E92FF0E08D
:1021C000EA55F94D8287993019F41092BD2603C063
:1021D0009F5F9093BD26FF91EF919F918F910F90FC
:1021E0000BBE0F900FBE0F901F9018951F920F926D
:1021F0000FB60F920BB60F9211248F93EF93FF93AC
:102200008091BA26893019F41092BA2603C08F5FE4
:102210008093BA26E091BA268091BB26E81739F060
:10222000F0E0EA55F94D80818093CE0002C0109213
:10223000BE26FF91EF918F910F900BBE0F900FBEB6
:102240000F901F901895813011F080E00895CB0118
:10225000642F0E948C100895813011F080E0089561
:10226000CB01642F0E9446100895813011F085E85B
:10227000089560E076E980E090E00E94201080E020
:1022800008959093991780939817089590939B17AA
:1022900080939A17089590939D1780939C170895A3
:1022A0001F920F920FB60F920BB60F9211242F931D
:1022B0003F934F935F936F937F938F939F93AF93CE
:1022C000BF93EF93FF93E0919817F09199170995B9
:1022D000FF91EF91BF91AF919F918F917F916F91FE
:1022E0005F914F913F912F910F900BBE0F900FBEBA
:1022F0000F901F9018951F920F920FB60F920BB66A
:102300000F9211242F933F934F935F936F937F937B
:102310008F939F93AF93BF93EF93FF93E0919A179F
:10232000F0919B170995FF91EF91BF91AF919F910C
:102330008F917F916F915F914F913F912F910F906E
:102340000BBE0F900FBE0F901F9018951F920F920B
:102350000FB60F920BB60F9211242F933F934F930A
:102360005F936F937F938F939F93AF93BF93EF93FD
:10237000FF93E0919C17F0919D170995FF91EF91C4
:10238000BF91AF919F918F917F916F915F914F918D
:102390003F912F910F900BBE0F900FBE0F901F908B
:1023A00018951F920F920FB60F9211240F900FBE27
:1023B0000F901F9018951F920F920FB60F92112435
:1023C0000F900FBE0F901F9018951F920F920FB68F
:1023D0000F9211240F900FBE0F901F9018951F920F
:1023E0000F920FB60F9211240F900FBE0F901F90F7
:1023F00018951F920F920FB60F9211240F900FBED7
:102400000F901F9018951F920F920FB60F921124E4
:102410000F900FBE0F901F9018951F920F920FB63E
:102420000F9211240F900FBE0F901F9018958FEFF1
:102430009FEF0E941913FBCFCF92DF92EF92FF9292
:102440000F931F93CF93DF938C017B016A01CB0124
:10245000800F911F8150904110F085E816C0C0E0B8
:10246000D0E00FC0C8010E9419C1F601EC0FFD1F9A
:102470006081861719F0C8010E9421C10F5F1F4FAC
:102480002196CE15DF0570F380E0DF91CF911F918B
:102490000F91FF90EF90DF90CF900895CF92DF9251
:1024A000EF92FF920F931F93CF93DF938B017A01EB
:1024B00069018130910531F4862F642FA9010E94B2
:1024C000DB161DC0892B11F088EE19C0CA01860FDA
:1024D000971F8150904110F085E811C0C0E0D0E016
:1024E0000AC0CE01800F911F0E9419C1F601EC0FA6
:1024F000FD1F80832196CE15DF0598F380E0DF91E4
:10250000CF911F910F91FF90EF90DF90CF900895A2
:102510000E94F71408950E9493120E94D8160E94F8
:10252000B41280E008959FB7F894E0E0F0E089E00D
:102530008093570084919FBF8F70823011F090E09C
:1025400001C09FE080E80FB6F894809361009093FB
:1025500061000FBE80E18093350180933401809348
:10256000330180933201089510929E1710929F17A5
:102570008FEF8093A0178093A1178093A217E4ECAC
:10258000F6E29FEF948311821082399687E2E63655
:10259000F807C1F780E28093B60088EA8093DC00F8
:1025A0008FE08093F4009093F3009093F200909367
:1025B000F10082E08093E0008091DF0082608093F0
:1025C000DF0008950895FC018091DE0080FDFCCFBE
:1025D0002091E100822F2091E200922F2091E300D0
:1025E000A22F2091E400B22F24E0880F991FAA1F88
:1025F000BB1F2A95D1F780839183A283B38308956B
:10260000FC012091E900822F2091EA00922F209175
:10261000EB00A22F2091EC00B22F34E0880F991F1D
:10262000AA1FBB1F3A95D1F780839183A283B383FE
:102630000895AC018436910518F060E070E01EC08A
:102640007FB7F89461E01AC057FD02C09A0102C03A
:102650002FEF3FE7C901880F991F909581959F4FF4
:102660009093250180932401FABBE0932101D09B34
:10267000FECF421B530B1092210102C0F1E0E2E0B9
:102680004115510509F761117FBF089520E090E0E1
:10269000FC01B3E0EE0FFF1FBA95E1F7E80FF91F59
:1026A000E054F94D84819581892B09F021E0822F36
:1026B0000895EF92FF920F931F938091A01790E0DF
:1026C000FC0113E0EE0FFF1F1A95E1F7E80FF91F69
:1026D000E054F94DE080F1800281138180919E17D2
:1026E000882309F449C01093F8000093F700F09292
:1026F000F600E092F5008091DF0080FD08C081E0E7
:102700008093E0008091DF0081608093DF00209162
:10271000E100822F2091E200922F2091E300A22F6E
:102720002091E400B22F9C01AD012F5F3F4F4F4F2E
:102730005F4FDA01C9018E259F25A027B127807040
:102740009070A070B87F0097A105B10531F4E21632
:10275000F30604071507B0F018C08FEF9FEFAFEF37
:10276000B7E0E822F9220A231B2357702E153F05F4
:102770004007510738F009C08091DF008E7F8093B9
:10278000DF0003C081E080939F171F910F91FF909E
:10279000EF9008951F931FB7F89480919F17882397
:1027A00009F44CC010929F1730919E17332309F4FF
:1027B00045C08091A1178F3F59F48091A2178F3F98
:1027C00039F48091A0178093A2178093A11712C0AB
:1027D0002091A0178091A21790E0FC0153E0EE0F2A
:1027E000FF1F5A95E1F7E80FF91FE054F94D2087D4
:1027F0002093A2178091A01790E0FC0143E0EE0F18
:10280000FF1F4A95E1F7E80FF91FE054F94D808565
:102810008093A0178091A21790E0FC0123E0EE0FB7
:10282000FF1F2A95E1F7E80FF91FE054F94D8FEFEC
:102830008087315030939E170E9459131FBF1F91FC
:102840000895FF920F931F93182F823110F08AE89A
:10285000C5C0FFB6F8940E94CA1300919E170023CA
:1028600009F4C0C04091A017242F842F302F1217D5
:10287000F1F5212F30E0141781F4F901A3E0EE0FF8
:10288000FF1FAA95E1F7E20FF31FE054F94D808591
:102890008093A0170E94591318C090E0DC01E3E078
:1028A000AA0FBB1FEA95E1F7A80FB91FA054B94DB5
:1028B000F90173E0EE0FFF1F7A95E1F7E20FF31FC6
:1028C000E054F94D808518968C93812F90E0FC019F
:1028D00063E0EE0FFF1F6A95E1F7E80FF91FE05480
:1028E000F94D8FEF8087015000939E1762C0822FB1
:1028F00090E0FC0153E0EE0FFF1F5A95E1F7E80F5F
:10290000F91FE054F94D50853150822F09F46AC007
:10291000252FADCF1217D1F52091A2171317B1F4BF
:10292000121721F48FEF8093A2170DC0812F90E032
:10293000FC0143E0EE0FFF1F4A95E1F7E80FF91F96
:10294000E054F94D80858093A11733C0842F90E027
:10295000DC0133E0AA0FBB1F3A95E1F7A80FB91FBE
:10296000A054B94D812F90E0FC0103E0EE0FFF1F52
:102970000A95E1F7E80FF91FE054F94D80851896A4
:102980008C931217B1F44093A21713C0822F90E0DA
:10299000FC0173E0EE0FFF1F7A95E1F7E80FF91FD6
:1029A000E054F94D422F20852F3F09F0B3CF80E04E
:1029B0000FC0812F90E0FC0163E0EE0FFF1F6A95CE
:1029C000E1F7E80FF91FE054F94D1582148281E018
:1029D000FFBE882311F489E801C080E01F910F91A8
:1029E000FF9008953091A117232F432FDDCF1F9320
:1029F0000E94CA131FEF25C06FB7F894822F90E092
:102A0000FC01B3E0EE0FFF1FBA95E1F7E80FF91FE5
:102A1000E054F94D20854481558186819781108746
:102A200015821482178216822F3F09F43FEF6FBF81
:102A30004115510551F03093A2172093A117FA01C7
:102A400009953091A2172091A1172F3FA9F6309335
:102A5000A2172093A1171F9108952F923F924F9292
:102A60005F926F927F928F929F92AF92BF92CF921E
:102A7000DF92EF92FF920F931F93DF93CF9300D0DB
:102A800000D00F92CDB7DEB7582E1801FB82EA8234
:102A900001E1081710F48AE820C12114310409F477
:102AA00019C190E09D838C83FC01A3E0EE0FFF1F12
:102AB000AA95E1F7E80FF91FE054F94D848195815B
:102AC000892B11F088E809C1E4E076956795579560
:102AD0004795EA95D1F72115310529F021303105C7
:102AE00009F0F8C026C0DB01CA010897A109B109A5
:102AF000885F9F4FAF4FB74008F0EEC02091E100D4
:102B0000822F2091E200922F2091E300A22F2091AA
:102B1000E400B22F7A018B01E80EF91E0A1F1B1F79
:102B20008FEF9FEFAFEFBFE0E822F9220A231B23CC
:102B300020C02091E100822F2091E200922F20916D
:102B4000E300A22F2091E400B22F8A019B01081B11
:102B5000190B2A0B3B0BD901C801BF700897A109BB
:102B6000B109885F9F4FAF4FB74008F0B5C07A01F9
:102B70008B012FB72983F8946FEF862E6FEF962E77
:102B80006FEFA62E6FE0B62E8E209F20A022B122DE
:102B90000E94CA136090A0173FEF631671F0409037
:102BA0009E17C62CD62C77248FEF9FEFAFEFB7E0A0
:102BB000E822F9220A231B2367C05092A017EC8158
:102BC000FD8153E0EE0FFF1F5A95E1F7AC81BD8107
:102BD000EA0FFB1FE054F94D60865AC0BFEFDB16C9
:102BE00009F44DC06D2D70E0FB0143E0EE0FFF1FB7
:102BF0004A95E1F7E60FF71FE054F94D2081318146
:102C000042815381D501C40182279327A427B52788
:102C100080709070A070B87F0097A105B10539F45D
:102C2000281539054A055B0508F46FC007C05770C1
:102C3000E216F3060407150708F467C0EC81FD816E
:102C400033E0EE0FFF1F3A95E1F70C811D81E00F95
:102C5000F11FE054F94DD0866D1419F45092A0176D
:102C600017C08C2D90E0FC0123E0EE0FFF1F2A958A
:102C7000E1F7E80FF91FE054F94D508609C08FEFD6
:102C8000DC2C7394CD2CD82E741408F4A7CF49C033
:102C9000EC81FD8193E0EE0FFF1F9A95E1F72C8107
:102CA0003D81E20FF31FE054F94D80829182A282B0
:102CB000B382358224828A819B8197838683809127
:102CC0009E178F5F80939E170E94591399819FBF13
:102CD00080E003C088EE01C08BE80F900F900F904A
:102CE0000F900F90CF91DF911F910F91FF90EF9078
:102CF000DF90CF90BF90AF909F908F907F906F901C
:102D00005F904F903F902F900895FB0183E0EE0F6E
:102D1000FF1F8A95E1F7E60FF71FE054F94D808514
:102D2000B0CF8C2D90E0FC0103E0EE0FFF1F0A9561
:102D3000E1F7E80FF91FE054F94D5086EC81FD8171
:102D400013E0EE0FFF1F1A95E1F7AC81BD81EA0F8A
:102D5000FB1FE054F94D8FEF80879ACF1F920F929F
:102D60000FB60F9211248F9380919E17882319F02C
:102D700081E080939F178F910F900FBE0F901F904F
:102D800018951F920F920FB60F9211248F938FEF09
:102D90008093E4008093E3008093E2008093E1005D
:102DA0008F910F900FBE0F901F90189581E008959E
:102DB000A59A9D9A0895DF93CF93CDB7DEB7C054FF
:102DC000D0400FB6F894DEBF0FBECDBFA82FB62FF0
:102DD000749A759A6C9A6D9A5E9A5F9A569A579AF7
:102DE000A2989A9AA5989D9A84B1876084B983E540
:102DF0008CBDFE0131966E2F93E09E01205C3F4F0B
:102E00008E2F861BA5980000000000000000000027
:102E100000000000000000000000000000000000B2
:102E20000000000000009EBD0DB407FEFDCF8F77AF
:102E30008EBD0DB407FEFDCF1EBC0DB407FEFDCF49
:102E40008EB5A59A8083E217F30711F03196D8CF9B
:102E50001CBCFE01319620E030E0BE016F5B7F4F6D
:102E600081912827022E2295207F2025032E322FA4
:102E700022952F700226269532272327220F220F14
:102E8000220F2025E617F70759F7232B11F085E8C5
:102E90000CC09E012F5F3F4F2A0F311DCA01B9019F
:102EA0004B2F50E00E94FEBB80E0C05CDF4F0FB6AE
:102EB000F894DEBF0FBECDBFCF91DF910895BC0166
:102EC000009721F089E69BE10E949617089589E614
:102ED0009BE160E070E00E94331808950F931F9308
:102EE000CF93DF9389E69BE166E00E948E17C1E5F0
:102EF000DBE103EA17E11983088389E69BE1BE0160
:102F00000E949617249603561F4F8BE1C936D807A7
:102F100091F7DF91CF911F910F910895FC011182DC
:102F2000108213821282158264830895CF93DF93F7
:102F3000DC01EB012FB7F89415969C911597149628
:102F40008C911497981711F48CE819C0992321F4E7
:102F500011967C936E9306C01296ED91FC91139797
:102F6000738362831396DC93CE9312971B821A822B
:102F700015968C9115978F5F15968C9380E02FBFD7
:102F8000DF91CF9108959F92AF92BF92CF92DF923F
:102F9000EF92FF920F931F93CF93DF938C015B010E
:102FA0006A019FB6F894DC0115968C91882319F478
:102FB000C0E0D0E04AC0F801C081D181411551057F
:102FC000B1F07E0111C0D60112966D917C911397DC
:102FD000ED91FC91888199810995882359F47E01AE
:102FE0008A819B819C01E901209769F72EC0209777
:102FF00061F17E01AB2849F5F801808191812A8138
:103000003B81C817D90719F43183208305C0D70144
:1030100013963C932E931297F80182819381C817DF
:10302000D90711F4F382E282D80115968C91159795
:10303000815015968C9315978D919C911197892BA2
:1030400021F413961C921E9212979FBECE01DF911F
:10305000CF911F910F91FF90EF90DF90CF90BF9095
:10306000AF909F900895AB0160E070E00E94C3179D
:103070000895AB0161E070E00E94C3170895CF93FB
:10308000DF93EC010BC0CE0160E070E00E943318CA
:10309000009711F41D8205C00E945F178D8188235F
:1030A00091F7DF91CF9108950F931F93DF93CF9303
:1030B000CDB7DEB728970FB6F894DEBF0FBECDBFF1
:1030C000809141018F71883029F581E080934F0113
:1030D00089E080934201CE0101960E94E3128E01A5
:1030E0000B5F1F4F80914F0180FD14C0C8010E94EB
:1030F000E3128D819E81AF81B88529813A814B8110
:103100005C81821B930BA40BB50B8D3D9105A10532
:10311000B10540F328960FB6F894DEBF0FBECDBFC1
:10312000CF91DF911F910F910895CF93DF93EC0121
:1031300080918327909184270F9709F033C0809165
:1031400039018D7F8093390194E6809141018F711F
:103150008830C9F0915031F48091390182608093B8
:103160003901EDCF00000000000000000000000069
:10317000000000000000000000000000000000004F
:1031800000000000E2CFC830D10519F0C330D105EE
:1031900049F488E090E0909384278093832728E087
:1031A00030E0E1C18091410190E08F719070909387
:1031B000842780938327C830D10509F44FC0C930D4
:1031C000D10560F4C430D10509F49AC0C630D105E8
:1031D00009F4A3C0239709F0B9C157C0CF30D10576
:1031E00079F0C031D10520F4299709F0AFC164C04E
:1031F000C631D10509F4CBC0699709F0A7C136C122
:1032000083E0809342010E940AB880936D0180910F
:103210006E019770887F982B90936E0100000000DC
:10322000000000000000000000000000000000009E
:103230000000000000000000000000008091390143
:1032400082608093390183E290E00E941913D09349
:103250008427C09383272FE030E085C1089709F4C5
:1032600075C188E08093420100000000000000006A
:10327000000000000000000000000000000000004E
:10328000000000000000000061C1089709F45EC161
:1032900083E0809342010000000000000000000075
:1032A000000000000000000000000000000000001E
:1032B0000000000000004AC18830910539F18930D2
:1032C000910520F4069709F041C106C086319105A9
:1032D00019F0499709F03AC189E080934201000052
:1032E00000000000000000000000000000000000DE
:1032F000000000000000000000000000000026C1E7
:103300008830910519F0099721F420C10E945418C2
:103310001DC184E08093420119C18930910569F093
:103320008A30910520F4089709F010C11AC086313F
:10333000910519F0499709F009C186E0809342018F
:10334000000000000000000000000000000000007D
:10335000000000000000000000000000000000006D
:10336000F5C00E94541886E08093420100000000DE
:10337000000000000000000000000000000000004D
:10338000000000000000000000000000DFC08830E6
:10339000910509F18930910520F4069709F0D6C00E
:1033A00030C08930910519F0499709F0CFC086E106
:1033B00080934201000000000000000000000000B7
:1033C00000000000000000000000000000000000FD
:1033D00000000000BBC00E94541886E180934201A7
:1033E00000000000000000000000000000000000DD
:1033F00000000000000000000000000000000000CD
:10340000A5C089E080934201000000000000000098
:1034100000000000000000000000000000000000AC
:10342000000000000000000080914101282F30E0E2
:103430002F713070309384272093832729303105F2
:1034400009F091C086E18093420100000000000075
:10345000000000000000000000000000000000006C
:103460000000000000000000000070C088309105DE
:1034700009F457C08930910520F4069709F066C019
:103480001BC08930910521F0469709F05FC014C038
:1034900089E180934201000000000000000000006C
:1034A000000000000000000000000000000000001C
:1034B0000000000000004AC089E080934201000043
:1034C00000000000000000000000000000000000FC
:1034D00000000000000000000000000000008091DB
:1034E0004101282F30E02F713070309384272093D2
:1034F00083272930310509F036C089E180934201E4
:1035000000000000000000000000000000000000BB
:1035100000000000000000000000000000000000AB
:1035200015C00E94541889E18093420100000000F8
:10353000000000000000000000000000000000008B
:103540000000000000000000000000008091410128
:10355000282F30E02F7130702F313105B9F32093CF
:10356000832730938427C901DF91CF9108958091FB
:103570006F1B9091701B892BA9F48DE90E9467172E
:103580009093701B80936F1B892B61F08091732740
:10359000882341F080918D27882321F486E190E0F3
:1035A0000E94951880917927882351F084E797E24B
:1035B00060E070E00E943318009711F00E94E91A51
:1035C00080918D27882321F0823011F40E94341CD1
:1035D0000895EF92FF920F931F93CF93DF937C0197
:1035E000DC010D911C91D8011696ED91FC91179775
:1035F000808180938627C82FD0E02196CE0FDF1FD1
:10360000988129812D3310F02CE303C0222309F483
:1036100021E092959695969593708FEF989FC001B3
:10362000112430E0FC01E29FC001E39F900DF29F66
:10363000900D112464EB70E00E9446B66F3F710557
:1036400011F008F06FEF6883D8011296FC92EE92A9
:103650001197C8010E94A525DF91CF911F910F916D
:10366000FF90EF900895CF92DF92EF92FF920F9329
:103670001F93CF93DF93E0916F1BF091701BC0817C
:10368000D181C0904701D0907B01D7FC34C082E04B
:10369000D80E0DE910E00D191109EEEFDE0E0C0F3A
:1036A0001D1FED2CFF2497012F5F3F4FC80160E8DD
:1036B00071E0A9010E94FEBBF801D292FF83EE8364
:1036C000EE0EFF1EF701C28260916F1B7091701B9E
:1036D00084E797E20E9496178DE90E9467179093FE
:1036E000701B80936F1B892B31F489E0809342011A
:1036F00081E080937327DF91CF911F910F91FF900D
:10370000EF90DF90CF90089580918D278823F1F07E
:10371000809142018295869587708093711B1092EB
:10372000721B82E080938D2780916F1B9091701B9C
:10373000892B41F489E090E00E94951881E0809304
:103740007327089586E190E00E9495180895FF92EE
:103750000F931F93CF93DF93EC018B01442349F028
:1037600090916C01809182278295807F9F70892B38
:1037700003C080916C018F7080936C010230110541
:1037800098F4442369F090916C0180917A27880F16
:103790008E70917F892B80936C0110926F0117C0FE
:1037A00080916C018E6011C080917E278295807F10
:1037B00090918127892B80936F0190916C0180916A
:1037C0007A27880F8E70917F892B80936C0189E115
:1037D00090E00E9495184997D1F7FFB6F894013010
:1037E000110559F480918627833118F080E492E026
:1037F00002C080E890E00E94191380913901826034
:1038000080933901809139018D7F8093390128811E
:1038100030E02150304080E891E0BE01A9010E94D3
:10382000FEBB81E080938D27FFBEDF91CF911F917A
:103830000F91FF900895FC0180918D27882311F04E
:1038400086E80895F0938027E0937F27868197810B
:103850009093882780938727009711F488EE089526
:103860000E94A71B80E0089510928D278091711B04
:103870009091721B83309105B9F08430910528F442
:10388000009731F00197E1F409C00597C9F412C01F
:1038900060917F277091802780E017C060917F271B
:1038A0007091802787E811C060917F2770918027F1
:1038B00081EE0BC060917F277091802789EE05C053
:1038C00060917F277091802785E80E942D360895AA
:1038D000282F85FD03C0982F9F7304C0982F9195C2
:1038E0009F719195E1E8F6E08491891734F03F9655
:1038F0008491981714F0822F0CC0803E3CF08032E7
:103900003CF487FF06C08F71806203C080E201C073
:103910008FE18068089584E080937A2723E02093E4
:1039200081278FEF9FEF90936F2780936E2790935F
:103930007227809371278BE080937C2710926D27EC
:1039400080E098EFAFEFB7E08093892790938A27C4
:10395000A0938B27B0938C278AE091E090936C27FB
:1039600080936B278AE08093852782E080937B2772
:1039700085E080937E272093822783E80E94681C3D
:103980008093622781E08093702710927D270895AD
:1039900085FD03C0982F9F7304C0982F91959F7148
:1039A0009195E1E8F6E080E02491921724F0291740
:1039B0003CF4815008958F5F31968031A9F780E003
:1039C000089580916E2790916F2780936201909364
:1039D0006301E3E6F7E2A4E6B1E081918D9387E22B
:1039E000EB36F807D1F78091712790917227809379
:1039F00060019093610190914801809170278295B8
:103A0000880F80769F79892B8093480190916F0170
:103A1000809181278F70907F892B80936F01909187
:103A20006E0180917D27880F880F880F8870977F9F
:103A3000892B80936E0190916F0180917E278295F2
:103A4000807F9F70892B80936F01909148018091B6
:103A50007C278F71907E892B80934801809162270B
:103A60000E94C81C909145018F70907F892B809394
:103A700045010895CF93DF93EB018E3431F0893502
:103A800041F4888180938227EFC0888180937A27D0
:103A9000EBC020918327309184272F30310511F41A
:103AA00081E8E3C08B3009F4CDC08C3070F48230F3
:103AB00009F487C0833018F48823B1F115C083302E
:103AC00009F490C0843081F466C0833511F18435E7
:103AD00028F48F3459F0803539F410C0873509F453
:103AE00064C0803F09F48BC084EFBFC0988190937D
:103AF000812780916F019F70807F5FC0888199814D
:103B000080936E2790936F27809362019093630157
:103B1000ABC088819981809371279093722780939D
:103B2000600190936101A0C080918D27882309F0E6
:103B300097C080E098EFAFEFB7E0088004C0B6957B
:103B4000A795979587950A94D2F781709070892BE5
:103B500009F488C02830310519F428E030E008C0A5
:103B600088E090E00E9495180897D1F726E130E0B0
:103B7000988190937C27809148019F71807E982B3B
:103B8000909348012830310509F46EC086E190E039
:103B90000E94951869C080918D27882309F060C024
:103BA0008881882309F460C05DC0988190937E2746
:103BB00080916F019295907F8F70982B90936F01F9
:103BC00053C08881809362270E94681C809362277B
:103BD0000E94C81C909145018F70907F892B809323
:103BE000450142C088818093702790914801829559
:103BF000880F80769F79892B8093480135C0888112
:103C0000809363278981809364278A8180936527C5
:103C10008B81809366278C81809367278D81809329
:103C200068278E81809369278F8180936A27E3E6D6
:103C3000F7E2A4E6B1E081918D9387E2EB36F807D5
:103C4000D1F712C0888180937D2790916E01880FF3
:103C5000880F880F8870977F892B80936E0104C02E
:103C600086E803C088EE01C080E0DF91CF9108951F
:103C7000DF93CF930F92CDB7DEB781E090E065E19F
:103C800070E041E050E09E012F5F3F4F0E944E12D6
:103C9000809139018D7F8093390180EF90E00E94FF
:103CA0001913809139018E7F8093390181E090E072
:103CB0000E9419138091390181608093390120E0BD
:103CC00030E0809141012F5F3F4F93E0293E39075B
:103CD00011F485E815C090E08F71907088309105DF
:103CE00081F790938427809383279981992339F0D2
:103CF000809152019F70807F982B9093520180E0B9
:103D00000F90CF91DF9108950E940AB880936D01C2
:103D1000EEE6F1E080819770887F982B908380E0B9
:103D20000E941B200E9409200895882311F00E9400
:103D30008B1C0E94381E882311F085E8089580911D
:103D40006E01806280936E018CE480934E010E942C
:103D5000841E80917927882359F40EC084E797E266
:103D600060E070E00E943318009711F00E945F1726
:103D700080917927882391F70E94E11C10928D276A
:103D80001092732788E080934F0180E480934F0165
:103D900084E080934F010E94263D80E008950F93B8
:103DA0001F93CF93DF930E948B12882309F00CC1DD
:103DB00080913901816080933901809139018D7F33
:103DC000809339018CE791E00E94191380913901A9
:103DD0008E7F8093390181E090E00E9419138091D9
:103DE000390181608093390188E08093420120E0AD
:103DF00080914101215009F4E7C090E08F719070EB
:103E000088309105A9F79093842780938327809128
:103E10005C01833809F0D8C0DDC080916E018062FA
:103E200080936E018CE480934E0186E090E00E94C6
:103E3000951810924E01C0E0D0E010E0809146014C
:103E4000CC0FDD1FCC0FDD1F90E08076907025E059
:103E5000969587952A95E1F7C82BD92B1F5F1830C7
:103E600069F783E090E00E94951880914F011093CC
:103E70004F0180E480934F018CE480934E01CE018A
:103E80000E940FB80E94841E09C0C3E6D7E20E94B8
:103E90000AB8899387E2CB36D807C9F780916327A0
:103EA000309164274091652760916627709167275C
:103EB000F0916827B091692750916A27082F015027
:103EC00091E0081708F090E0832F815021E08317DC
:103ED00008F020E0192F180F91E0181708F090E073
:103EE000292B842F815031E0841708F030E0A22F75
:103EF000A80F91E0A81708F090E0392B862F815089
:103F000021E0861708F020E0E32FE80F91E0E817A2
:103F100008F090E0292B872F815031E0871708F0B7
:103F200030E0622F680F91E0681708F090E0392BBD
:103F30008F2F815021E08F1708F020E0432F480F8A
:103F400091E0481708F090E0292B8B2F815091E0E9
:103F50008B1708F090E0322F380F21E0381708F067
:103F600020E0922B5195591779F43F3F69F44F3F68
:103F700059F46F3F49F4EF3F39F4AF3F29F41F3F45
:103F800019F40E3F08F081CF81E090E20E944611C3
:103F900089EF9FE10E9441110E946E178DE90E94F6
:103FA00067179093701B80936F1B84E797E265E01F
:103FB0000E948E170E948B1C0E94E11C10928D277C
:103FC0001092732780E001C085E8DF91CF911F91A7
:103FD0000F91089580E090E060E070E048E050E0EC
:103FE00023E637E20E944E120E94381E882361F7B2
:103FF00014CF1F931FB7F8940E94841B1FBF1F91FB
:1040000008951F931FB7F8940E94331B1FBF1F9181
:10401000089580918327909184270F9711F082E86B
:10402000089588E090E00E949518089711F085E8BF
:10403000089580E00895882311F088EE0895809116
:104040008327909184270F9711F481E80895809138
:104050008D27882391F41092732788E090E00E94C6
:1040600095180897D1F78FE090E00E9495180F9768
:1040700021F40E94263D80E0089586E80895982F57
:1040800080918D27882311F086E80895983041F4B7
:1040900088E090E00E9495181092732788E00895B8
:1040A00080916F1B9091701B892B31F086E190E01D
:1040B0000E94951886E0089581E08093732786E03A
:1040C0000895CF93DF93DC019C9111962C91119769
:1040D00080918E27882321F4CD010E945F171AC09A
:1040E000E92FF22F9F012F5F3F4F41E558E288E013
:1040F000EA010990AE01E90109929E018150C1F7E0
:1041000080916328818783E1808387EB98E2BD01FA
:104110000E949617DF91CF910895DC01ED91FC91FB
:10412000119784E1808363835283418387EB98E214
:10413000BD010E94961708950F931F93DF93CF93AD
:1041400000D0CDB7DEB7A091F127B091F227ED9165
:10415000FC91119784E180838BEE83830FEF1FEF37
:104160001283018387EB98E2BD010E94961710929B
:10417000DF271A83098380E5BE016F5F7F4F0E94AE
:104180005830109328280093272810923628109230
:104190003728109238281092392810923A28109215
:1041A0003B2810923C2810923D280E94A22E0F908E
:1041B0000F90CF91DF911F910F910895EF92FF9291
:1041C0000F931F93E0903228F090332880E061E055
:1041D00040E020E030E000E010E00E94CF2888239B
:1041E000A9F4A091F127B091F227ED91FC911197DC
:1041F00084E1808381EE83838FEF9FEF92838183BD
:1042000087EB98E2BD010E94961719C0A70160E0F4
:1042100070E084E0440F551F661F771F8A95D1F721
:1042200080E020E030E00CE910E2EE24FF240E9460
:104230002D15882321F080E090E00E949C201F91A2
:104240000F91FF90EF900895FF920F931F93DF93CC
:10425000CF9300D0CDB7DEB7F09065280E945F17EE
:10426000FF20B1F583E563E678E20E9458302091A3
:10427000632830916428809151288093362880915A
:104280005228809337288091532880933828809132
:104290005428809339288091552880933A2880911A
:1042A000562880933B288091572880933C28809102
:1042B000582880933D2881E080936D281092DF2755
:1042C0008091EB27833031F582E08093EB2722C089
:1042D0001092DF270FEF1FEF1A83098380E5BE01DD
:1042E0006F5F7F4F0E945830109328280093272833
:1042F00010923628109237281092382810923928B8
:1043000010923A2810923B2810923C2810923D2897
:104310002FEF3FEFE091F127F091F227A081B181DB
:1043200084E18C931396FC92139712963C932E93F0
:10433000119787EB98E2BF010E9496170E94A22E68
:104340000F900F90CF91DF911F910F91FF900895E3
:10435000CF92DF92EF92FF920F931F93DF93CF9351
:10436000CDB7DEB72C970FB6F894DEBF0FBECDBF2A
:10437000D82EC92E082F192FDE011196F801808141
:1043800091819C01F9018CE001900D928150E1F73F
:10439000D801ED90FC9080916D288250823020F001
:1043A000C8010E945F175AC082E0F7018083D701DD
:1043B000A956BF4FFD0181938A859B8512969C93D8
:1043C0008E9311978C8582839D0128503040D901AE
:1043D000E3E6F7E288E001900D928150E1F7F90100
:1043E00038979F01AE014E5F5F4F88E0DA010D9074
:1043F000AD01D9010D929D018150C1F780916E27C9
:1044000090916F27929382938091EC2782938F5F94
:104410008093EC2783E69CEC929382938BE18293CA
:10442000D7011796FC93EE93169780E997E2B801AF
:104430000E9496178C3829F481EFB8010E94AD2EA6
:104440000DC08D2D9C2D0E940E2E81E00E944613E2
:10445000882311F40E94392BF70114822C960FB691
:10446000F894DEBF0FBECDBFCF91DF911F910F91AA
:10447000FF90EF90DF90CF900895EF92FF920F930F
:104480001F93DF93CF93CDB7DEB72F970FB6F89476
:10449000DEBF0FBECDBFAC018C01DE011196FC0169
:1044A000808191819C01F9018FE001900D928150F2
:1044B000E1F74093F1275093F2278C81823019F471
:1044C0008F8198851AC08F81809336288885809344
:1044D00037288985809338288A85809339288B8569
:1044E00080933A288C8580933B288D8580933C2847
:1044F0008E8580933D288EEF9FEF909328288093A0
:10450000272880E5BE016B5F7F4F0E945830809165
:10451000B528813011F40E947D2ED801ED90FC90D9
:1045200081E0F701808312830183E756FF4F808388
:104530008F8581839F0128503040D901E3E6F7E25F
:1045400088E001900D928150E1F7F9018FEF9FEF24
:10455000929382938C81823051F48091272890919C
:1045600028289293829345E123E238EC11C0F901A7
:104570003A979F0146E358E288E0DA010D90AD01D9
:10458000D9010D929D018150C1F74BE123E23CEC32
:1045900080916E2790916F27929382938091EC2760
:1045A00082938F5F8093EC27329322934293D701BB
:1045B0001796FC93EE93169780E0BE016E5F7F4FD7
:1045C0000E94583084E0BE016D5F7F4F0E945830DA
:1045D000882361F4C70162E070E041E00E941B1C87
:1045E000882321F481E080936E2812C0D801ED91D8
:1045F000FC9184E1808381EE83838FEF9FEF928330
:10460000818387EB98E2B8010E9496170E94A22E40
:104610002F960FB6F894DEBF0FBECDBFCF91DF91BE
:104620001F910F91FF90EF900895DC011696ED9188
:10463000FC91179782818695869583708330A9F4C3
:104640008091731B9091741B08979093741B8093B7
:10465000731BDC01369688E001900D928150E1F7E2
:104660008091751B8F5F8093751B80E00895FC011E
:10467000A681B78112968C91129786958695837044
:104680008230A1F4E091731BF091741B3297F09388
:10469000741BE093731B16968D919C9117979183D1
:1046A00080838091751B8F5F8093751B80E00895D8
:1046B000AF92BF92CF92DF92EF92FF920F931F9330
:1046C000DF93CF9300D000D0CDB7DEB7FB01A08041
:1046D000B180D50112967C936E9311978AE08C93EA
:1046E0007BE9C72ED12CCA0CDB1C8091ED278823D7
:1046F00019F46DE0E62E0EC0482F50E0C41AD50A1A
:104700005DE0E52EE80E23EF37E2C601B90150E087
:104710000E94FEBBD092741BC092731B1092751B3B
:1047200087E393E29A83898380E997E28E010F5FA2
:104730001F4FB8010E943918F090751B1092751B1D
:1047400085E193E29A83898380E997E2B8010E9428
:1047500039188091751BE091731BF091741B319790
:1047600090E09C0144E0220F331F4A95E1F72F2986
:104770002083880F991F880F991F8F0D911D880F17
:10478000991F8093751B4E2D480FE82FF0E0E095A0
:10479000F095EC0DFD1D129280916D28833019F477
:1047A0002FEF3FE402C02FEF3FE080918E27811171
:1047B0003068DF013E932E9380917127909172278C
:1047C0002FEF8E3F920789F43A974A5F9F0163E685
:1047D00077E288E0DB010D90BD01D9010D929D01CA
:1047E0008150C1F720E030EC05C0FD019293829327
:1047F00020E030E880916E2790916F27929382930A
:104800008091EA2782938F5F8093EA2732932293E5
:104810004293D5011796FC93EE931697C50162E07B
:1048200070E040E00E941B1C81E080936E280F9096
:104830000F900F900F90CF91DF911F910F91FF90EC
:10484000EF90DF90CF90BF90AF900895BC0180E0D3
:104850000E94582308950F931F938C01DC01ED9162
:10486000FC9181810E948740C8010E945F171F91BF
:104870000F9108950F931F938C01DC01ED91FC9132
:10488000818162810E94D543C8010E945F171F91F8
:104890000F910895AF92BF92CF92DF92EF920F9354
:1048A0001F935C01DC01ED91FC910481158126814F
:1048B0003781818162814381E08439966F010E9452
:1048C000BA44C5010E945F171F910F91EF90DF90CE
:1048D000CF90BF90AF9008950F931F938C01DC0190
:1048E000ED91FC9181810E94B043C8010E945F1745
:1048F0001F910F9108950F931F938C01DC01ED918F
:10490000FC9181810E945A40C8010E945F171F914B
:104910000F9108950F931F938C01DC01ED91FC9191
:10492000818162813396AF010E943344C8010E94A5
:104930005F171F910F9108950F931F93DF93CF93EC
:10494000CDB7DEB766970FB6F894DEBF0FBECDBF0A
:104950008C01DC01ED91FC91818192819B838A83A2
:10496000838189839E012C5F3F4FAF014C5F5F4F76
:1049700088E0DA010D90AD01D9010D929D018150C1
:10498000C1F7818192819E878D8784858C879E0166
:10499000215F3F4FAF01435F5F4F88E0DA010D9029
:1049A000AD01D9010D929D018150C1F7CE01019653
:1049B000BE01645F7F4F45890E948540C8010E9407
:1049C0005F1766960FB6F894DEBF0FBECDBFCF91CE
:1049D000DF911F910F910895CF92DF92EF92FF9296
:1049E0000F936C01DC01ED91FC91BF016E5F7F4F75
:1049F00024893589E788F08C8181438906890E9462
:104A00005840C6010E945F170F91FF90EF90DF9012
:104A1000CF900895EF92FF920F937C01DC01ED910E
:104A2000FC91218132814381548165817681878126
:104A3000908501850E944F45C7010E945F170F9125
:104A4000FF90EF9008950F931F938C01DC01ED917F
:104A5000FC918181928163810E949943C8010E94E7
:104A60005F171F910F9108950F931F938C01DC0125
:104A7000ED91FC91818162810E945C40C8010E949D
:104A80005F171F910F9108956F927F928F92AF924F
:104A9000CF92EF920F93DF93CF93CDB7DEB76697A8
:104AA0000FB6F894DEBF0FBECDBF3C01DC01ED9127
:104AB000FC9181818983828193819B838A839E017A
:104AC0002C5F3F4FAF014C5F5F4F88E0DA010D90E4
:104AD000AD01D9010D929D018150C1F784858C876C
:104AE000858596859E878D879E01215F3F4FAF010B
:104AF000415F5F4F88E0DA010D90AD01D9010D9261
:104B00009D018150C1F7258D368DCE010196BE01E4
:104B1000645F7F4F448D0789E08CC18CA28C838CAD
:104B20000E940C46C3010E945F1766960FB6F89468
:104B3000DEBF0FBECDBFCF91DF910F91EF90CF9031
:104B4000AF908F907F906F900895FC0110826181EB
:104B500072816115710521F08CE298E20E9496172E
:104B60000895AF92BF92CF92DF92EF92FF920F9390
:104B70001F93DF93CF930F92CDB7DEB77C01FC017B
:104B8000A080B180F501A681B7813C913093412886
:104B9000FD01E30FF11D8181809361281196CD9075
:104BA000DC901297D0923F28C0923E2813968C91A9
:104BB000139780934228AD014C5F5F4F7D2D729516
:104BC0007695769573706D2D66956695637019F47C
:104BD000FA0120E049C014968D919C91159790930D
:104BE000452880934428FD0136966230E1F4109206
:104BF000462810924728109248281092492810926F
:104C00004A2810924B2810924C2810924D28169644
:104C10008D919C9117979093472880934628FD018A
:104C2000389624E021C0633011F022E01DC01696B2
:104C30008C911697809346288181809347288281A2
:104C400080934828838180934928848180934A28CF
:104C5000858180934B28868180934C28878180931F
:104C60004D28FD013E962AE0772309F447C0C6FC93
:104C700008C0819191919093502880934F282E5F86
:104C800008C08091442890914528909350288093A3
:104C90004F287230C1F4109251281092522810926D
:104CA000532810925428109255281092562810928A
:104CB0005728109258288081918190935228809390
:104CC00051282E5F1BC07330C9F480818093512816
:104CD000818180935228828180935328838180939D
:104CE0005428848180935528858180935628868115
:104CF00080935728878180935828285F3550321B2E
:104D00003093622870934E28609343288A01020FE3
:104D1000111D8C2D877080934028833021F4F80179
:104D20008081809360281982C3FE0DC0F5016681E1
:104D300077816F5F7F4F8EE398E2A8019E012F5F1E
:104D40003F4F0E9434A330914028313009F461C0B4
:104D5000313020F0333009F04DC16FC02981F801A6
:104D6000E20FF11D808191819093642880936328E4
:104D7000822F8E5F8983F801E80FF11D8081809377
:104D800065282D5F29832350877019F02C5F280F29
:104D900029838981F801E80FF11D9081909366289D
:104DA000482F4F5F4983292F2770892F90E0807704
:104DB000907034E0959587953A95E1F7382F222346
:104DC00011F48823A1F0C801840F911D90936828E5
:104DD00080936728222319F0220F240F298333237D
:104DE00031F0330F330F330F8981380F39838091BE
:104DF00062289981981750F4891B80936928090FBC
:104E0000111D10936B2800936A28F8C0109269282E
:104E1000F5C080916228882369F0863718F086E70C
:104E2000809362288981080F111D109364280093D4
:104E30006328E4C010926228E1C081E08983209158
:104E40006028243009F4DAC0253030F4213059F0DC
:104E5000223009F0CFC00DC0273009F4CFC0283070
:104E600009F0C8C012C0F80181818093632882E0F4
:104E70002EC0F801818192819093642880936328E9
:104E80003983838180936528B9C0F801818192813B
:104E900090936428809363283983838194819093CD
:104EA00066288093652885E08983858180936728BB
:104EB00086E089838681978190936928809368280A
:104EC0002983D4FE9BC0808580936A2889E08983EA
:104ED00095C080914028833061F4809160288430AF
:104EE00011F0873031F48CE298E2B7010E949617F6
:104EF0008BC08091DF27813009F467C0813020F0BA
:104F0000843008F077C03AC08091E927882341F5C2
:104F100090916D28933090F0933009F06BC08091A0
:104F20004028813009F462C0833009F063C0809169
:104F300060288430B9F1873079F543C080914028EA
:104F4000813009F453C0833009F054C08091602847
:104F5000843041F1873001F5923009F04BC031C007
:104F6000823019F0843009F045C0809140288823B0
:104F700009F040C0C7010E949A3446C00E94003424
:104F800080914028813091F18330A1F58091602893
:104F9000843041F0873089F0813061F5C7010E948B
:104FA000612032C080919527882321F0C7010E949B
:104FB00092292AC00E9476281DC080916D288230D7
:104FC000C9F4C7010E9426241FC080914028833065
:104FD00059F480916028823069F480E00E942114A5
:104FE000C7010E94242110C0813021F4C7010E9412
:104FF000552B0AC0C7010E945F1706C080916E281A
:10500000882309F066CF75CF0F90CF91DF911F9164
:105010000F91FF90EF90DF90CF90BF90AF900895E9
:10502000CF93DF93DB01EC01EE81FF8182818695D6
:1050300086958370823011F040E009C040E02D91E8
:105040003C91868197812817390709F441E0842F24
:10505000DF91CF910895CF93DF93DB01EC01EE81D7
:10506000FF818281869586958370833011F020E0E0
:105070002FC020E09C918681981751F511969C9144
:1050800011978781981721F512969C911297808528
:105090009817F1F413969C91139781859817C1F492
:1050A00014969C9114978285981791F415969C916B
:1050B00015978385981761F416969C9116978485A9
:1050C000981731F417969C918585981709F421E07B
:1050D000822FDF91CF910895FB0140E02081318143
:1050E0002817390709F441E0842F08950F931F937F
:1050F000CF93DF938DE90E9467178C01009709F425
:1051000049C0DC014D915C918CE0FA0180831283EF
:105110000183E556FF4F80914E28833069F438971C
:10512000EF01A1E5B8E288E00D9009928150E1F726
:105130006FE021E03CE009C0809151289091522815
:105140009293829369E021E038E080914F2890911A
:105150005028929382938091EC2782938F5F809363
:10516000EC27329322936293DA011796FC93EE9325
:105170001697F8018081918161E070E040E00E9423
:105180001B1C882321F481E080936E2803C0C80192
:105190000E945F17DF91CF911F910F9108956F9239
:1051A0007F929F92AF92BF92CF92DF92EF92FF9247
:1051B0000F931F93CF93DF93D82E962EC42E5901B1
:1051C00038018DE90E9467177C01009709F49BC0A4
:1051D000DC010D911C91DD2021F084E0F801808339
:1051E00003C08BE0D8018C93F801F282E182E6568D
:1051F000FF4F84E080832091712730917227C9018D
:105200000296029710F0992069F03897EF01A3E613
:10521000B7E288E00D9009928150E1F762E183E204
:1052200090EC05C0329322936CE083E290E8CC20AE
:1052300061F020916E2730916F276216730629F076
:105240006E5F3293229370E002C0806471E022E0CE
:10525000C21641F4AC015860D5018D919C91929396
:10526000829328C0B3E0CB1661F4AC015C60389740
:105270006A5FEF01D50188E00D9009928150E1F756
:1052800019C020912728309128284FEF2E3F34074E
:1052900029F0AC015860329322930CC0AC015C60E1
:1052A00038976A5FEF01A6E3B8E288E00D900992B3
:1052B0008150E1F73297772339F080916E279091F2
:1052C0006F279183808302C0718260828091EC2776
:1052D00082938F5F8093EC27529342936293D8011D
:1052E0001796FC93EE931697C80162E070E041E0D8
:1052F0000E941B1C882321F481E080936E2804C047
:10530000C7010E945F1780E0DF91CF911F910F913D
:10531000FF90EF90DF90CF90BF90AF909F907F90E5
:105320006F900895DF92EF92FF920F931F93DF9398
:10533000CF9300D000D0CDB7DEB710926C280E947A
:105340005F1780916D28823008F4BDC080914E288F
:10535000823021F0833009F0B6C003C080E198E2CA
:1053600002C08BE298E29A83898381E598E29C836C
:105370008B8380E997E2BE016F5F7F4F0E943918EF
:10538000BC01009789F0DC014D915C91DA01169621
:10539000ED91FC91179720914F28309150288481EE
:1053A00095812817390719F00E9476288CC081E072
:1053B000FA01848380914E28823021F0833009F0F5
:1053C0006DC023C02091512830915228ACEBB7E238
:1053D00014968C911497882391F0ED91FC9111977C
:1053E0000190F081E02D8481882349F40680F781C3
:1053F000E02D868197812817390709F441C0159659
:10540000E7E2AF3DBE0721F749C0D0905128E090B8
:105410005228F0905328009154281091552830912B
:1054200056282091572890915828ACEBB7E2149653
:105430008C911497882369F1ED91FC91119701905B
:10544000F081E02D8481882321F50680F781E02D0D
:1054500086818D15F1F487818E15D9F480858F159D
:10546000C1F481858017A9F48285811791F4838521
:10547000831779F48485821761F48585891749F447
:10548000DA011696ED91FC911797818180618183F5
:1054900005C01596E7E2AF3DBE0749F6DA0114965E
:1054A0001C92149712967C936E931197CA0161E037
:1054B00070E040E00E941B1C882329F481E0809367
:1054C0006E2880936C280F900F900F900F90CF91C3
:1054D000DF911F910F91FF90EF90DF900895DC0115
:1054E000ED91FC911197E081E43278F4F0E0EE0F59
:1054F000FF1FEF56F94F259134912115310519F011
:10550000F901099508950E945F1708951F938091EE
:105510006E28882381F48091E827882361F083EE48
:1055200097E260E070E00E943318009721F00E943B
:105530006F2A11E001C010E080913128882359F0D2
:105540008CE298E260E070E00E943318009719F056
:105550000E946F2A11E0812F1F910895DC01ED91C7
:10556000FC91119780E180834183628387EB98E20D
:10557000BD010E94961708957F928F929F92AF92DD
:10558000BF92CF92DF92EF92FF920F931F93DF9320
:10559000CF9300D000D0CDB7DEB70CEB17E29CE67E
:1055A000892E98E2992E5E010894A11CB11C80E11D
:1055B000782ED80114968C9114978823C9F11296ED
:1055C0008D919C911397019713969C938E931297AC
:1055D000892B71F514961C921497ED90FC90F701AD
:1055E000C080D1809A828982FC82EB8280E997E236
:1055F000B5010E943318D6018C91823019F08D309C
:10560000A1F405C080EFB7010E94AD2E0EC0F601D7
:105610008381D701ED91FC917082818380EF828339
:1056200087EB98E2B7010E949617F8011182108269
:105630000B5F1F4FF7E20F3D1F0709F0BACF0E9423
:10564000312E80919527882311F00E94392B0F90DD
:105650000F900F900F90CF91DF911F910F91FF90BE
:10566000EF90DF90CF90BF90AF909F908F907F9002
:105670000895EF92FF920F931F9381E040E050EE68
:1056800061E070E020E030E00CEB1AE2EE24FF2451
:105690000E942D15882321F080E090E00E94BC2A12
:1056A0001F910F91FF90EF9008950F931F93DF9339
:1056B000CF93CDB7DEB728970FB6F894DEBF0FBEF5
:1056C000CDBFAC01DC019C9111962C918091622898
:1056D000882321F4CA010E945F1705C1E92FF22F28
:1056E00080914228808F80914E2881838250823021
:1056F000A8F480914F2890915028938382839F0132
:105700002C5F3F4F61E578E288E0DB010D90BD0141
:10571000D9010D929D018150C1F70AC013821282F6
:1057200014821582168217821086118612861386BD
:10573000208D80918F27281761F594818091B22761
:10574000981739F595818091B327981711F59681AF
:105750008091B4279817E9F497818091B52798171D
:10576000C1F490858091B627981799F4918580911E
:10577000B727981771F492858091B827981749F444
:1057800093858091B927981721F4CA010E945F1769
:1057900060C020938F2784818093B2278581809376
:1057A000B32786818093B42787818093B52780852E
:1057B0008093B62781858093B72782858093B82709
:1057C00083858093B92780914328848782508230D3
:1057D000A8F48091442890914528968785879F0159
:1057E000215F3F4F66E478E288E0DB010D90BD0168
:1057F000D9010D929D018150C1F70AC01686158608
:105800001786108A118A128A138A148A158A168AB0
:1058100080916128878B809159288770818F809132
:1058200059288695869586958370828F80915F280A
:10583000838F80916228848F80916328909164285F
:10584000968F858F81E1808387EB98E2BA010E9471
:10585000961780913E2884FF46C080916D28833042
:1058600009F443C080914E28823071F48091512810
:10587000909152289A83898300914F281091502843
:1058800080E060E042E021C0833019F5809151282A
:105890008983809152288A83809153288B838091B9
:1058A00054288C83809155288D83809156288E832F
:1058B000809157288F8380915828888700914F289E
:1058C0001091502880E060E043E09E012F5F3F4F41
:1058D00007C080E060E040E020E030E000E010E061
:1058E0000E94CF2802C00E94A22E28960FB6F894DC
:1058F000DEBF0FBECDBFCF91DF911F910F910895F5
:10590000AF92BF92CF92DF92EF92FF920F931F93CD
:10591000DF93CF93CDB7DEB768970FB6F894DEBFAD
:105920000FBECDBFB82EA92E082F192FDE01149659
:10593000F801808191819C01F90185E101900D922E
:105940008150E1F78A8982FD11C08091DF27882389
:1059500021F48091E927882349F09989D801ED91B4
:10596000FC9180E18083918381EE0BC1F801E0809E
:10597000F1808DE0D7018C93898913968C938E8961
:105980008B5F898385502BE9C22ED12CC81AD10890
:10599000CE0CDF1CDB82CA828B89882371F0CE019A
:1059A0000296BE016C5F7F4FAE014F5F5F4F0E945A
:1059B000CDA2282F882309F0C2C08D81823079F4CE
:1059C000EA81FB813297FB83EA8389818E5F898339
:1059D00080917127909172279183808313C08330C7
:1059E00089F42A813B81285030403B832A83898176
:1059F000885F8983D901E3E6F7E288E001900D92A0
:105A00008150E1F720916E2730916F278F81988523
:105A10002817390749F48D81882331F08E81882336
:105A200019F040E450E00FC08D81882351F0EA81E5
:105A3000FB813297FB83EA8389818E5F898331837F
:105A4000208340E050E03E81332349F18A819B81ED
:105A50002981323059F4FC013297FB83EA832E5FAF
:105A6000298389859A85918380830DC008979B83BC
:105A70008A83285F2983FC01DE01199688E00D9056
:105A800001928150E1F7EA81FB813297FB83EA833F
:105A900089818E5F89838F81988591838083EA8154
:105AA000FB813197FB83EA838091EC2780838F5FB2
:105AB0008093EC27BA0161608B89882319F0BA01C1
:105AC000696070618A8980FD60628E89873608F01E
:105AD00070618E81382F330F330F20E04D81942F6A
:105AE0009295990F990F907C80E0282B392B8A8111
:105AF0009B81FC013297FB83EA83262B372B318372
:105B00002083298127FF02C025EE19C0FC013397AD
:105B1000FB83EA8320838A819B81F70197838683B5
:105B20008B89882309F465C0C701B601AE014C5FBB
:105B30005F4F0E94A1A4282F882309F45AC08989A5
:105B4000D801ED91FC9190E190838183228387EBD2
:105B500098E2B8010E94961750C080916D2882503B
:105B60008230F8F480E997E2B8010E9496178C38E9
:105B700051F49989D801ED91FC9180E18083918362
:105B800081EF8283E4CF8B2D9A2D0E940E2E81E02F
:105B90000E944613882311F40E94392BF7011482C6
:105BA0002CC08091B528813011F40E947D2ED70140
:105BB00012961C930E931197C70162E070E041E0CA
:105BC0000E941B1C882321F481E080936E2815C05D
:105BD0009989D801ED91FC9180E18083918381EED8
:105BE000828387EB98E2B8010E9496170E94A22E4A
:105BF00004C08A8982FFD5CFB0CF68960FB6F894DB
:105C0000DEBF0FBECDBFCF91DF911F910F91FF90EF
:105C1000EF90DF90CF90BF90AF900895AC01E0EC93
:105C2000F7E220E030E080818823A1F4F901EE0F53
:105C3000FF1FEE0FFF1FE20FF31FE454F84D80919A
:105C4000EE279091EF27938382835183408381E0F5
:105C5000848308952F5F3F4F35962730310519F71C
:105C6000089520E001C0292F822F90E0FC01EE0F63
:105C7000FF1FEE0FFF1FE80FF91FE454F84D84815A
:105C8000922F9F5F882379F7392F41E033C0832F0C
:105C900090E0DC01AA0FBB1FAA0FBB1FA80FB91F02
:105CA000A454B84D14968C911497882311F1822F27
:105CB00090E0FC01EE0FFF1FEE0FFF1FE80FF91F32
:105CC000E454F84D44838D919C9111979183808386
:105CD00012968D919C9113979383828314961C92B4
:105CE000149711961C921E9213961C921E92129754
:105CF0002F5F3F5F373058F208958091B52881308B
:105D000051F40E940920853831F081E090E00E9432
:105D1000E2121092B52808958091B528882389F45D
:105D200080E090E00E94E21280E00E941B20882325
:105D300021F481E08093B528089581E090E00E94ED
:105D4000E212089580919627882331F480912928C2
:105D5000882311F40E948C2E0895DF93CF93CDB742
:105D6000DEB728970FB6F894DEBF0FBECDBF482F21
:105D70009B01DB01ED91FC910680F781E02DDE01B6
:105D80001196369688E001900D928150E1F7D90185
:105D9000ED91FC918CE1808380916E2790916F272B
:105DA0009283818393E0938380916327848380919E
:105DB0006427858380916527868380916627878302
:105DC00080916727808780916827818780916927E4
:105DD000828780916A2783879487898185878A81D2
:105DE00086878B8187878C81808B8D81818B8E814B
:105DF000828B8F81838B8885848B458B87EB98E2A0
:105E0000B9010E94961728960FB6F894DEBF0FBE10
:105E1000CDBFCF91DF9108950F931F93082F10925C
:105E20006E2810926D281092B5281092E9271092D2
:105E3000EB271092DF2710928F278FEF8093B227E6
:105E40008093B3278093B4278093B5278093B62798
:105E50008093B7278093B8278093B927ECEBF7E2BC
:105E600014821182108213821282359687E2EF3DEE
:105E7000F807B1F710926C281092292888E00E9448
:105E80003F201FB7F89480E00E94211481E00E9417
:105E9000211482E00E9421141FBF002309F452C084
:105EA0001092B62882EC97E09093E2278093E12746
:105EB00080E098E7909333288093322811E0109384
:105EC000BB2710928E271092ED270E940AB880936C
:105ED000EA2784EF91E09093EF278093EE271093C9
:105EE000E02786E08093B127109236281092372859
:105EF000109238281092392810923A2810923B2894
:105F000010923C2810923D288FEF9FEF9093282805
:105F1000809327280E940AB88093EC271092962736
:105F2000109291281092A3281092A8281092A928C4
:105F30001092AA281092AB281092AC2810929727A2
:105F40001092A8271F910F9108950F931F93CF933D
:105F5000DF93EC01088119818091B528813011F41B
:105F60000E947D2EF801018180E090E00E94E21203
:105F700080E0011181E00E94951E182F81E090E0E1
:105F80000E94E212802F0E940C2F0E94A22E83EE0C
:105F900097E20E943F188CE298E20E943F1887EB3C
:105FA00098E20E943F1880E997E20E943F18E8813A
:105FB000F981118380E2808387EB98E2BE010E9421
:105FC0009617DF91CF911F910F910895DF93CF9393
:105FD00000D000D0CDB7DEB78091B528813011F464
:105FE0000E947D2E8FEF9FEF9A8389839C838B8302
:105FF00083E5BE016F5F7F4F0E94583080E5BE0190
:106000006D5F7F4F0E94583081E00E940C2F0E94EC
:10601000A22E0F900F900F900F90CF91DF910895C7
:106020000E94CF1E8823D1F40E94D6168823B1F097
:1060300081E00E940C2F0E94A22E83EE97E26FEF68
:106040000E948E178CE298E26FEF0E948E1780E913
:1060500097E267E00E948E1780E0089585E8089532
:10606000E82F853419F48091ED270895883030F4B5
:10607000E82FF0E0E752F94F849108958054803280
:1060800028F4F0E0EF55F94F849108958E2F815751
:10609000833128F4F0E0E057F94F84910895E03F10
:1060A00010F480E00895F0E0EC5DF94F84910895DC
:1060B0001F93CF93DF93182FEB018091B528813088
:1060C00051F40E947D2E812FBE010E943A1D182F8F
:1060D0000E94A22E04C0812F0E943A1D182F812FEA
:1060E000DF91CF911F9108950F931F93CF93DF936B
:1060F0008C01FC01C081D181BE016D5F7F4F898120
:10610000833509F4F5C0843508F04CC0823409F4B5
:10611000B5C08334F8F4843009F4A2C0853068F443
:10612000813009F4F8C0813008F4F2C0823009F4FB
:10613000FBC0833009F07CC0FAC0863009F498C0F7
:10614000863008F490C0873009F495C0813409F096
:106150006FC097C08B3409F4B5C08C3480F486349A
:1061600009F49CC0873420F4853409F061C08CC0E8
:10617000893409F496C08A3409F05AC09AC08F3421
:1061800009F4ABC0803538F48C3409F4A0C08E34E7
:1061900009F04EC09FC0803509F4A2C0823509F0D5
:1061A00047C0A3C0833709F4D1C08437F8F48935D8
:1061B00009F44BC08A3560F48635E1F1873518F46F
:1061C0008535B1F571C08735C1F1883589F538C09D
:1061D0008D3509F442C08E3518F48A3549F538C03A
:1061E000813709F4A7C0823719F5ADC08C3709F49F
:1061F000D2C08D3760F4853709F4B4C0853708F410
:10620000AEC0863709F4B7C0873791F4B7C082387B
:1062100009F4D6C0833830F4803809F4C5C0813819
:1062200039F4C5C0833809F4CFC0803F09F467C092
:1062300094EFD3C08091B628C5C080917E27C2C09C
:106240008091E1279091E22757C080918227BAC0C0
:1062500080913228909133284FC08091BB27B2C0E3
:1062600080916D27AFC080916B2790916C2744C0BF
:1062700080918527A7C080917B27A4C08091E027CB
:10628000A1C080918E279EC04091ED2723EF37E279
:10629000CB01B90150E00E94FEBB9EC08091ED276A
:1062A00091C08091EA278EC08091EE279091EF27D0
:1062B00023C0DB01E6E3F8E288E001900D92815013
:1062C000E1F78AC0809127289091282815C08091F5
:1062D000EC2778C080917A2775C08091812772C0A1
:1062E00080916E2790916F2707C0809196276AC092
:1062F00080917127909172279C838B836DC0DB0105
:10630000E3E6F7E288E001900D928150E1F764C086
:1063100080917C2757C08091892790918A27A091EE
:106320008B27B0918C2732C0809162274BC080911F
:10633000702748C0DB01EFE6F8E282E201900D929F
:106340008150E1F749C0809191283CC0DB01E2E92E
:10635000F8E281E101900D928150E1F73DC080911A
:10636000A32830C08091A4289091A528A091A628A8
:10637000B091A7280BC08091A82824C08091A9289B
:106380009091AA28A091AB28B091AC288B839C83D4
:10639000AD83BE8321C0DB01EDEAF8E288E0019025
:1063A0000D928150E1F718C0809197270BC0DB0157
:1063B000E8E9F7E280E101900D928150E1F70CC02D
:1063C0008091A8278B8308C0DB01E9EAF7E288E027
:1063D00001900D928150E1F790E089818A838EE1EE
:1063E0008883998387EB98E2B8010E949617DF9122
:1063F000CF911F910F910895FF920F931F93CF9309
:10640000DF93182FEB01F42E853509F4AFC08635E4
:1064100008F040C0873409F4E4C08834F8F48234CA
:1064200009F487C0833468F4853038F4823008F08A
:10643000D8C0882309F4D5C06CC0813409F069C084
:1064400080C0843409F479C0843408F4CAC0853427
:1064500009F47BC0863409F05CC080C0813598F4B3
:106460008E3408F0BEC08A3409F487C08B3420F41F
:10647000893409F04EC076C08B3409F497C08C344F
:1064800009F047C09AC0823509F49BC0823508F4F0
:1064900040C0A7C0843709F422C18537E8F48A35A3
:1064A00009F440C08B3550F4873509F49AC087351C
:1064B00090F18835A1F1893561F593C0813709F4F0
:1064C000F8C0823718F48D3521F5ECC0823709F415
:1064D000F9C08337F1F4FAC0803809F42BC1813850
:1064E00060F4863709F40CC1863708F4FCC087379E
:1064F00009F40AC18C3769F414C1823809F42AC13D
:10650000823808F41EC1833809F42BC1803F09F496
:1065100068C004EF2FC188818093B6282AC1888182
:106520009981BBC0888199819093332880933228C8
:1065300020C188818093E0271CC188818093B12786
:1065400018C1888180938E2714C123EF37E24091D0
:10655000ED27C90150E00E94FEBB0BC188818093EA
:10656000ED2707C188818093EA2703C1888199813B
:106570009093EF278093EE27FCC088818093362884
:106580008981809337288A81809338288B818093F2
:1065900039288C8180933A288D8180933B288E8185
:1065A00080933C288F8180933D28E3C08881998126
:1065B0009093282880932728DCC088818093EC273B
:1065C000D8C06881611161E060939627662331F03D
:1065D0000E947D2E86E00E943F20CBC00E94A22E0A
:1065E000C8C0812FBE010E943A1D082F813871F466
:1065F0000E940920812FBE010E943A1D082F882386
:1066000009F0B8C081E08093761B03C0882309F0AD
:10661000B1C080917A27282F30E080917E27482FC3
:1066200050E060918127CA01861B9109281739071C
:106630000CF4C901A82F281B310981E090E002C0A9
:10664000880F991F4A95E2F70197289FA001299F7B
:10665000500D389F500D112420E030E070E0E1E053
:10666000F0E00DC0C901860F971FEF0102C0CC0FEB
:10667000DD1F8A95E2F74C0F5D1F2F5F3F4F2A17F2
:1066800088F384E190E09C01429FC001439F900DFC
:10669000529F900D1124865F9E4F9093E227809326
:1066A000E12767C090E08881811191E09093BB273A
:1066B00060C0AFE6B8E2FB0182E201900D9281502A
:1066C000E1F757C088818093912853C0A2E9B8E2CE
:1066D000FB0181E101900D928150E1F74AC0888170
:1066E0008093A32846C088819981AA81BB81809329
:1066F000A4289093A528A093A628B093A72839C0D2
:1067000088818093A82835C088819981AA81BB811E
:106710008093A9289093AA28A093AB28B093AC2883
:1067200028C0ADEAB8E2FB0188E001900D928150EB
:10673000E1F71FC090E08881811191E09093972745
:1067400018C0A8E9B7E2FB0180E101900D928150E9
:10675000E1F70FC090E08881811191E09093A82724
:1067600008C0A9EAB7E2FB0188E001900D928150D0
:10677000E1F700E0FF2049F08091761B882329F0A3
:1067800080E00E941B201092761B802FDF91CF911A
:106790001F910F91FF900895EF92FF920F931F9317
:1067A0007C01FC0100811181B8016E5F7F4FF8010F
:1067B000818141E00E94FC31F801918192839FE147
:1067C0009083818387EB98E2B7010E9496171F910F
:1067D0000F91FF90EF900895CF93DF93EC01E88144
:1067E000F98183E280836183662311F00E94A22EE7
:1067F00087EB98E2BE010E949617DF91CF91089532
:10680000809140288823E1F080E00E94211480914B
:106810004028813031F480916228882311F060E0B3
:1068200001C06BEE8091DF27823031F48091F12737
:106830009091F2270E94EC3310926E281092DF277D
:1068400008958091DF27823039F48091F12790916B
:10685000F2276BEE0E94EC331092DF2710926E2825
:106860000895CF92DF92EF92FF920F931F93DF93E1
:10687000CF93CDB7DEB728970FB6F894DEBF0FBE23
:10688000CDBFD82EC92E8091DF27882309F03EC0C6
:1068900080916D288330D1F18091E9278823B1F56B
:1068A0008091B528813011F40E947D2EED2CFC2CB6
:1068B000D701ED91FC9181819F012C5F3F4F823088
:1068C00031F4848195819A83898342E00DC0AE01C1
:1068D0004F5F5F4F88E0D9010D909D01DA010D9265
:1068E000AD018150C1F743E00281138181E060E096
:1068F0009E012F5F3F4F0E94CF28882311F4C701CC
:1069000007C0D092F127C092F22705C08D2D9C2D93
:1069100061EE0E94EC3328960FB6F894DEBF0FBEEE
:10692000CDBFCF91DF911F910F91FF90EF90DF903E
:10693000CF9008955F926F927F928F929F92AF92C5
:10694000BF92CF92DF92EF92FF920F931F93DF934C
:10695000CF93CDB7DEB761970FB6F894DEBF0FBE09
:10696000CDBFBC014091E927423011F0443069F4B9
:106970008091E027882349F0E091F127F091F227F8
:1069800020813181D901199604C0A0E0B0E020E057
:1069900030E050914E28598300914F281091502893
:1069A0001B830A83523069F41E821F82188619865F
:1069B0001A861B8680915128909152289D838C8342
:1069C00018C0809151288C83809152288D838091AA
:1069D00053288E83809154288F83809155288887EF
:1069E000809156288987809157288A8780915828D6
:1069F0008B8790907C279C86B0906D27BD86809178
:106A00006328909164289F878E87188A80916528D3
:106A100087FF02C081E0888B80916128898B42309A
:106A200019F0443009F06FC08091E027882309F401
:106A30006AC0F901F084EC81FD815C806D807E800C
:106A40008F80A884C984DA84EB8440E049C0119621
:106A50008D919C9112970817190709F03FC08C91EE
:106A60005817E1F51B968C911B979816B9F51C9653
:106A70008C911C97B81691F5523041F413968D9174
:106A80009C911497E817F90749F53DC013968C912E
:106A90001397851519F514968C9114978615F1F4B2
:106AA00015968C9115978715C9F416968C911697A3
:106AB0008815A1F417968C9117978A1579F4189672
:106AC0008C9118978C1551F419968C9119978D15F6
:106AD00029F41A968C911A978E15A9F04F5F51964A
:106AE0004F1508F4B4CF59C0FD01DE01119681E1C4
:106AF0000D9001928150E1F7D90118968C91189769
:106B00008F5F18968C9390916628809169288823CE
:106B100021F48091E0278823E1F5DB01ED91FC91E0
:106B200087E180838091422881839F012E5F3F4FC0
:106B3000AE014F5F5F4F81E1DA010D90AD01D901E8
:106B40000D929D018150C1F780916628838B892F1A
:106B5000877059F4892F90E08077907024E09595A4
:106B600087952A95E1F7882331F0809167289091E5
:106B70006828958B848B80916928868B80916A2800
:106B800090916B28908F878B87EB98E20E949617E5
:106B900009C0CB010E945F1705C0E4E0EF1508F4BF
:106BA000B2CFA2CF61960FB6F894DEBF0FBECDBFB5
:106BB000CF91DF911F910F91FF90EF90DF90CF90D9
:106BC000BF90AF909F908F907F906F905F9008954F
:106BD0000F931F93DF93CF9300D000D0CDB7DEB7D4
:106BE0008C018CE698E29A838983F80181819281F5
:106BF0009C838B8380E997E2BE016F5F7F4F0E9489
:106C00003318F80141815281ECEBF7E220E030E0EB
:106C1000808191814817590779F4F901EE0FFF1F20
:106C2000EE0FFF1FE20FF31FE454F84D14821182A0
:106C300010820E94312E06C02F5F3F4F35962730BD
:106C4000310531F710926C280F900F900F900F9034
:106C5000CF91DF911F910F910895EF92FF920F93C3
:106C60001F93CF93DF93182FEB0110926E28809122
:106C7000E9278250823020F4812F0E942439B5C048
:106C80008881883009F4A5C0893050F4823009F435
:106C900097C0843009F44DC0813009F0A4C01DC0F4
:106CA0008B3009F446C08C3020F48A3009F09BC048
:106CB00096C08C3009F493C08D3009F094C0809157
:106CC0006C28882319F0CB010E94E83589819A81CC
:106CD000612F4B810E94AE2A86C0193E11F0113EF1
:106CE00041F489819A81612F4FEF5FEF0E948D20DF
:106CF0007AC08093DF27409132285091332860E09A
:106D000070E024E0440F551F661F771F2A95D1F7C6
:106D100080E020E030E00EED10E2EE24FF240E943F
:106D20002D15882309F461C080E090E00E94DE20E8
:106D30005CC089819A810E945F178091DF27813032
:106D400009F453C088818430A1F4173881F0E091B0
:106D5000F127F091F227A081B18183E28C93119603
:106D60001C9387EB98E2BF010E9496173CC082E01B
:106D700005C0193EC1F1113EB1F183E08093DF27D8
:106D80004091E1275091E22760E070E094E0440FE9
:106D9000551F661F771F9A95D1F780E020E030E0FD
:106DA00001E214E3EE24FF240E942D1591E090935C
:106DB0006E288823D1F080E090E00E94213415C035
:106DC000CB010E94E83569817A81812F0E94AD2E26
:106DD0000AC069817A81812F0E94783904C0898133
:106DE0009A810E945F170E94A22EDF91CF911F917E
:106DF0000F91FF90EF900895CF93DF93E0913428A7
:106E0000F0913528C081D181DE01A656BF4FFA83AB
:106E1000E983882339F087E088838C9323E038E086
:106E20004AE013C086E088838C9318979D0143E65F
:106E300057E288E0FA010190AF01F90101929F0148
:106E40008150C1F723E438EC42E1FD018FEF9FEF61
:106E50009293829332979183808315978091EC2748
:106E60008C938F5F8093EC273E932E93FD0142938A
:106E7000FF83EE83CE0162E070E040E00E941B1CC5
:106E8000882311F080E003C081E080936E28DF91B9
:106E9000CF910895CF92DF92FF920F931F93DF93CC
:106EA000CF930F92CDB7DEB7F82E6B01FB010081B7
:106EB000118184E06DE77BE10E9458304091E92721
:106EC0005091E02720917C1B66C0423011F0443085
:106ED00039F4552329F0F8018085853008F05EC02B
:106EE000322F3F5FF80184819581A681B781022E00
:106EF00004C0B695A795979587950A94D2F78170A7
:106F00009070892B09F446C020937C1BF1E0FF169A
:106F100021F482E08093E92705C083E0F81611F49C
:106F2000F092E92780E06CE77BE10E945830F82E70
:106F30008823B9F080913428909135280E945F17FA
:106F400010923528109234280E94A22E8AEEF80161
:106F50008183108687EB98E2B6010E949617109203
:106F6000E9271091E927123009F05DC0FF2061F494
:106F700081E00E94FC36882309F055C01983CE01B8
:106F800001960E94F0384FC080917C1B8F5F8093E8
:106F90007C1B49C0232F2B3108F497CF20937C1BF7
:106FA000F1E0FF1609F03FC0809134289091352818
:106FB0000E945F1710923528109234288091E027A4
:106FC000882341F0F8018085853010F08AEF07C0F2
:106FD000882319F0F801118203C08AEEF801818339
:106FE00080E56AE278E20E9458306091F127709162
:106FF000F22787EB98E20E9496178091F027809302
:107000007C1B80E06CE77BE10E9458308091BA27BE
:1070100080937D1B84E06DE77BE10E9458301092E5
:10702000E9270E94A22E0F90CF91DF911F910F911F
:10703000FF90DF90CF900895CF92DF92EF92FF9272
:107040000F931F93DF93CF9300D0CDB7DEB7D82E29
:10705000C92E082F192FD801ED91FC9180917C2722
:107060008093F02780916D278093BA278681809343
:107070007E1B81818093771B82819381A481B5815E
:107080008093781B9093791BA0937A1BB0937B1B02
:10709000278120937D1BD092F127C092F2278BE1AC
:1070A00080838091771B82838091781B9091791BDC
:1070B000A0917A1BB0917B1B84839583A683B783B1
:1070C0002383108611868091DF27882341F48091E5
:1070D000E927882321F48091771B882341F488EEE7
:1070E000818387EB98E2B8010E9496176EC0809169
:1070F000B528813011F40E947D2EF801E080F180E6
:107100008BE080937C1B8091771B8150823008F04C
:1071100052C08FEF9FEF9A83898380916E27909161
:107120006F2790932B2880932A2880E5BE016F5FFC
:107130007F4F0E9458308091771B813021F4D0928C
:107140003428C09235288DE90E9467179093F22762
:107150008093F127009729F488EED70111968C933C
:107160002DC08091771B823019F4C8010E945F17EF
:107170002091F1273091F227D901ED91FC918BE11B
:1071800080838091771B828380917D1B8383809194
:10719000781B9091791BA0917A1BB0917B1B848303
:1071A0009583A683B783108611868091771BB901DA
:1071B0000E944A370AC088EEF701818387EB98E284
:1071C000B8010E9496170E94A22E0F900F90CF91A7
:1071D000DF911F910F91FF90EF90DF90CF90089576
:1071E000CF93DF93C091F127D091F2279881298125
:1071F0008091E9278250833020F5E92FF22F21E09A
:1072000030E040E050E000907C1B04C0220F331FB0
:10721000441F551F0A94D2F72095309540955095FC
:1072200084819581A681B78182239323A423B523EA
:1072300084839583A683B7838091771BBE010E94C8
:107240004A37DF91CF910895DF92EF92FF920F932B
:107250001F93DF93CF930F92CDB7DEB7982F809116
:10726000EC278F5F8093EC27D090E92782E0D81637
:10727000B1F5992341F540EC53E060E070E00090F7
:107280007E1B04C0440F551F661F771F0A94D2F758
:1072900040545C4F6F4F7F4F94E0440F551F661F63
:1072A000771F9A95D1F720E030E000EF18E3EE2445
:1072B000FF240E942D15882391F0D982CE010196DA
:1072C0000E94F0380CC080917C1B8F5F80937C1BE8
:1072D0006091F1277091F22781E00E944A370F9068
:1072E000CF91DF911F910F91FF90EF90DF90089564
:1072F000CF93DF93EB01882391F462E87BE10E9456
:107300005830882361F484E063E87BE10E945830C0
:1073100080E560E87BE10E94583090E001C098EE83
:10732000E881F98182E28083918387EB98E2BE0154
:107330000E9496170E94A22EDF91CF910895EF929E
:10734000FF920F931F93CF93DF937C01DC01CD91CC
:10735000DC91AFE7BBE1FE018AE001900D92815024
:10736000E1F780917127909172278F5F9F4F39F4D9
:10737000D701ED91FC9182E280838CEE1FC0BE01AB
:10738000695F7F4F8BE00E9458308091881B882373
:10739000E1F04091801B5091811B88E0B701209162
:1073A000821B0091831B0E943B3A882309F05CC03A
:1073B000D701ED91FC9182E2808388EE818387EB97
:1073C00098E2B7010E9496174FC0BE016B5F7F4FD6
:1073D00087E40E9458308D818F3009F48E83269681
:1073E00084E5BE010E9458308091B528813011F4A7
:1073F0000E947D2E80E560E87BE10E94583080E0AD
:1074000062E87BE10E945830182F84E063E87BE15A
:107410000E9458308BE066E87BE10E9458301123CF
:10742000A9F486E00E943F20863081F48091861B7B
:10743000882311F083E001C082E080936D28D7019A
:10744000ED91FC9182E28083118207C0D701ED911A
:10745000FC9182E2808388EE818387EB98E2B7011A
:107460000E9496170E94A22EDF91CF911F910F913B
:10747000FF90EF900895DF92EF92FF920F931F938A
:10748000DF93CF93CDB7DEB72C970FB6F894DEBF5E
:107490000FBECDBF182FFB01F42EE52ED22EBE015C
:1074A0006F5F7F4F808191819C018CE0D9010D90AD
:1074B0009D01DB010D92BD018150C1F740815181D9
:1074C000DA011C931296FC93EE931197BA016E5653
:1074D0007F4FFB0188E08193DB011196FC92DF0175
:1074E0001196E1829D012F5F3F4F80917127119688
:1074F0008C93F901319680917227D90111968C9362
:10750000DF011196D182FD0131969F012F5F3F4F20
:10751000193029F48A8511968C938B8503C08FEFDF
:1075200011968C938183F901319600839B01285039
:107530003040D901E3E6F7E288E001900D928150F6
:10754000E1F7F90180916E2790916F2792938293D2
:10755000193099F4F9013A979F01BE016E5F7F4F90
:1075600088E0DB010D90BD01D9010D929D01815094
:10757000C1F762E223E23CED07C08FEF9FEF9293E9
:1075800082936CE123E038ED8FEF9FEF929382932B
:107590008091EC2782938F5F8093EC273293229324
:1075A0006293DA011796FC93EE931697CA0162E094
:1075B00070E041E00E941B1C882311F080E003C0B2
:1075C00081E080936E282C960FB6F894DEBF0FBE34
:1075D000CDBFCF91DF911F910F91FF90EF90DF9082
:1075E00008950F931F93CF93DF93EC018DE90E94D1
:1075F00067178C010097F9F0DC01ED91FC918EE0AA
:1076000080838881818389819A8193838283349660
:10761000DE01139688E00D9001928150E1F783EE30
:1076200097E2B8010E949617882311F481E004C004
:10763000C8010E945F1780E0DF91CF911F910F91E9
:1076400008958F929F92AF92CF92DF92EF92FF9226
:107650000F931F93CF93DF934C01F62ED42E122F4E
:107660008DE90E946717EC010097C9F0E881F98164
:107670008DE0808392828182F38215830683E78284
:10768000C086A186D48283EE97E2BE010E9496173F
:10769000882311F481E004C0CE010E945F1780E0CE
:1076A000DF91CF911F910F91FF90EF90DF90CF90DE
:1076B000AF909F908F900895BF92CF92DF92EF92FC
:1076C000FF920F931F93CF93DF93182F6A017B01D3
:1076D000B22E8DE90E946717EC010097B9F0E8819E
:1076E000F9818BE080831183C282D382E482F582A8
:1076F000B682078383EE97E2BE010E949617882325
:1077000011F481E004C0CE010E945F1780E0DF9198
:10771000CF911F910F91FF90EF90DF90CF90BF908E
:1077200008951F93CF93DF93182F8DE90E94671759
:10773000EC01009789F0E881F98188E0808311836A
:1077400083EE97E2BE010E949617882311F481E030
:1077500004C0CE010E945F1780E0DF91CF911F919E
:1077600008951F93CF93DF93182F8DE90E94671719
:10777000EC01009789F0E881F98189E08083118329
:1077800083EE97E2BE010E949617882311F481E0F0
:1077900004C0CE010E945F1780E0DF91CF911F915E
:1077A00008957F928F929F92AF92BF92CF92DF9275
:1077B000EF92FF920F931F93CF93DF93F22ED32E6E
:1077C000C42EB52EA62E972E882E792E8DE90E94D6
:1077D0006717EC010097D9F0E881F98182E0808396
:1077E000F182D282C382B482A58296828782708619
:1077F00012870187E38683EE97E2BE010E94961707
:10780000882311F481E004C0CE010E945F1780E05C
:10781000DF91CF911F910F91FF90EF90DF90CF906C
:10782000BF90AF909F908F907F900895DF92EF92DE
:10783000FF920F931F93CF93DF93F82ED62EEA017A
:10784000E22E8DE90E9467178C01009731F1DC016F
:10785000ED91FC9181E08083F1828881838389812D
:107860009A81958384839F012A5F3F4FDE0113969F
:1078700088E00D90E90109929E018150D1F7E686DA
:10788000D28283EE97E2B8010E949617882311F402
:1078900081E004C0C8010E945F1780E0DF91CF91B2
:1078A0001F910F91FF90EF90DF9008955F926F927C
:1078B0007F928F929F92AF92BF92CF92DF92EF9280
:1078C000FF920F931F93DF93CF93CDB7DEB7D82EE0
:1078D0003B01F42E922E532EB02E86E7841708F427
:1078E00055C08DE90E9467178C01009709F44EC0BE
:1078F000DC01ED91FC9183E08083D182D3012C9156
:10790000228311968D919C91129794838383CF014A
:107910000596A3014D5F5F4F223079F415821682E0
:1079200017821086118612861386148613968D91FF
:107930009C911497968385830AC09C0188E0DA01A4
:107940000D90AD01D9010D929D018150C1F7B58611
:10795000E686C786A08A818AF28A2BE930E02F1951
:1079600031092E0F3F1FC901692D752D4F2D50E094
:107970000E94FEBB83EE97E2B8010E94961788230F
:1079800011F481E004C0C8010E945F1780E0CF912C
:10799000DF911F910F91FF90EF90DF90CF90BF90FC
:1079A000AF909F908F907F906F905F900895FF921F
:1079B0000F931F93CF93DF93182F062FF72E8DE988
:1079C0000E946717EC010097E1F0812F0E94303090
:1079D000482FE881F98186E0808311833296CF01B8
:1079E000602F7F2D50E00E94FEBB83EE97E2BE0128
:1079F0000E949617882311F481E004C0CE010E94F2
:107A00005F1780E0DF91CF911F910F91FF90089554
:107A10001F930E94862A182F87EB98E260E070E09F
:107A20000E943318009719F00E946F2A11E00E94FB
:107A3000B71A0E948812812F1F91089587EB98E250
:107A40006FEF0E948E170E941030089581E080939E
:107A5000891B08953F924F925F926F927F928F920F
:107A60009F92AF92BF92CF92DF92EF92FF920F93CD
:107A70001F93DF93CF93CDB7DEB762970FB6F8941D
:107A8000DEBF0FBECDBF4C015B013A01322ED02EBE
:107A9000FE2C8091891B882321F00E94B03F109218
:107AA000891B4F2D50E09A0123703070211531054C
:107AB00011F4EE240AC02F5F3F4F81E090E002C036
:107AC000880F991F2A95E2F7E82E487F452BA1F4ED
:107AD0008114910489F0A114B10471F0432C552450
:107AE00082010D0D111D8E2D90E09A8B898B800FD8
:107AF000911F8038910520F00E94A63F81E0A3C02D
:107B000080917706882339F06114710409F50E9489
:107B1000A63F82E098C061147104D1F040E130E0EA
:107B20004150E42FF0E0D301AE0FBF1FE657F44EF3
:107B30008C912081822790E0232F30E0822B932BA1
:107B400030E0892B09F031E0442351F73093770678
:107B500080917706882379F0C30160E040E00E94BD
:107B6000D13FAAE8BBE1F30180E101900D92815081
:107B7000E1F71092770681E0F5018083EE2061F055
:107B80008E2D90E002979595879523E0880F991F99
:107B90002A95E1F781608083332021F0F50180810F
:107BA0008064808384E0782E7F20F50160801686D3
:107BB000CC20D1F4EE2051F0D786080D191DC40158
:107BC000B801A501232D0D2D0E94243F7720C1F17E
:107BD00081E0F5018083C401840D951DB5014E2D12
:107BE0002D2D0E943E3E2CC0772059F081E0F501FA
:107BF0008083C401840D951DB5014E2D2D2D0E944D
:107C00003E3EEE20E9F0F5016082D786C4017E0198
:107C10000894E11CF11CB701A501232D0D2D0E9434
:107C2000243F832D90E08D0D911D880D991DB70186
:107C300049895A890E94F1BB009711F083E003C083
:107C40000E94A63F80E062960FB6F894DEBF0FBE9A
:107C5000CDBFCF91DF911F910F91FF90EF90DF90FB
:107C6000CF90BF90AF909F908F907F906F905F90DC
:107C70004F903F9008950E948A3F08954F925F92DF
:107C80006F927F928F929F92AF92BF92CF92DF922C
:107C9000EF92FF920F931F93DF93CF93CDB7DEB791
:107CA00060970FB6F894DEBF0FBECDBF5C016B01CD
:107CB000642E122F80E090E060E040E00E94D13F0F
:107CC0007724EE24FF24412E55244E010894811C74
:107CD000911C25C07394D6011F967C92C6010E9408
:107CE0008B3FC4010E949D3FC8010131110514F072
:107CF00080E190E0D501F401282F30E0A401420F8B
:107D0000531F04C08C91919189278D93E417F50737
:107D1000C9F7A20EB31EE0EFFFEFEE0EFF1E8701C4
:107D2000040D151D10161106ACF26620E9F0D601FF
:107D30001F961C92C6010E948B3F8E010F5F1F4F42
:107D4000C8010E949D3F20E030E00CC0F801E20F26
:107D5000F31FD5018C9190818927F50181935F01F3
:107D60002F5F3F4F621691F760960FB6F894DEBF13
:107D70000FBECDBFCF91DF911F910F91FF90EF907C
:107D8000DF90CF90BF90AF909F908F907F906F903B
:107D90005F904F900895CF92DF92EF92FF920F93F2
:107DA0001F93DF93CF93CDB7DEB760970FB6F894EC
:107DB000DEBF0FBECDBF6C01F62E8C01E62E07C0D4
:107DC000C8010E948B3F005F1F4F80EFE80E8FE0DD
:107DD0008E15B0F30F2D0F70F2949FE0F9222F2D26
:107DE00030E084E0220F331F8A95E1F72C0D3D1D12
:107DF0000023D9F010E07E010894E11CF11CC701BA
:107E0000B901402F50E00E94FEBBE0E1F0E0E01B32
:107E1000F10B9701200F311FC90160E070E0AF0145
:107E20000E9419BCC7010E948B3F60960FB6F89460
:107E3000DEBF0FBECDBFCF91DF911F910F91FF909D
:107E4000EF90DF90CF9008959F92AF92BF92CF9224
:107E5000DF92EF92FF920F931F93DF93CF93CDB7F3
:107E6000DEB760970FB6F894DEBF0FBECDBF6C01D2
:107E70005B017A01122F902EFA01078780E090E0D3
:107E800060E040E00E94D13FC7010E948B3F80E04C
:107E900090E061E040E00E94D13F112301F1012F09
:107EA0001F3008F00EE019821A83E02EFF249E0195
:107EB0002D5F3F4FC901B601402F50E00E94FEBB2D
:107EC000602F6E5FCE0101960E94CB3E011738F401
:107ED000612F601BC6018E0D9F1D0E94CB3EC60107
:107EE000810F911D692D0E94CB3EC5010E949D3FCF
:107EF00060960FB6F894DEBF0FBECDBFCF91DF9175
:107F00001F910F91FF90EF90DF90CF90BF90AF90B7
:107F10009F9008950895FC0190E0819180933E0127
:107F20009F5F9031D1F780919B1B806880933C01CB
:107F300080913D0180FFFCCF0895FC0190E080918D
:107F40003E0181939F5F9031D1F708958091BC1BD2
:107F50009091BD1B0F9719F480E00E941B2008959B
:107F600080918327909184279093BD1B8093BC1BA5
:107F70000F9711F40E94092080917806882319F048
:107F8000ECEAFBE102C0ECE9FBE190E08191809337
:107F90003F019F5F9031D1F780919B1B80933C0103
:107FA00008950F931F93DF93CF93CDB7DEB76097FC
:107FB0000FB6F894DEBF0FBECDBFDC01162F042F25
:107FC0000097F1F010929A1B82E0809378062CE9DA
:107FD0003BE1AD0180E1FA010190AF01F9010192AD
:107FE0009F018150C1F720E030E0FD01E20FF31F57
:107FF000808180933F012F5F3F4F20313105A9F7EA
:10800000002321F0013009F047C00EC080917806AE
:10801000813079F5ECE9FBE1819180933F018BE1BF
:10802000EC3AF807C9F725C0809178068130A1F1B4
:1080300080919A1B8823A1F410929B1B10923C0103
:10804000CE0101960E948B3FECEAFBE180913F015B
:1080500081938BE1EC3BF807C9F781E080939A1B91
:10806000ECEAFBE1819180933F018BE1EC3BF80767
:10807000C9F700937806123078F4802F880F880FA4
:10808000880F88701295110F1072812B80939B1BA3
:1080900080933C0181E001C080E060960FB6F894C7
:1080A000DEBF0FBECDBFCF91DF911F910F9108951D
:1080B000089508950895089508951092BE28109285
:1080C000BD281092BF281092C0281092C12810928B
:1080D000C2281092C3281092C4281092C52810926A
:1080E000C628E7ECF8E28FEF9FEF9183808312823E
:1080F00013821482158216821782108611863A9690
:1081000029E2E132F20789F708950895089580EF92
:108110000E94913B89E796E00E9460BD81E08093D8
:10812000C21B80E50E94913B08958F929F92AF926F
:10813000BF92CF92DF92EF92FF920F931F93DF9344
:10814000CF93CDB7DEB7C65CD0400FB6F894DEBF94
:108150000FBECDBF282F6B015A01833309F487C1AD
:10816000843320F4823309F095C2E7C0863321F0CE
:108170008C3309F08FC282C2DA0112969C91129759
:1081800011968C91C82EDD24C90ED11CE5E0F0E0DB
:10819000CE0EDF1EC40ED51E8091F8149091F914F6
:1081A000009709F0BCC000D000D0EDB7FEB7319603
:1081B0008AE896E0ADB7BEB712969C938E9311975E
:1081C000DA018C91828313820E9424BD750100E044
:1081D00010E00F900F900F900F902EEB822E26E064
:1081E000922E22C00115110521F08AE390E00E9431
:1081F00059BD00D000D0EDB7FEB73196ADB7BEB7D0
:1082000012969C928E921197D70115968C9182832B
:1082100013820E9424BD0F5F1F4F0894E11CF11CC4
:108220000F900F900F900F90F501818190E008174B
:108230001907C0F200D081EC96E0ADB7BEB7129638
:108240009C938E9311970E9424BD00E010E00F9044
:108250000F909EEBE92E96E0F92E24C00115110532
:1082600021F08AE390E00E9459BD00D000D0ADB764
:10827000BEB71196EDB7FEB7F282E182F5018181BA
:10828000E00FF11FE80FF11D858112968C93129774
:1082900013961C920E9424BD0F5F1F4F0F900F90EA
:1082A0000F900F90D50112968C9190E00817190746
:1082B000A8F28E01055C1F4FB601685F7F4FC801B1
:1082C0000E948C8C00D000D086EC96E0EDB7FEB713
:1082D00092838183148303830E9424BD0F900F90A7
:1082E0000F900F90B601685E7F4FC8010E948C8C82
:1082F00000D000D087ED96E0ADB7BEB712969C9344
:108300008E93119714961C930E9313970E9424BD7D
:108310000F900F900F900F908AED96E004C0029797
:1083200020F48CED96E00E9460BDF50163817481BC
:10833000C60140810E94608DE5C1DA018C918530D3
:1083400009F48BC0863040F48330B9F0843028F5CE
:10835000813009F0D7C10CC0873009F440C08730A4
:1083600070F18B3009F442C08D3009F0CBC15FC091
:10837000FA0181818093A307C5C18A010F5F1F4F56
:1083800080E5B8010E94D73C80E50E94913B8EE0D9
:1083900090E062E070E0A8010FC0DA0111968D91C3
:1083A0009C9112979093BF1B8093BE1B8CE490E02E
:1083B00062E070E04EEB5BE10E941C12A3C1A5E6F7
:1083C000B6E2FA01319688E001900D928150E1F712
:1083D000B5016F5F7F4F80EF0E94D73C93C14F5F25
:1083E0005F4F88E090E066E070E0E6CF87E0E82E3F
:1083F000F12CEC0EFD1E89E0F70111928A95E9F748
:108400008CE2888782E08F878E01075E1F4FCA014A
:108410000196B8010E94E38B882309F473C1C80157
:10842000B70141E021E030E00E94E0846BC18AEFB7
:1084300096E0BE016F5F7F4F0E94FF948981809319
:108440006329C501029660E820E030E040E050E09A
:1084500003E010E00E94546655C10E94B561FC0122
:10846000E95EFE4FD50111968C91878B4BC1FA01C5
:108470002081253009F4EFC0263070F4223011F14C
:10848000233020F4213009F03DC118C02330E9F039
:10849000243009F037C11EC0283009F45BC02930F0
:1084A00030F4263029F1273009F02CC139C02930A9
:1084B00009F48AC02A3009F025C1A9C08091A30718
:1084C0002A83D2C02A832B83D0C08091A4079091A5
:1084D000A50704C08091BE1B9091BF1B2C839E8377
:1084E0008D8383E363E070E0AE014C5F5F4FC3C0F8
:1084F000FE01709689E0DF011D928A95E9F7288BCD
:10850000DE015196E5E6F6E288E001900D92815099
:10851000E1F783E369E070E0AE01405F5F4FABC01D
:108520008E01005F1F4F89E0F80111928A95E9F7EB
:10853000288B80E090E068E070E046E050E09E012B
:108540002F5E3F4F0E944E1283E369E070E0A80166
:108550000E942A8EFE01B99682E1DF011D928A9562
:10856000E9F788E089A70E94B561AC01B2E0CB16BB
:10857000D10408F4C7C0F501818190E027E131E022
:10858000829FF001839FF00D929FF00D1124E40F64
:10859000F51FD50112968C912DE1829FC001112407
:1085A0004996DE019B96E80FF91F80E101900D923C
:1085B0008150E1F7F50181818AA783E362E170E0F0
:1085C000AE01475D5F4F57C0FE01ED59FF4F82E39B
:1085D000DF011D928A95E9F721938F0181E00E94C6
:1085E0004998009741F0F801DC0181E30D90019278
:1085F0008150E1F705C081E3D8011D928A95E9F722
:1086000083E362E370E0AE014D595F4F34C0FE0179
:10861000EB56FF4F82E3DF011D928A95E9F789E06F
:1086200081938F0180E00E944998009741F0F80102
:10863000DC0181E30D9001928150E1F705C081E3F7
:10864000D8011D928A95E9F783E362E370E0AE01F9
:108650004B565F4F10C01B821A822A830E94B5615D
:10866000FC01E95EFE4F87898B8383E362E070E063
:10867000AE014E5F5F4F0E942A8E44C081E080931E
:108680006D26AEE6B6E2FA0186E001900D928150C9
:10869000E1F738C0EDB7FEB738970FB6F894FEBFD4
:1086A0000FBEEDBF31968FEF96E0ADB7BEB7129615
:1086B0009C938E931197B382A28224831582D782D2
:1086C000C6820E9424BD750100E010E0EDB7FEB740
:1086D00038960FB6F894FEBF0FBEEDBF0CC0609188
:1086E000793970917A39D7018D917D0190E00E949E
:1086F000F8BC0F5F1F4F0C151D0588F38FE297E044
:108700000E9460BDC5010E9457B7CA53DF4F0FB624
:10871000F894DEBF0FBECDBFCF91DF911F910F91B7
:10872000FF90EF90DF90CF90BF90AF909F908F9091
:108730000895662341F080E397E00E9460BD81E0E8
:108740000E94B13B08959093BF1B8093BE1B81E0B4
:1087500080932B298093C21B80E50E94913B089552
:10876000DF93CF930F92CDB7DEB7882321F081E05E
:108770000E94B13B16C021E02093C11B8091810370
:1087800090918203892B31F40E945D4083E56EEB6A
:108790007BE105C0298382E5BE016F5F7F4F0E94A8
:1087A000D73C0F90CF91DF9108950F93DF93CF9334
:1087B00000D00F92CDB7DEB721E02983882321F0C6
:1087C00081E00E94B13B48C0663409F440C0673480
:1087D00020F4613409F040C018C06235D9F0633527
:1087E000D9F58091810390918203892BA9F52A8381
:1087F00081E4BE016E5F7F4F0E94D73C84E18B8392
:1088000086E4BE016D5F7F4F25C082E5BE016F5FCC
:108810007F4F20C08091810390918203892B99F42E
:1088200041E050E060E070E00090A30704C0440F16
:10883000551F661F771F0A94D2F781E021E000E000
:108840000E945C3B09C080EF0E94913B05C085E41B
:1088500066EA77E00E94D73C0F900F900F90CF917F
:10886000DF910F910895EF92FF920F93DF93CF93D3
:10887000CDB7DEB729970FB6F894DEBF0FBECDBFD8
:108880007A01882321F081E00E94B13B67C0603FFC
:1088900009F047C0A5E6B6E2FA0188E001900D9222
:1088A0008150E1F78091810390918203892B91F0AF
:1088B00041E050E060E070E00090A30704C0440F86
:1088C000551F661F771F0A94D2F781E025E000E06C
:1088D0000E945C3B8091C11B882309F43FC0109229
:1088E000C11B88E08987F7018081888781818F8318
:1088F00082818E8383818D8384818C8385818B8328
:1089000086818A8387818983CE0101960E94E18ACC
:108910008091810390918203892B01F50E9434A6F6
:108920001DC06035D9F4FA01408151815093A507EB
:108930004093A4078091C21B882381F01092C21B30
:108940008091BF1B89838091BE1B8A8382E08987C7
:10895000CA01BE016F5F7F4F0E943E8A29960FB603
:10896000F894DEBF0FBECDBFCF91DF910F91FF9086
:10897000EF900895AF92CF92DF92EF920F93CF9343
:10898000DF93282F8091810390918203892BA1F49A
:108990008091A4079091A5076091A30740E02FE084
:1089A0000FE0EE24E394CC24AA240E94213B84E42B
:1089B00097E00E9460BD6BC02223E9F5E60100E06C
:1089C00031E5C32E37E0D32E5FC04B858091A307DE
:1089D0004817E1F58C858823C9F529813A81809172
:1089E000A4079091A5072817390781F5888182305F
:1089F00039F48B819C8190932229809321291FC077
:108A00008330C9F48B81809323298C81809324291E
:108A10008D81809325298E81809326298F81809353
:108A200027298885809328298985809329298A8503
:108A300080932A2904C081E00E94B13B28C0842F82
:108A400060E0AE0120E80E94163C21C000D000D0BA
:108A500000D0EDB7FEB73196ADB7BEB71296DC9237
:108A6000CE9211974283138289819A819583848360
:108A70000E9424BD61960F5F8DB79EB706960FB614
:108A8000F8949EBF0FBE8DBF0E1508F49ECFDF91E8
:108A9000CF910F91EF90DF90CF90AF9008956F92AC
:108AA0007F928F929F92AF92BF92CF92DF92EF927E
:108AB000FF920F931F93CF93DF93D22EC32EB42E2A
:108AC000A52E962E872E782E692E8DB79EB70A97E3
:108AD0000FB6F8949EBF0FBE8DBFEDB6FEB60894DC
:108AE000E11CF11C85E897E0EDB7FEB79283818326
:108AF000872D962D00E20E94CBAFC901BA01F70184
:108B00002283938344837583D682C782B086A186ED
:108B10000E9424BDE7ECF8E2C1E0D0E08DB79EB73B
:108B20000A960FB6F8949EBF0FBE8DBF00811181CB
:108B30009FEF0F3F190759F182818D1509F057C03A
:108B400083818C1509F053C084818B1509F04FC0C7
:108B500085818A1509F04BC08681891509F047C0C7
:108B60008781881509F043C08085871509F03FC0CB
:108B700081858615E1F52D2D3C2D4B2D5A2D692D26
:108B8000782D872D962DEE240E94D13B36C0FE0114
:108B9000EE0FFF1FCE0163E0880F991F6A95E1F782
:108BA000E80FF91FE354F74DC08311822D2D3C2DA2
:108BB0004B2D5A2D692D782D872D962D0C2F10E0D9
:108BC000EE240E94D13BFE01EE0FFF1FEE0FFF1FB0
:108BD000EC0FFD1FEE0FFF1FE154F74DD082C18255
:108BE000B282A382948285827682678206C02196B1
:108BF0003A96CA30D10509F099CFDF91CF911F91F4
:108C00000F91FF90EF90DF90CF90BF90AF909F902B
:108C10008F907F906F900895EF920F93DF93CF9393
:108C2000CDB7DEB70E940647CF91DF910F91EF904D
:108C30000895FC01DB0118968C911897883099F5FE
:108C40008C9192E089279085981709F057C09185FB
:108C500011968C911197981709F050C09285129631
:108C60008C911297981709F049C0938513968C91AF
:108C70001397981709F042C0948514968C91149715
:108C80009817E1F5958515968C9115979817B1F57C
:108C9000968516968C911697981781F520E0978502
:108CA00017968C9154C0863061F58C9192E089279B
:108CB0009085981719F5918511968C9111979817B1
:108CC000E9F4928512968C9112979817B9F48385DE
:108CD0008F3FA1F484858E3F89F4958513968C91FE
:108CE0001397981759F4968514968C9114979817A2
:108CF00029F420E0978515968C9129C080E090E0BA
:108D00000895823011F080E00895208530E0809150
:108D1000603190E08D7F28173907F9F491858091B3
:108D200061319817D1F482858823B9F483858F3F08
:108D3000A1F484858E3F89F48585882371F4968516
:108D40008C91981751F420E0978511968C91981387
:108D500021E081E02827822F089580E090E00895A7
:108D600081E08093E620089591E09093D8201092BE
:108D7000D92080E28093DA2082E08093DB208DE0AE
:108D80008093DC2088EB8093DD209093E62008958B
:108D90000F931F93CF93DF93EC011092E620109175
:108DA000D82001E010C0113061F48AED90E2BE01DC
:108DB00048E050E00E94F1BB009719F428ED30E242
:108DC00008C00093E6208091E620882361F320E02C
:108DD00030E0C901DF91CF911F910F9108950F935A
:108DE0001F93CF93DF93EC018B010E94C846892B20
:108DF00011F480E006C0CE01B8010E94194681112D
:108E000081E0DF91CF911F910F910895CF92DF9272
:108E1000EF92FF920F931F93DF93CF93CDB7DEB7FF
:108E20002A970FB6F894DEBF0FBECDBF7C016B0151
:108E300081E0809363291092C71B1092C51B80911B
:108E40005F29909160298093C31B9093C41B40932A
:108E5000612910926229B90150E00E94FEBBD7013E
:108E60002C91223081F414968C9114978983139657
:108E70008C918A8389819A8190934E2980934D2980
:108E800020935529B2C0233009F09AC0F7012381FD
:108E9000348145815681678170858185928508E39B
:108EA0000E94CBAF2B83D70113962C911397149666
:108EB0003C91149715964C91159716965C911697C0
:108EC00017966C91179718967C91189719968C9114
:108ED00019971A969C9100E30E94CBAF2C83F7015F
:108EE0002381348145815681678170858185928592
:108EF00008E20E94CBAF2D83D70113962C911397D4
:108F000014963C91149715964C91159716965C9172
:108F1000169717966C91179718967C911897199633
:108F20008C9119971A969C9100E20E94CBAF2E83E8
:108F3000F701238134814581568167817085818560
:108F4000928508E10E94CBAF2F83D70113962C9115
:108F5000139714963C91149715964C911597169665
:108F60005C91169717966C91179718967C911897A5
:108F700019968C9119971A969C9100E10E94CBAF9B
:108F80002887F70123813481458156816781708567
:108F90008185928508E00E94CBAF2987D70113967F
:108FA0008C918A87E1E6F9E27497DE01139688E0F6
:108FB0000D9001928150E1F788E08093552915C00A
:108FC00000D000D000D0EDB7FEB731968AEB97E025
:108FD000ADB7BEB712969C938E9311978EEC97E027
:108FE0009383828380E396E0C4C0D6012C91223023
:108FF00081F414968C911497898313968C918A83AB
:1090000089819A81909357298093562920935E29CC
:10901000BDC0233009F099C0F60123813481458118
:109020005681678170858185928508E30E94CBAF68
:109030002B83D60113962C91139714963C91149779
:1090400015964C91159716965C91169717966C91FC
:10905000179718967C91189719968C9119971A96CC
:109060009C9100E30E94CBAF2C83F60123813481D5
:1090700045815681678170858185928508E20E94CD
:10908000CBAF2D83D60113962C91139714963C9158
:10909000149715964C91159716965C9116971796FE
:1090A0006C91179718967C91189719968C9119972F
:1090B0001A969C9100E20E94CBAF2E83F601238189
:1090C000348145815681678170858185928508E16B
:1090D0000E94CBAF2F83D60113962C911397149631
:1090E0003C91149715964C91159716965C9116978E
:1090F00017966C91179718967C91189719968C91E2
:1091000019971A969C9100E10E94CBAF2887F6012F
:10911000238134814581568167817085818592855F
:1091200008E00E94CBAF2987D60113968C918A87DD
:10913000A6E5B9E2FE01339688E001900D928150D8
:10914000E1F788E080935E2921C000D000D000D0F4
:10915000EDB7FEB731968AEB97E0ADB7BEB7129682
:109160009C938E9311978EEC97E0938382838AE48D
:1091700096E0958384830E9424BDEDB7FEB73696B2
:109180000FB6F894FEBF0FBEEDBF1DC580ED90E297
:109190000E941287892B41F01092C91B1092C81BA4
:1091A0001092CB201092CA20E091C31BF091C41BF7
:1091B000908180E02181422F50E0482B592BCA0139
:1091C0008070987F892F9927803C910549F0803ED7
:1091D0009105C9F0EE24FF2410E020E030E025C026
:1091E0007FEFE72E77E0F72EE422F522928180E0F0
:1091F000238130E0282B392B8091C51B8C5F809315
:10920000C51B10E012C01481928180E0238130E000
:10921000282B392B6FEFE62E67E0F62EE422F5229D
:109220008091C51B8B5F8093C51B8091CA20909154
:10923000CB20892B39F1E114F10409F4C4C48091E5
:10924000C81B9091C91BE816F90609F0BCC48091AF
:10925000CE209091CF208217930709F0B4C40091DB
:109260004C2984E499E26DE479E2402F50E00E94B9
:10927000F1BB009709F0A7C480915529081709F0A0
:10928000A2C422C0E114F104F9F0F092C91BE092EB
:10929000C81B3093CF202093CE2080ED90E240E297
:1092A00051EA67E070E00E943B8724E439E2409194
:1092B0005529EDE4F9E2C901BF0150E00E94FEBB6F
:1092C0008091552980934C299091C51B953009F4C4
:1092D00008C44091C31B5091C41B292F30E0FA01F0
:1092E000E20FF31F6081862F807E803609F0DEC397
:1092F0002E5F3F4F240F351F3093E5202093E4204D
:10930000818187FF06C02F5F3F4F3093E520209378
:10931000E4208091C51BE091C31BF091C41BE80FB2
:10932000F11D808190E09C012071307083FD47C069
:10933000E091E420F091E520232B71F5ABECBBE14B
:10934000319683E001900D928150E1F7E091E420A5
:10935000F091E52040813496F093E520E093E420FD
:10936000242F30E0C9018F7390709595879595955E
:10937000879580668093CA1B46954695407396E014
:10938000220F331F9A95E1F7422B8091CB1B8F70F0
:10939000482B4093CB1B3FC080E68093CA1B908133
:1093A000892F8695869580739F70892B8093CB1B20
:1093B000818192819093CD1B8093CC1B1DC0232B68
:1093C00009F5E091E420F091E5208081869586956D
:1093D0008F7080668093CA1B8081982F9695969592
:1093E00090738295880F880F807C892B8093CB1B8C
:1093F0001092CD1B1092CC1B3396F093E520E09396
:10940000E42009C080E68093CA1B1092CB1B109207
:10941000CD1B1092CC1B8091C51BE091C31BF0911A
:10942000C41BE80FF11D808182FD0BC0E091E42098
:10943000F091E52081918093D01BF093E520E0939B
:10944000E4208091C51BE091C31BF091C41BE80F81
:10945000F11D808190E0837090708130910561F002
:10946000823091051CF4892B79F019C08230910566
:1094700029F00397A1F406C081E001C080E4809345
:10948000D11B0DC08FEFFBCFE091E420F091E520E0
:1094900081918093D11BF093E520E093E420E0914B
:1094A000C31BF091C41B8091C51BE80FF11D2181E6
:1094B000822F90E026FF86C027FD02C020E003C077
:1094C000228122952F7080739070892BF1F0109279
:1094D000E62091E00DC08091D820813039F4809150
:1094E000D920821719F488ED90E208C09093E62005
:1094F0008091E620882379F380E090E09093E32048
:109500008093E220892B09F4ECC28091C51BE09185
:10951000C31BF091C41BE80FF11D818190E08073A3
:10952000907080319105A9F0813191051CF4892B4F
:1095300041F0BFC08032910531F1C09709F0B9C048
:1095400032C080E1E2EDFBE1DF011D928A95E9F78F
:10955000B0C0E091E220F091E320A2EDBBE13296B1
:1095600088E001900D928150E1F7AAEDBBE1809176
:10957000E4209091E5209C01F90188E001900D9292
:109580008150E1F761C0E091E220F091E320A2ED8B
:10959000BBE1329688E001900D928150E1F786E0C0
:1095A000EAEDFBE160C0E091E220F091E320A2ED62
:1095B000BBE1329688E001900D928150E1F782ED97
:1095C0009BE173C0807390708031910521F18131EE
:1095D00091051CF4892B41F06CC080329105D1F1CA
:1095E000C09709F066C052C0A2EDBBE18091E420B3
:1095F0009091E5209C01F90180E101900D9281504C
:10960000E1F78091E4209091E52040969093E52049
:109610008093E4204EC08EEF8093D21B80E880932D
:10962000D31BE4EDFBE186E0DF011D928A95E9F7AB
:1096300036962091E4203091E520C901DC0188E0D4
:109640000D9001928150E1F78091E4209091E52006
:109650000896DCCF8EEF8093D21B80E88093D31BDB
:109660008CE0E4EDFBE1DF011D928A95E9F7E091E2
:10967000E420F091E520819191919093E11B8093FA
:10968000E01BF093E520E093E42013C08EEF80937D
:10969000D21B80E88093D31BE4EDFBE186E0DF0181
:1096A0001D928A95E9F7CF0102976DE479E20E9455
:1096B0000966E091C31BF091C41B8091C51BE80FA4
:1096C000F11D4181842F90E09C012470307043FF94
:1096D00078C0232B09F055C18370907081309105BB
:1096E000D9F0823091051CF4892B41F04AC18230B7
:1096F0009105A1F1039709F044C14EC0A2EEBBE170
:109700008091E4209091E5209C01F90180E1019095
:109710000D928150E1F7E1C08FEF8093E21BE09161
:10972000E420F091E52081918093E31B24EE3BE15E
:1097300089E0D9011D928A95E9F7D901199685E04A
:1097400001900D928150E1F78091E4209091E52005
:1097500006969093E5208093E42013C18FEF8093C9
:10976000E21BE091E420F091E52081918093E31BDE
:1097700024EE3BE18BE0D9011D928A95E9F7D901EE
:10978000199683E001900D928150E1F78091E420D9
:109790009091E5200496DDCF8FEF8093E21B82E06D
:1097A0008093E31B8DE0E4EEFBE1DF011D928A95DF
:1097B000E9F7E091E420F091E52081918093F11B9D
:1097C000C8C0232B09F46AC047FD02C090E002C064
:1097D00092819F701092E62021E00DC08091D820E8
:1097E000813039F48091D920891719F428ED30E2BD
:1097F00008C02093E6208091E620882379F320E0BA
:1098000030E03093E3202093E2202115310509F464
:1098100068C18091C51BE091C31BF091C41BE80F88
:10982000F11D818190E08370907082309105E9F0A4
:109830008330910539F1019709F0A3C0A2EEBBE195
:10984000F901329688E001900D928150E1F7AAEE7D
:10985000BBE18091E4209091E5209C01F90188E032
:1098600001900D928150E1F757C0A2EEBBE1F901E2
:10987000329688E001900D928150E1F786E0EAEEA1
:10988000FBE159C0A2EEBBE1F901329688E00190FC
:109890000D928150E1F782EE9BE16FC08370907072
:1098A0008130910501F1823091051CF4892B41F042
:1098B00068C082309105B1F1039709F062C04EC0D3
:1098C000A2EEBBE18091E4209091E5209C01F9019A
:1098D00080E101900D928150E1F78091E420909118
:1098E000E520409636CF8EEF8093E21B80E8809390
:1098F000E31BE4EEFBE186E0DF011D928A95E9F7C8
:1099000036962091E4203091E520C901DC0188E001
:109910000D9001928150E1F78091E4209091E52033
:10992000089617CF8EEF8093E21B80E88093E31BAD
:109930008CE0E4EEFBE1DF011D928A95E9F7E0910E
:10994000E420F091E520819191919093F11B809317
:10995000F01BF093E520E093E42013C08EEF80939A
:10996000E21B80E88093E31BE4EEFBE186E0DF018D
:109970001D928A95E9F7CF01029766E579E20E9488
:1099800009668091C71B885D8093C71B8091C51BAA
:10999000E091C31BF091C41BE80FF11D808182FF91
:1099A00056C0A091E420B091E5208C91887F803F43
:1099B00009F04DC081E18093D01B8C91803F29F14B
:1099C000833F09F08EC0EAECFBE1B89611968C91CA
:1099D000119782958F7090E080559F409093F21B75
:1099E000818311968C91119790E08F7090708055C3
:1099F0009F409283838312968D919C9113979093AD
:109A0000F91B8093F81B149619C011968D919C91A7
:109A100012979093F31B8093F21B13968D919C9158
:109A200014979093F51B8093F41B15968D919C9140
:109A300016979093F91B8093F81B1796B093E52027
:109A4000A093E4208091C71B885F8093C71B9091EF
:109A5000E4208091C31B981B9093C51BE114F10473
:109A600051F41092CE1B8091C71B8852891B909194
:109A70006129890F0CC0E8EDFFEFEE0EFF1EF0929A
:109A8000CE1B88E290E0E80EF91E8E2D885280935E
:109A9000CF1B8091D01B813121F58091CE1B9091FD
:109AA000CF1B9093F71B8093F61B1BC0613409F00A
:109AB0008AC0892F8F5F8093C51BAAECBBE1FA0196
:109AC000E80FF11D88E201900D928150E1F780913D
:109AD000C51B885D8093C51B8091C71B885D8093E3
:109AE000C71B409161299091C51B491B4093C61B20
:109AF000212F30E083E0220F331F8A95E1F7809118
:109B0000C71B280F311D2653344EE091C31BF09123
:109B1000C41BE90FF11DC901BF0150E00E94FEBB4B
:109B2000EF28C9F08091CA209091CB20892B31F485
:109B30008091C71B8093CA201092CB202091C61B16
:109B40008091CA209091CB20820F911D9093CB20C1
:109B50008093CA200BC02091C71B8091C61B90E048
:109B6000820F911D9093C91B8093C81B2091CA201E
:109B70003091CB202115310539F08091C81B90918F
:109B8000C91B28173907F9F403EE19E22AEC3BE167
:109B90004091C81B5091C91BC801B9010E94FEBB6E
:109BA0006091C81B7091C91B1092C91B1092C81BF1
:109BB0001092CB201092CA2010926529109264292D
:109BC000C8010E9489692A960FB6F894DEBF0FBEBD
:109BD000CDBFCF91DF911F910F91FF90EF90DF905C
:109BE000CF9008956F927F928F929F92AF92BF9283
:109BF000CF92DF92EF92FF920F931F93DF93CF9359
:109C0000CDB7DEB72B970FB6F894DEBF0FBECDBF32
:109C10003C01FE0131968BE0DF011D928A95E9F748
:109C200082E089832091A4073091A5076114710413
:109C300039F48FEF9FEF9D838C833B832A8313C07E
:109C40003B832A83F3014085423079F4308120E060
:109C5000818190E0822B932B9D838C8349838F5F3E
:109C60009F4F09F0B8C050E0B7C0483009F09EC01F
:109C7000D3012C9130E040E050E060E070E080E003
:109C800090E008E30E944AB0122FF32EE42ED52E66
:109C9000C62EB72EA82E992EF301218130E040E088
:109CA00050E060E070E080E090E000E30E944AB0A5
:109CB000122BF32AE42AD52AC62AB72AA82A992AD7
:109CC000D30117968C911797182B12962C9130E090
:109CD00040E050E060E070E080E090E008E20E9448
:109CE0004AB0122BF32AE42AD52AC62AB72AA82A70
:109CF000992AF301238130E040E050E060E070E019
:109D000080E090E000E20E944AB0122BF32AE42A9D
:109D1000D52AC62AB72AA82A992AD30114962C91A3
:109D200030E040E050E060E070E080E090E008E18A
:109D30000E944AB0122BF32AE42AD52AC62AB72A4F
:109D4000A82A992AF301258130E040E050E060E044
:109D500070E080E090E000E10E944AB0122BF32A0C
:109D6000E42AD52AC62AB72AA82A992AD301169600
:109D70002C9130E040E050E060E070E080E090E066
:109D800008E00E944AB0122BF32AE42AD52AC62AF8
:109D9000B72AA82A992A1C83FD82EE82DF82C88610
:109DA000B986AA869B8683E0898315C000D000D03F
:109DB00000D0EDB7FEB7319682EF97E0ADB7BEB7F2
:109DC00012969C938E9311978EEC97E093838283E7
:109DD00080E395E029C051E08091632990E0FC0187
:109DE000B3E0EE0FFF1FBA95E1F7E80FF91FE45952
:109DF000F64D8085823029F1883011F483E022C04D
:109E000000D000D000D0EDB7FEB7319682EF97E0DA
:109E1000ADB7BEB712969C938E9311978EEC97E0D8
:109E2000938382838BE395E0958384830E9424BD92
:109E3000EDB7FEB736960FB6F894FEBF0FBEEDBF76
:109E400015C082E020915F2930916029BE016F5FCB
:109E50007F4F4091612900E2E52ECC24AA2488247A
:109E60000E94563C10926229109261292B960FB6DF
:109E7000F894DEBF0FBECDBFCF91DF911F910F9140
:109E8000FF90EF90DF90CF90BF90AF909F908F901A
:109E90007F906F9008951F93CF93DF93EC01109202
:109EA000C71B1092C51B1092622910926129E09184
:109EB0005F29F0916029F093C41BE093C31B329695
:109EC000F093E520E093E420329780E68083809150
:109ED000C51BE091C31BF091C41BE80FF11D11825B
:109EE0008091C51BE091C31BF091C41BE80FF11DCD
:109EF00012828BEF99E20E94C846892B31F48BEED7
:109F000099E20E94C846892BB1F08091C51B90E070
:109F10000196E091C31BF091C41BE80FF91F8081EB
:109F2000806880838091E4209091E5200196909351
:109F3000E5208093E4208091E329482F50E0909120
:109F4000E4299A0184E0220F331F8A95E1F7892FD3
:109F500082958F70822B282F269526958295880FC3
:109F6000880F807C282B692F70E0CB018F70907058
:109F7000892B99F58091E5299091E629892B69F53E
:109F80008091C51BE091C31BF091C41BE80FF11D2C
:109F90008081886080838091E32990E08F70907049
:109FA000892B81F48091E429807F61F48091C51B25
:109FB000E091C31BF091C41BE80FF11D808180610B
:109FC000808355C0E091E420F091E52020838091CA
:109FD000E4209091E520019646C04F705070452BCB
:109FE00041F5862F807F29F58091C51BE091C31B29
:109FF000F091C41BE80FF11D808180618083E091A6
:10A00000E420F091E520207C8091E4298F70282BBA
:10A010002083E091E420F091E5208091E529909162
:10A02000E629928381838091E4209091E520039634
:10A030001AC0E091E420F091E5208091E32990910D
:10A04000E429A091E529B091E62980839183A28338
:10A05000B383E091E420F091E52020838091E42017
:10A060009091E52004969093E5208093E4208091E0
:10A07000E929813161F48091C51BE091C31BF09106
:10A08000C41BE80FF11D8081846080830EC0E091C5
:10A09000E420F091E52080838091E4209091E520F8
:10A0A00001969093E5208093E4208091EA29803402
:10A0B00079F08F3FC9F0813011F58091C51BE09197
:10A0C000C31BF091C41BE80FF11D808181600AC0A1
:10A0D0008091C51BE091C31BF091C41BE80FF11DDB
:10A0E00080818260808319C08091C51BE091C31B71
:10A0F000F091C41BE80FF11D80818360F3CFE091E4
:10A10000E420F091E52080838091E4209091E52087
:10A1100001969093E5208093E4208091EB29909123
:10A12000EC29892BB9F58091ED299091EE29892BA5
:10A1300089F58091EF299091F029892B59F580912B
:10A14000F1299091F229892B29F58091F329909199
:10A15000F429892BF9F48091F5299091F629892B1E
:10A16000C9F48091F7299091F829892B99F480916D
:10A17000F9299091FA29892B69F48091C51B90E007
:10A180000196E091C31BF091C41BE80FF91F808179
:10A19000806446C08BEE99E20E94C8469093E3200B
:10A1A0008093E220892B09F46EC08091C51B90E05A
:10A1B0000196E091C31BF091C41BE80FF91F808149
:10A1C000806C80838091C51B90E00296A091C31B98
:10A1D000B091C41BA80FB91FE091E220F091E320D9
:10A1E00081818295807F9C91892B8C9360916329DA
:10A1F00089E0689FB00111246459764D8BEE99E295
:10A200000E941946882371F08091C51B90E0019649
:10A21000E091C31BF091C41BE80FF91F808180639C
:10A220008083B3C08091F3299091F429892B81F424
:10A230008091F5299091F629892B51F48091F72985
:10A240009091F829892B21F48091F92987FF4AC040
:10A250008091C51B90E00196E091C31BF091C41B57
:10A26000E80FF91F8081806180832091E420309184
:10A27000E520C901DC01E3EFF9E288E001900D92ED
:10A280008150E1F766C08091EB298E3F09F067C0ED
:10A290008091EC29803809F062C06091632989E0DF
:10A2A000689FB00111246459764D8BEE99E20E94AB
:10A2B0001946882309F0A8CF8091F3299091F429B9
:10A2C000892B69F58091F5299091F629892B39F52B
:10A2D0008091F7299091F829892B09F58091F92926
:10A2E00087FD1DC08091C51B90E00196E091C31BC6
:10A2F000F091C41BE80FF91F808180628083E09198
:10A30000E420F091E5208091F9299091FA29918338
:10A3100080838091E4209091E520029632C0809164
:10A32000C51B90E00196E091C31BF091C41BE80FA0
:10A33000F91F8081806180832091E4203091E520A5
:10A34000C901DC01E3EFF9E288E001900D92815050
:10A35000E1F78091E4209091E520089612C0809169
:10A36000E4209091E5209C01D901EBEEF9E280E137
:10A3700001900D928150E1F78091E4209091E520C9
:10A3800040969093E5208093E4208091FB298F3FB5
:10A3900009F0DDC08091C51B90E00196E091C31BE0
:10A3A000F091C41BE80FF91F808188608083809141
:10A3B000FC29823009F042C08091FD299091FE294C
:10A3C000892BE1F58091FF299091002A892BB1F525
:10A3D0008091012A9091022A892B81F58091032A8C
:10A3E0009091042A892B51F58091052A9091062A93
:10A3F000892B21F58091072A9091082A892BF1F465
:10A400008091092A8823D1F48091C51B90E00196A0
:10A41000E091C31BF091C41BE80FF91F808183609A
:10A420008083E091E420F091E52080910A2A8083E6
:10A430008091E4209091E520019671C18091FD29E1
:10A440009091FE29892B09F074C08091FF29909189
:10A45000002A892B09F06DC08091012A9091022A6F
:10A46000892B09F066C08091032A9091042A892BD8
:10A4700081F58091052A9091062A892B51F58091CA
:10A48000072A882331F58091C51B90E00196E09161
:10A49000C31BF091C41BE80FF91F80818260808389
:10A4A000E091E420F091E5208091FC298083E09107
:10A4B000E420F091E5203196A8E0BAE283E00D9027
:10A4C00001928150E1F78091E4209091E52004967B
:10A4D00026C18091032A9091042A892B51F58091FD
:10A4E000052A882331F58091C51B90E00196E09103
:10A4F000C31BF091C41BE80FF91F8081816080832A
:10A50000E091E420F091E5208091FC298083E091A6
:10A51000E420F091E5203196A6E0BAE285E00D90C6
:10A5200001928150E1F78091E4209091E520069618
:10A53000F6C08091E4209091E5209C01D901EBEFD9
:10A54000F9E280E101900D928150E1F7E3C08BEFD9
:10A5500099E20E94C8469093E3208093E220892BE1
:10A5600009F459C08091C51B90E00196E091C31B8E
:10A57000F091C41BE80FF91F808184608083809173
:10A58000C51B90E00296E091C31BF091C41BE80F3D
:10A59000F91FA091E220B091E320808111969C9157
:10A5A000892B80838BEF99E2BE010E941946882394
:10A5B00009F042C08091032A9091042A892B81F4EA
:10A5C0008091052A9091062A892B51F48091072ABF
:10A5D0009091082A892B21F48091092A87FF50C085
:10A5E0008091C51B90E00196E091C31BF091C41BC4
:10A5F000E80FF91F8081816080832091E4203091F1
:10A60000E520C901DC01E3E0FAE288E001900D9267
:10A610008150E1F76CC08091FB298E3F09F06DC03D
:10A620008091FC29803809F068C08BEF99E2BE0167
:10A630000E941946882371F08091C51B90E0019615
:10A64000E091C31BF091C41BE80FF91F8081836068
:10A65000808369C08091032A9091042A892B69F52F
:10A660008091052A9091062A892B39F58091072A35
:10A670009091082A892B09F58091092A87FD1DC030
:10A680008091C51B90E00196E091C31BF091C41B23
:10A69000E80FF91F808182608083E091E420F091CF
:10A6A000E5208091092A90910A2A918380838091E4
:10A6B000E4209091E520029632C08091C51B90E085
:10A6C0000196E091C31BF091C41BE80FF91F808134
:10A6D000816080832091E4203091E520C901DC0174
:10A6E000E3E0FAE288E001900D928150E1F7809179
:10A6F000E4209091E520089612C08091E42090918A
:10A70000E5209C01D901EBEFF9E280E101900D9287
:10A710008150E1F78091E4209091E520409690935C
:10A72000E5208093E42088E28093C71B8091E9298B
:10A73000813109F064C090910B2A80910C2A805BD2
:10A74000904F0F9770F590910D2A80910E2A20EF6F
:10A75000803B920730F18F5B904F18F5E091E42039
:10A76000F091E52083EF8083E091E420F091E520F3
:10A7700090910E2A905B80910C2A8295807F980F91
:10A780009183E091E420F091E5208091112A90914D
:10A79000122A938382838091E4209091E52004968D
:10A7A00025C0E091E420F091E52080EF8083E091E6
:10A7B000E420F091E52080910B2A90910C2AA09141
:10A7C0000D2AB0910E2A81839283A383B483E091F2
:10A7D000E420F091E5208091112A9091122A96832D
:10A7E00085838091E4209091E52007969093E52061
:10A7F0008093E4208091C71B885F8093C71BA09142
:10A80000E4208091C31BA81BA093C51B8091C71B8C
:10A81000482F50E0E0916429F0916529E41BF50B85
:10A820002A2F30E085E690E0821B930B6091C31BDA
:10A830007091C41B8E179F0708F0EAC0CB010496E5
:10A840004A2F50E00E9407BCE091C31BF091C41B4B
:10A850008091642990916529906C9083E091C31B4D
:10A86000F091C41B809164298183E091C31BF09116
:10A87000C41B8091CD208283E091C31BF091C41B47
:10A880008091CC2083838091C51B8C5F8093C51BF6
:10A8900015E6412F481B487F4093C61B6091C31BA0
:10A8A0007091C41B680F711D2091C71B30E02D51A2
:10A8B000364DCB01B90150E00E94FEBB2091C51B73
:10A8C0008091C61B90E0820F911D90936229809326
:10A8D0006129CE010E94F24D2091C71B8091C61BB9
:10A8E00090E0820F911D9093CB208093CA2085E049
:10A8F0008093C51BE091C31BF091C41B8091642918
:10A9000090916529906E9083E091C31BF091C41BD8
:10A910008091642981838091C51B181B187F109337
:10A92000C61B5CC0E091C31BF091C41B13E03695BD
:10A9300027951A95E1F72483609164297091652920
:10A940004091CA205091CB209B01241B350B809154
:10A95000C61B90E02817390720F4862F841B8093AC
:10A96000C61B8091C51B6091C31B7091C41B680FEF
:10A97000711D4091C61B2091CA203091CB202D51D2
:10A98000364DCB01B90150E00E94FEBB2091C51BA2
:10A990008091C61B90E0820F911D90936229809355
:10A9A0006129CE010E94F24D1092E62007C00E945C
:10A9B000083D8091E6208F5F8093E6208091E6201D
:10A9C0008233A8F32091C61B8091CA209091CB209E
:10A9D000820F911D9093CB208093CA202091CA2092
:10A9E0003091CB20809164299091652928173907EF
:10A9F00008F498CF8091CC209091CD20019690932F
:10AA0000CD208093CC201092CB201092CA201CC065
:10AA1000260F371F4D51564DC901BA01AF010E9493
:10AA2000FEBB2091C51B8091642990916529820FFE
:10AA3000911D2091C71B821B9109909362298093DD
:10AA40006129CE010E94F24D81E0DF91CF911F91EB
:10AA50000895FC015381560F50936B29272F3327FC
:10AA60004281420F40936A29A181A0936929E08124
:10AA7000E0936829842F90E08217930748F48A2F87
:10AA80008F5F80936929882319F4EF5FE093682929
:10AA9000852F90E070708617970790F4842F8F5F52
:10AAA00080936A29882361F4809169298F5F80935C
:10AAB0006929882329F4809168298F5F8093682908
:10AAC00008959C0141505040460F571FFB010EC096
:10AAD000708160E08181DB01A80FB11D2A0F3B1F4F
:10AAE0002A173B0710F42F5F3F4F3296E417F50704
:10AAF00078F3E417F50749F4908180E0280F391FB7
:10AB00002817390710F42F5F3F4FC90108959C01A2
:10AB1000AB0180E090E0B9010E946155282F892F98
:10AB2000922F089580E090E063EE79E248E250E0F1
:10AB30000E946155009719F42FEF3FEF02C0382FA4
:10AB4000292FC90108950F931F931091E72900E061
:10AB50009091E820091B11099091E829090F111D16
:10AB60009801280F311DC9016BEE79E240E250E0F7
:10AB70000E9461556091E82070E0655F754DA80105
:10AB80000E946155009719F42FEF3FEF02C0382F54
:10AB9000292FC9011F910F9108958AE30E94A3559F
:10ABA000089586E00E94A355089581E10E94A3556F
:10ABB00008950F931F93CF93DF93182F092F409180
:10ABC000EB205091EC20BCE24F5F5F4F8DE74030AF
:10ABD000580710F040E050E1342F252FA0E00EC0C0
:10ABE000AB9FF0011124E957F64D85A1882329F088
:10ABF000808991898217930739F3AF5FA23081F77B
:10AC00004093EB205093EC201092EA20E0E0F0E03B
:10AC100020E03CE21AC0239FD0011124A957B64D71
:10AC200095968C919597882321F42093EA20FD0135
:10AC300010C0873049F4309731F096969C919697E2
:10AC400086A1891708F4FD012F5F223020F320939D
:10AC5000EA20309771F182E085A38091ED20808F0A
:10AC60008091EE20818F8091EF20828F8091F02063
:10AC7000838F84EC94E0978F868F91A380A381E0EB
:10AC800090E0958F848F17A281E086A383E084A350
:10AC900012A280E183A3508B418B738B628BEF01F7
:10ACA000212F302FC901DC0180E10D9009928150E4
:10ACB000E1F7CF01DF91CF911F910F910895AC0182
:10ACC0001092EA2020E013C0E22FF0E0322F3F5F25
:10ACD000EE0FFF1FE152F64D808191818417950799
:10ACE00029F42093EA20118210820895232F223024
:10ACF00058F32093EA200895AC011092EA2020E056
:10AD000012C0E22FF0E0322F3F5FEE0FFF1FE15243
:10AD1000F64D80819181892B29F42093EA2051837B
:10AD200040830895232F223060F32093EA20089572
:10AD3000BC01809185299091862944960E942955CD
:10AD4000E0918529F091862980916829848B8091F2
:10AD50006929858B80916A29868B80916B29878BE5
:10AD60000895282F892F922F0895EF92FF920F9325
:10AD70001F939C0144275527F22EE32E00E010E09C
:10AD8000362F272F40E050E0A90133272227E22A5F
:10AD9000F32A042B152BB701C8011F910F91FF90C7
:10ADA000EF900895FC01409166295091672923EEA8
:10ADB0003EE2241B350B621773070CF49B0112163D
:10ADC000130664F42093E52E3093E62EE417F5077E
:10ADD00029F0CA01BF01A9010E94FEBB089582E0CB
:10ADE0008093E920A091E8202A2F30E0F901E55F67
:10ADF000F54D8181682F70E0F3E0660F771FFA95BB
:10AE0000E1F7695F7F4F42E0285D3F4F3CC0F901A9
:10AE1000E80FF91FED51F64D8081882319F081303C
:10AE200019F42EC04F5F2FC090E0807C9070803866
:10AE3000910549F0803C910549F08034910501F578
:10AE40004093E92009C04093E92008C04093E920DD
:10AE50008091FB298F3F11F481E00895242F30E089
:10AE600040E050E02A0F311D411D511D285D3F4F2C
:10AE70004F4F5F4F84E062E00E94CE6D82E0089504
:10AE800081818E5F480F842F90E0681779070CF05E
:10AE9000BECF4093E92080E008950F931F93CF9396
:10AEA000DF93C0918529D0918629843009F4C5C2E9
:10AEB0000FE11AE2109384290093832910936729E4
:10AEC00000936629833069F48DA18F70833011F06F
:10AED0000C94F25F8C8D9D8D892B11F00C94F25F98
:10AEE00093C0823009F094C01092652910926429B1
:10AEF0001092E62E1092E52E8091F0208F5F8093C5
:10AF0000F020882399F48091EF208F5F8093EF20C9
:10AF1000882361F48091EE208F5F8093EE20882358
:10AF200029F48091ED208F5F8093ED202DA12730B3
:10AF300011F0253051F48EA18F5F8EA3883711F068
:10AF40000C94F25F1DA20C94F25F222311F40C9476
:10AF5000F25F8C8D9D8D892B09F452C08EA181509A
:10AF60008EA38F5F11F00C94F25F3FA1383029F06F
:10AF70002150223048F4353039F41DA280E8809306
:10AF80007E290E94B36FD0C6353010F080E307C031
:10AF900083E090E002C0880F991F3A95E2F78EA3F4
:10AFA0008FA18F5F8FA38DA190E08F709070833001
:10AFB000910501F1843091054CF48130910509F43B
:10AFC00061C4029711F00C94F25F0DC086309105B8
:10AFD00009F4BEC68830910509F4BAC6049711F089
:10AFE0000C94F25FB5C6E091E820F0E0E55FF54D26
:10AFF00015864FC484E080937E290E94B36FD6C625
:10B000002F70233009F0EEC788E080937E2980C638
:10B01000853019F5E0918129F09182298089918903
:10B02000892B09F4DFC71092862910928529C8015F
:10B030000C97909384298093832990936729809318
:10B0400066291092E62E1092E52E10926529109234
:10B05000642988E080937E29EEC18091E329807F76
:10B06000803609F0BFC79091E72980E02091E82958
:10B07000AC01420F511D9A0180916429909165297C
:10B080008417950708F4AEC7285D3F4F30936529B4
:10B09000209364298091EB298F3F09F4A3C7C8014D
:10B0A000849760E840E050E00E94B063892B09F08B
:10B0B00067C0C80184970E942561882309F060C099
:10B0C0008091FB298F3F09F058C08091FC29823084
:10B0D00009F053C08091FD299091FE29892B09F038
:10B0E0004CC08091FF299091002A892B01F5809115
:10B0F000012A9091022A892BD1F48091032A909100
:10B10000042A892BA1F48091052A9091062A892B83
:10B1100071F48091072A9091082A892B41F480913B
:10B12000092A882321F480910A2A813049F18091EB
:10B13000FF299091002A892B01F58091012A909195
:10B14000022A892BD1F48091032A9091042A892B19
:10B15000A1F48091052A9091062A892B71F480919F
:10B16000072A9091082A892B41F48091092A882383
:10B1700021F480910A2A823019F00E9401603AC7B6
:10B1800089EE99E29093802980937F291092E8209C
:10B190001092E720E0917F29F091802980818B3205
:10B1A00009F44BC08C3248F4863009F4B1C18131C6
:10B1B00009F4B5C0882389F06BC08A3309F474C0E0
:10B1C0008B3320F48C3209F063C00CC78B3309F445
:10B1D00009C78C3309F05CC006C08091E72080FD70
:10B1E00057C0816009C08091E72081FF04C086FDBF
:10B1F0004FC0806401C082608093E7200E94EF56B8
:10B20000813009F4EFC6813018F0823019F6F2C6A9
:10B210002091E820E22FF0E0CF01855F954D9093DB
:10B22000802980937F29285FFC018181880F880F06
:10B23000880F280F2093E820ADCF8091E72082FD72
:10B2400027C084608093E7209091E820E92FF0E008
:10B25000DF01A55FB54D13968C911397882349F0B4
:10B26000BA969F01442737FD4095542F84E060E053
:10B2700018C0B0938029A0937F29985FE55FF54DB2
:10B280008181880F880F880F980F9093E82082CFD4
:10B29000E35EF9429F01442737FD4095542F84E037
:10B2A00061E00E94CE6DA6C60E94CD558F5F9F4F74
:10B2B00009F098C6E091E820F0E0E55FF54DE08107
:10B2C000E538B9F0E63828F4E038B1F0E138D9F4DF
:10B2D00018C0E73829F0E73848F0E838A1F403C08F
:10B2E0000E94187914C00E94347711C00E94F57032
:10B2F0000EC00E94207E0BC00E9458050E94AD6EB9
:10B3000006C00E94289D10926529109264298091A0
:10B31000642990916529892B09F464C66BC68091D4
:10B32000642990916529C097909365298093642939
:10B3300083E19AE29093842980938329E091E82025
:10B34000F0E0E55FF54D86819781892B31F00E9411
:10B35000D5558F5F9F4F09F045C687EE9EE29093CB
:10B3600082298093812948C028893989211531058E
:10B37000F1F18091E820E82FF0E0E55FF54D828162
:10B3800093818217930799F52A893B892115310505
:10B3900029F0808191818217930749F588819981ED
:10B3A000892BE1F48A819B81892BC1F48C819D8159
:10B3B000892BA1F48E819F81892B81F488859985C1
:10B3C000892B61F48A859B85892B41F48C859D8529
:10B3D000892B21F48E859F85892BC1F08BEE99E214
:10B3E000BE0140E150E00E94F1BB009779F0699600
:10B3F000D0938229C0938129C0918129D09182293B
:10B40000BFE2C931DB0708F4AFCFECC51092862943
:10B410001092852982E080937E2983E19AE29093BD
:10B4200084298093832990936729809366291092B9
:10B43000E62E1092E52E0E94736D2091E52E30913C
:10B44000E62E2115310509F4CDC5C901C0969093AA
:10B45000652980936429285F3F4F3093E7298852FC
:10B460008093E829A0918129B091822954968C91EA
:10B4700054978093EA2981E18093E929E091E820BB
:10B48000F0E0E55FF54D34832583178216825096F0
:10B490008D919C9151979183808352968D919C912F
:10B4A000539793838283ABEFB9E220918129309146
:10B4B0008229C901FC0180E101900D928150E1F7E0
:10B4C0008BEE99E26BEF79E20E9411658FE19AE2CF
:10B4D00090938429809383298091E820C82FD0E01D
:10B4E000C55FD54D0E94D555809590959F838E83DD
:10B4F0008091E820E82FF0E0E55FF54D86819781A7
:10B50000892B09F065C58FEF9FEF9783868360C510
:10B510000E94D1558F5F9F4F09F064C58091E8204C
:10B52000082F10E0055F154DC7E8D9E28DA18823EB
:10B53000D9F0D80112962D913C9113978889998959
:10B540002817390789F42D913C918A899B892817FE
:10B55000390751F48BEE99E2BE0140E150E00E94C0
:10B56000F1BB009709F4B2C1AC96B9E2C33BDB076B
:10B57000E9F2E0F2F80185858F73823001F582816E
:10B5800093819093F3208093F2201092EA2013C0CD
:10B59000E42FF0E0EE0FFF1FE152F64D2091F22074
:10B5A0003091F320808191812817390709F489C0EF
:10B5B0004F5F4093EA204091EA20423048F3809167
:10B5C000E820E82FF0E0DF01A55FB54D1D968C91D6
:10B5D0001D9782FD07C584E11D968C931D978CE312
:10B5E00090E09093652980936429FD0180E584872C
:10B5F00097811B968C911B9717968C93179793871F
:10B6000096811A968C911A9716968C931697928714
:10B61000958119968C91199715968C93159791870A
:10B6200094819093EA2018968C91189714968C9395
:10B63000149790871B968C911B978F5F1B968C930A
:10B640001B978823C1F41A968C911A978F5F1A96CC
:10B650008C931A97882379F419968C9119978F5F98
:10B6600019968C931997882331F418968C91189712
:10B670008F5F18968C93E091E820F0E0DF01A55FE2
:10B68000B54D2D913C9111973093F3202093F220EA
:10B69000FD01828193819183808313963C932E9345
:10B6A0001297EBEFF9E2DF01509780E10D900192E4
:10B6B0008150E1F78BEE99E26BEF79E20E94116520
:10B6C00054C41092EA20C0E0D0E04CE250E03CE2EA
:10B6D00025C0822F90E0849FF001859FF00D949FFC
:10B6E000F00D1124E957F64D85A1882339F48CE239
:10B6F000289FE0011124C957D64D14C0873059F452
:10B70000209721F096A18EA1891728F4239FE001AC
:10B710001124C957D64D2F5F2093EA202091EA20AB
:10B720002230B8F2209709F45DC4D0938629C093E3
:10B73000852983E08EA38CA31AA284E08BA31FA289
:10B74000E091E820F0E0E55FF54D82819381998BEF
:10B75000888B808191819B8B8A8BDE01EBEEF9E2F5
:10B7600080E101900D928150E1F781E08DA38091FD
:10B77000ED20888F8091EE20898F8091EF208A8F35
:10B780008091F0208B8F81E090E09D8F8C8FE091F5
:10B79000E820F0E0E55FF54D87818F8BE091E820B0
:10B7A000F0E0E55FF54D86818E8BE091E820F0E0DA
:10B7B000E55FF54D85818D8BE091E820F0E0E55F58
:10B7C000F54D84818C8B81E090E00E949856E09149
:10B7D000E820F0E0E55FF54D848590E0807F907093
:10B7E000813591050CF44EC01092EA2035C0F90164
:10B7F000ED51F64D84AD8093F120882309F442C0C9
:10B80000813021F44F5F4093EA2026C08230C1F49A
:10B8100085AD8430A9F436AD20E087AD90E0822B71
:10B82000932B9093F3208093F220F4E0853C9F07C4
:10B8300010F084EC94E09F8F8E8F99A388A322C090
:10B840008091EA20E82FF0E0E05EF54DE081EE2304
:10B85000C9F0E80FE093EA204091EA20242F30E07D
:10B86000E091E820F0E0E55FF54D848582958F70EA
:10B8700090E00597880F991F880F991F281739079F
:10B880000CF4B5CFE091E820F0E0E55FF54D80E104
:10B890008587E091E820F0E0DF01A55FB54D1D96BA
:10B8A0008C911D9782601D968C931D97FD0182E0FF
:10B8B000848B84E0858B868B84EC878B80E490E09E
:10B8C000909365298093642980E60EC3D0938629DE
:10B8D000C093852910927E298091E820A82FB0E09E
:10B8E000FD01E55FF54D858582FF03C01DA280E265
:10B8F00093C2848582958F70880F880F8093EA2089
:10B90000209164293091652928523040281B310943
:10B9100030936529209364298DA18F70823039F48A
:10B92000A55FB54D1D968C918F73823139F1232B14
:10B9300059F4E091E820F0E0E55FF54D858590E071
:10B9400083709070892BD1F08091E820E82FF0E08F
:10B95000E55FF54D94818C89981709F0B2C2958105
:10B960008D89981709F0ADC296818E89981709F0D4
:10B97000A8C297818F89981709F0A3C2E091E820A7
:10B98000F0E0E55FF54D858584FF52C06C8D7D8DBF
:10B990006115710509F44CC0CE0148960E942955E5
:10B9A0008091E820E82FF0E0E55FF54D208580915B
:10B9B00068292817E9F59185809169299817C1F5BB
:10B9C000928580916A29981799F5938580916B29C2
:10B9D000981771F5288F80916929898F80916A293C
:10B9E0008A8F80916B298B8F8FA18823D1F42AA114
:10B9F0009CA18EA1981B822F869586958695981B73
:10BA0000392F320F3AA38BA1282F26952695821B1A
:10BA100097FD9195890F8BA3369536953695830FB3
:10BA20008CA381E080937E298CA18EA31D8E1C8E19
:10BA30008DA1282F30E0C9018F709070843091055E
:10BA400009F4EFC1853091055CF48230910591F1E4
:10BA5000833091050CF0CAC0019709F0C3C210C031
:10BA60008630910509F425C2863091050CF4FDC19C
:10BA70008730910509F425C2089709F0B3C2C6C101
:10BA800080917E2980FFAEC283E08DA380E4809305
:10BA90007E291D8E1C8E20916429309165292115E7
:10BAA000310509F431C182E480937E29C9010E94E5
:10BAB00098562AC180917E2980FF8DC08091E82010
:10BAC000E82FF0E0E55FF54D85858F73823109F051
:10BAD00082C0848590E0807F9070813591050CF460
:10BAE0004EC01092EA2035C0F901ED51F64D84ADFB
:10BAF0008093F120882309F442C0813021F44F5F04
:10BB00004093EA2026C08230C1F485AD8430A9F488
:10BB100036AD20E087AD90E0822B932B9093F320FD
:10BB20008093F22024E0853C920710F084EC94E0AE
:10BB30009F8F8E8F99A388A322C08091EA20E82F3F
:10BB4000F0E0E05EF54DE081EE23C9F0E80FE09310
:10BB5000EA204091EA20242F30E0E091E820F0E054
:10BB6000E55FF54D848582958F7090E00597880F8D
:10BB7000991F880F991F281739070CF4B5CF83E058
:10BB80008DA3E091E820F0E0E55FF54D84818C8B9A
:10BB9000E091E820F0E0E55FF54D85818D8BE09147
:10BBA000E820F0E0E55FF54D86818E8BE091E8209E
:10BBB000F0E0E55FF54D87818F8B81E090E00E949A
:10BBC000985682E480937E291D8E1C8E10926529E2
:10BBD0001092642999C080E280937E290E94B36FFD
:10BBE000E0918529F091862915A2E9CC8091E82081
:10BBF000E82FF0E0E55FF54D858580FF25C024FD49
:10BC000023C08C8D9D8D892B09F0ECC18091642916
:10BC10009091652901960E94985620917E29822F45
:10BC2000806180937E298091642990916529892B78
:10BC300019F0226120937E290E94B36F81E090E089
:10BC40009D8F8C8F88E082C085FF25C0328920E0DF
:10BC5000838990E0282B392B809183299091842926
:10BC6000820F931F9093842980938329E091E82089
:10BC7000F0E0E55FF54D328920E0838990E0282BE4
:10BC8000392B8091642990916529821B930B9093A5
:10BC900065298093642920916429309165292115B3
:10BCA000310559F08DA184FD08C080917E29826004
:10BCB00080937E29C9010E949856E091E820F0E027
:10BCC000E55FF54D968580E02785820F911D909365
:10BCD000F3208093F22028A139A12817390710F00A
:10BCE000892B21F43093F3202093F2208091F220CD
:10BCF0009091F3209F8F8E8F80917E2990E08370AA
:10BD00009070892B09F46EC11092E62E1092E52EE8
:10BD10000E94B36F80917E29282F85FF0CC010925E
:10BD2000E62E1092E52E1DA2E091E820F0E0E55FFE
:10BD3000F54D84E1CCC084FF12C01092E62E109223
:10BD4000E52E81E090E09D8F8C8F84E08DA31FA273
:10BD5000E091E820F0E0E55FF54D81E1B8C0809129
:10BD6000E52E9091E62E892B01F120FF02C01D8E59
:10BD70001C8E8C8D9D8D0097A1F42E8D3F8D809112
:10BD8000E52E9091E62E2817390720F43093E62E01
:10BD90002093E52E8091E52E9091E62E9D8F8C8F3D
:10BDA00004C09093E62E8093E52E1FA28091662911
:10BDB0009091672990938429809383298091E52E1F
:10BDC0009091E62E892B81F08C8D9D8D009761F0EE
:10BDD000CC969093652980936429E091E820F0E067
:10BDE000E55FF54D88E110C080917E2981FFFAC0A2
:10BDF0008CE390E09093652980936429E091E8209A
:10BE0000F0E0E55FF54D80E1858768C080917E298F
:10BE100080FFE8C01DA280E180937E290E94B36F5D
:10BE2000E1C08091642990916529009711F00E94EA
:10BE30009856E091E820F0E0E55FF54D858590911A
:10BE40007E2980FF0BC090FF06C087E08DA31EA255
:10BE50001D8E1C8E1DC086E08DA31AC090FF22C0CF
:10BE600085E08DA31D8E1C8EBDC0809164299091AC
:10BE70006529009711F00E949856E091E820F0E0C3
:10BE8000E55FF54D858580FF0DC087E08DA31EA27F
:10BE900081E090E00E94985680E180937E290E9484
:10BEA000B36F0FC08091642990916529892B49F463
:10BEB00099C080917E2980FF95C087E08DA31EA246
:10BEC00091C0E091E820F0E0E55FF54D80E18587E5
:10BED0008CE390E09093652980936429E091E820B9
:10BEE000F0E0E55FF54D80E58487E091E820F0E043
:10BEF000E55FF54D8C8980878D8981878E89828762
:10BF00008F898387888D8483898D85838A8D8683B5
:10BF10008B8D878386E08093E9298889998991832D
:10BF200080838A899B8993838283ABEFB9E2FE0188
:10BF300080E101900D928150E1F78BEE99E26BEF79
:10BF400079E20E9411658DA1E091E82084FF06C08E
:10BF5000F0E0E55FF54D1786168607C0F0E0E55F77
:10BF6000F54D84E0868784EC87878091632990E093
:10BF700027E131E0829FF001839FF00D929FF00D49
:10BF80001124EE5CF04D84818093EA29809164292C
:10BF90009091652988979093E72980916429885228
:10BFA0008093E829E091E820F0E08F01055F154DCE
:10BFB000D80153961C92539752961C92F801118AFD
:10BFC000108A0E94D15580959095F801918B808BB5
:10BFD00080E68093E3291092E4291092E6291092DA
:10BFE000E52908C010926529109264291092E82072
:10BFF0001092E72010927E29DF91CF911F910F912F
:10C0000008951F9310916329212F30E087E191E07B
:10C01000289FF001299FF00D389FF00D1124EE5C50
:10C02000F04D8389882341F1109263290BC08BEF77
:10C0300099E20E94AD838823C1F4809163298F5FC8
:10C040008093632980916329823088F328C00E94FD
:10C05000CD7F892B51F4809163298F5F8093632971
:10C0600080916329823098F31DC08091EA29815024
:10C070008093EA29882329F4109265291092642973
:10C0800017C083EE99E2489660E840E050E00E94D5
:10C09000B063892B69F081E00E944D5709C010926E
:10C0A0006329DECF109265291092642910936329C9
:10C0B0001F9108950F931F93CF93DF938C014091AD
:10C0C000EB205091EC204F5F5F4F8DE740305807D9
:10C0D00010F040E050E1342F252F8091F72E909101
:10C0E000F82E8217930779F38091102F9091112FDA
:10C0F0008217930741F34093EB205093EC2010926A
:10C10000EA2020E0A9E1B0E01CC0322F3F5F822F7F
:10C1100090E08A9FF0018B9FF00D9A9FF00D112403
:10C12000E951F14D80899189892B51F42093EA20BE
:10C1300089E1289FD0011124A951B14D49F434C09F
:10C14000232F223010F32093EA20A0E0B0E02CC08F
:10C1500050965C93509751964C93519753967C937D
:10C160006E9352970115110531F480E1ED0119929A
:10C170008A95E9F707C0ED01F80180E10190099285
:10C180008150E1F78091632990E027E131E0829FBF
:10C19000F001839FF00D929FF00D1124EE5CF04DA5
:10C1A000848154968C935497CD01DF91CF911F9148
:10C1B0000F910895CF92DF92EF92FF920F930E941A
:10C1C0003A680E94B18580E009C0E82FF0E0EE0FE8
:10C1D000FF1FE152F64D118210828F5F8230A8F36B
:10C1E00020E04CE250E00DC0822F90E0849FF001EF
:10C1F000859FF00D949FF00D1124E957F64D15A27F
:10C200002F5F223088F380E094E09093EC208093BD
:10C21000EB2020E049E150E00EC0822F90E0849FA7
:10C22000F001859FF00D949FF00D1124E951F14D1F
:10C23000118A108A2F5F223080F32093EA200F9119
:10C24000FF90EF90DF90CF900895CF93DF93DC01C4
:10C250008C918F3F09F066C011968C9111978230B6
:10C2600009F060C012968D919C911397892B09F06B
:10C2700059C014968D919C911597892B09F052C045
:10C2800016968D919C911797892B09F04BC01896A3
:10C290008D919C911997892B09F044C01B968C9124
:10C2A0001B97813009F03EC01C968C911C978F3FE4
:10C2B000C9F51092FE202091632930E040E0CDE1E5
:10C2C000D0E087E191E0289FB001299F700D389F51
:10C2D000700D112423C0842F90E08C9FF0018D9F5E
:10C2E000F00D9C9FF00D1124E60FF71FEE5CF04D52
:10C2F00081A592A58F5F9F4F81F01D969C911D9700
:10C3000086A1981751F417969C91179780A19817BA
:10C3100021F44093FE2081E006C04F5F4830D8F200
:10C320004093FE2080E0DF91CF91089540E020E02F
:10C3300030E0FC01E20FF31F5081FB01E20FF31F1D
:10C34000E0815E1731F4485F2F5F3F4F403889F737
:10C350000AC0E527842F885FE7FD05C04F5F4817B7
:10C3600011F0EE0FF9CF842F089582E39FE2089534
:10C37000E0916329F0E0DF01A150BF4D1C92EE0F68
:10C38000FF1FDF01AB5FBE4D6D917C91EF5FFE4DF6
:10C39000808191810E94CA7B08950E940AB8AA27D1
:10C3A00097FDA095BA2FBC01CD0120E838E046EFFB
:10C3B00057E10E946DB69B01AC012058324C4243BC
:10C3C000544FB901CA0108954F925F926F927F92C4
:10C3D0008F929F92BF92CF92DF92EF92FF920F9334
:10C3E0001F938091632990E032E3C32E3FE2D32E66
:10C3F00027E1422E21E0522E849DF001859DF00D13
:10C40000949DF00D1124EC0DFD1D658176818781D1
:10C4100090850E940EB520E030E040E05FE30E948E
:10C42000C4B50E94E2B43B014C010E940AB8B82E88
:10C430000E940AB8FB2CEE24E80EF91E00E010E082
:10C440008091632990E09C01249DC001259D900D61
:10C45000349D900D1124C80ED91EF6016581768198
:10C46000878190850E940EB50E94E2B49B01AC01C9
:10C47000C801B7010E946DB69B01AC01260D371DA6
:10C48000481D591DB901CA011F910F91FF90EF90EE
:10C49000DF90CF90BF909F908F907F906F905F9034
:10C4A0004F9008951F93CF93DF939C0110916329C0
:10C4B000A12FB0E0FD01E150FF4D8081882309F0FC
:10C4C0004AC02115310591F0C9E0D1E2F90180E1BE
:10C4D000019009928150E1F7FD01EE0FFF1FEF5F20
:10C4E000FE4D89E091E29183808307C0FD01EE0F4C
:10C4F000FF1FEF5FFE4D118210826115710591F0F3
:10C50000C9E1D1E2FB0180E1019009928150E1F79C
:10C51000FD01EE0FFF1FEB5FFE4D89E191E291837C
:10C52000808307C0FD01EE0FFF1FEB5FFE4D118200
:10C530001082A150BF4D81E08C930E940AB86FEF2A
:10C540007FE70E945AB6AC01662757FD6095762FAB
:10C55000812F0E94AF87DF91CF911F910895EF92B5
:10C56000FF920F931F930E94CD617B018C01E0919C
:10C570006329F0E0E450FF4D8081833078F481E05E
:10C58000E81684E2F80684EF080780E0180730F028
:10C59000E12C24E2F22E24EF022F112D80E090E016
:10C5A00060E070E00E94CA7B80916329E82FF0E090
:10C5B000E450FF4D90819F5F9083B801A7010E94D6
:10C5C000EC871F910F91FF90EF9008958091632960
:10C5D000A82FB0E087E191E0A89FF001A99FF00D9E
:10C5E000B89FF00D1124EE5CF04D84898823E1F0B2
:10C5F000A450BF4D8C918823B9F40E94CD61AC0149
:10C60000CB01DA01AC01BD01413084E2580784EF6F
:10C61000680780E0780720F040E054E264EF70E0C3
:10C62000809163290E94EC8708951F9310916329DC
:10C63000E12FF0E0E650FF4D8081882399F40E94BD
:10C640000AB8AA2797FDA095BA2FBC01CD0120E812
:10C6500034E84EE150E00E948FB6AB01BC01812F5F
:10C660000E9429881F9108950E94CD7F892BD1F4C3
:10C67000E0916329F0E0E650FF4D8081843090F432
:10C680000E94E07480916329E82FF0E0E650FF4DAE
:10C6900090819F5F908340E45BE46CE470E00E94D3
:10C6A00029880895809163290E946C87E09163290D
:10C6B000F0E0E650FF4D10820E94736C0895AF9237
:10C6C000BF92CF92DF92EF92FF921F93CF93DF93AF
:10C6D0006C011092FE208091632990E03DE1A32E31
:10C6E000B12C27E131E0829F7001839FF00C929F73
:10C6F000F00C112427C0812F90E08A9D90018B9D22
:10C70000300D9A9D300D11242E0D3F1DF901EE5C68
:10C71000F04DEF01A99681A592A58F5F9F4F79F00B
:10C72000C901855B904DB60140E150E00E94F1BB2C
:10C73000009729F48FEF9FEF9983888307C01F5FCD
:10C740001093FE201091FE201830A8F2DF91CF91B7
:10C750001F91FF90EF90DF90CF90BF90AF90089522
:10C76000AF92BF92CF92DF92EF92FF920F931F93FF
:10C77000CF93DF936C01062F7A011092FE20209157
:10C78000632930E00695069506954DE1A42EB12C5F
:10C7900087E191E0289FE001299FD00D389FD00DBF
:10C7A000112438C0212F30E02A9DF0012B9DF00D7F
:10C7B0003A9DF00D1124EC0FFD1FEE5CF04D81A5AC
:10C7C00092A58F5F9F4F19F184A995A98E159F059A
:10C7D00019F0E114F104D9F42A9DC0012B9D900DAC
:10C7E0003A9D900D11248C0F9D1F855B904DB601D5
:10C7F000402F50E00E94F1BB009749F48DE1189F53
:10C80000900111242C0F3D1F255B304D09C01F5F87
:10C810001093FE201091FE20183020F220E030E02E
:10C82000C901DF91CF911F910F91FF90EF90DF90A1
:10C83000CF90BF90AF9008951F93CF93DF93BC012B
:10C8400010916329E12FF0E0EE0FFF1FEC50FF4D38
:10C850008081918140E150E00E94F1BB0097B9F4E2
:10C86000812F0E947887A0916329B0E0FD01EE0F2F
:10C87000FF1FEC50FF4D208131818FEF9FEFE901C9
:10C88000998B888B11821082A850BF4D1C92DF912A
:10C89000CF911F9108951F93DC0150968D919C912B
:10C8A0005197892B09F510916329E12FF0E0EE0FE4
:10C8B000FF1FEC50FF4D80819181892BA9F4B1833A
:10C8C000A0830E940AB8AA2797FDA095BA2FBC01A1
:10C8D000CD0120E834E84EE150E00E948FB6AB0174
:10C8E000BC01812F0E94BF881F9108951F93CF9391
:10C8F000DF9320916329A22FB0E0FD01EE0FFF1F0F
:10C90000EC50FF4D408151814115510509F485C01E
:10C91000C7E1D1E0AC9FF001AD9FF00DBC9FF00DE1
:10C920001124EE5CF04DA850BF4D9C91808D98175E
:10C9300048F580E090E060E070E00E9401761091A0
:10C940006329212F30E0F901E850FF4D80818F5F8E
:10C9500080832C9FF0012D9FF00D3C9FF00D112442
:10C96000EE5CF04D658576858785908928EE33E00D
:10C9700040E050E00E9427B6AB01BC01812F0E942D
:10C98000BF884BC0822F0E9478872091632930E0B6
:10C99000F901EE0FFF1FEC50FF4DA081B18181E046
:10C9A00090E051969C938E93509711821082F901DA
:10C9B000E850FF4D10821092FE2040E0ADE1B0E063
:10C9C0002C9FB0012D9F700D3C9F700D112421C034
:10C9D000242F2F5F842F90E08A9FF0018B9FF00D12
:10C9E0009A9FF00D1124E60FF71FEE5CF04D81A524
:10C9F00092A5892B69F44093FE208DE1489FC001E8
:10CA00001124860F971F855B904D0E944B6405C0D3
:10CA1000422F4830E8F24093FE20DF91CF911F91E2
:10CA200008955F926F927F928F929F92AF92BF9282
:10CA3000CF92DF92EF92FF920F931F93CF93DF93EA
:10CA4000682E592E7B01FB0180818E3F21F481816C
:10CA5000803821F465C08F3F09F462C081E0809383
:10CA6000FE20CC2400E0EDE18E2E912C77E1A72E64
:10CA700071E0B72E69E0762E4CC08091632990E07A
:10CA80002D2D30E0289DE001299DD00D389DD00D41
:10CA900011248A9DB0018B9D700D9A9D700D1124FB
:10CAA0006C0F7D1FFB01EE5CF04D81A592A50197F7
:10CAB00059F5655B704DC7010E949661182F8C1562
:10CAC00018F160916329862F90E09C012A9DC00196
:10CAD0002B9D900D3A9D900D11248C0F9D1F679DED
:10CAE000B00111246459764D855B904D0E94194622
:10CAF000882341F080916329813021F458E0C52ECC
:10CB0000C10E01C0C12E0D2D8091FE208F5F80933C
:10CB1000FE20D090FE2037E03D1508F0AECF44C097
:10CB20001092FE200DE110E0C7E1D1E049E0F42EC3
:10CB300036C060916329262F30E090E0809FA001ED
:10CB4000819F500D909F500D11242C9FC0012D9F4F
:10CB5000900D3C9F900D1124480F591FFA01EE5C77
:10CB6000F04D818D8E3FB1F4828D803899F46F9DA8
:10CB7000B00111246459764DCA01855B904D0E9425
:10CB80001946882339F080916329813019F4009186
:10CB9000FE200AC08091FE208F5F8093FE2080914E
:10CBA000FE20883030F200E0402F50E020916329D1
:10CBB00030E08DE190E0489FF001499FF00D589FD3
:10CBC000F00D112487E191E0AC01249FC001259F65
:10CBD000900D349F900D1124E80FF91F262D352D4F
:10CBE000C901DC01E55BF04D80E101900D928150BF
:10CBF000E1F7DF91CF911F910F91FF90EF90DF90C0
:10CC0000CF90BF90AF909F908F907F906F905F90EC
:10CC10000895CF93DF93FC01DB0118968C91189750
:10CC2000883039F4EF0128960D9009928150E1F790
:10CC30001BC08630E9F49F01285F3F4FAB0183E0C2
:10CC4000EA010990AE01E90109929E018150C1F704
:10CC50008FEF83878EEF8487EF012D96139683E005
:10CC60000D9009928150E1F7808592E0892714C0E8
:10CC70008230B1F411968C91119787878C918687B9
:10CC800015868EEF84878FEF8387128680916131BE
:10CC90008187809160318D7F8087DF91CF9108956A
:10CCA0008FEF9FEF0E94D8697F928F929F92AF92F1
:10CCB000BF92CF92DF92EF92FF920F931F93CF9389
:10CCC000DF93882E792E69017A010130110519F45C
:10CCD000603409F0C6C01092FE2090906329A92C00
:10CCE000BB2440E0ADE1B0E087E191E0A89EB00157
:10CCF000A99E700DB89E700D1124AEC0C42FD0E057
:10CD0000542F5F5FCA9F9001CB9F300DDA9F300D8B
:10CD10001124260F371FF901EE5CF04D81A592A575
:10CD20008F5F9F4F09F097C04093FE20F901E55BAC
:10CD3000F04D882D972D9C01D90180E10D90019235
:10CD40008150E1F70130110501F58DE190E09C0182
:10CD5000C29FC001C39F900DD29F900D112427E167
:10CD600031E0A901A49E9001A59E300DB49E300D26
:10CD70001124820F931F69E0969EB001112464591B
:10CD8000764D855B904D0E9409668091632990E005
:10CD90002091FE2030E0FDE1AF2EB12C2A9DA001B4
:10CDA0002B9D500D3A9D500D1124C7E1D1E0BC01DF
:10CDB0006C9FC0016D9F900D7C9F900D1124480FBA
:10CDC000591FFA01EE5CF04D12A611A615AB04AB8B
:10CDD000C114D104E104F10411F1CA01835A904D48
:10CDE000B701A6010E943B872091FE2030E0809190
:10CDF000632990E02A9DF0012B9DF00D3A9DF00DE6
:10CE000011249C012C9FC0012D9F900D3C9F900DE3
:10CE10001124E80FF91FEE5CF04D13AA02C081E067
:10CE200083AB8091FE202DE1829FC00111242091CF
:10CE3000632930E047E151E0B901649F9001659FAB
:10CE4000300D749F300D1124820F931F855B904D20
:10CE50000E944B6406C0452F483008F44FCF4093E2
:10CE6000FE20DF91CF911F910F91FF90EF90DF9007
:10CE7000CF90BF90AF909F908F907F900895EF924A
:10CE8000FF920F931F93CF93DF9381E08093FE2057
:10CE90000DE110E0C7E1D1E0EE24EA94FE2C47C09A
:10CEA0008091632990E030E0209FA001219F500DE8
:10CEB000309F500D11249C012C9FC0012D9F900D7F
:10CEC0003C9F900D1124480F591FFA01EE5CF04D64
:10CED00081A592A58F5F9F4F29F183A9813011F120
:10CEE000CA01835A904D0E941287892BD9F0209154
:10CEF000FE2030E08091632990E0209FF001219F87
:10CF0000F00D309FF00D11249C012C9FC0012D9F2E
:10CF1000900D3C9F900D1124E80FF91FEE5CF04D31
:10CF2000F2A6E1A68091FE208F5F8093FE202091E3
:10CF3000FE20283008F4B4CFDF91CF911F910F91DC
:10CF4000FF90EF9008959F92AF92BF92CF92DF92A1
:10CF5000EF92FF920F931F93DF93CF93CDB7DEB77E
:10CF6000E2970FB6F894DEBF0FBECDBF1092FE2041
:10CF70000DE1A02EB12C17E1E12E11E0F12E8E0172
:10CF80000F5F1F4FB2E2CB2EB8E0DB2EADE19A2E41
:10CF90005AC02E2F30E08091632990E02A9DF00145
:10CFA0002B9DF00D3A9DF00D1124AC014E9DC0015A
:10CFB0004F9D900D5E9D900D1124E80FF91FEE5CC2
:10CFC000F04D81A592A55FEF8F3F9507B9F1ADB701
:10CFD000BEB718970FB6F894BEBF0FBEADBFEDB782
:10CFE000FEB7319612961C930E931197D382C2828C
:10CFF00035832483978386830E9495BD2DB73EB7E2
:10D00000285F3F4F0FB6F8943EBF0FBE2DBF609113
:10D01000FE20699DB00111248091632990E0AC014C
:10D020004E9DC0014F9D900D5E9D900D1124680F87
:10D03000791F655B704DC8010E948C8C8091FE2029
:10D040008F5F8093FE20E091FE20E83008F4A1CFAE
:10D05000E2960FB6F894DEBF0FBECDBFCF91DF9141
:10D060001F910F91FF90EF90DF90CF90BF90AF9006
:10D070009F9008955F926F927F928F929F92AF924E
:10D08000BF92CF92DF92EF92FF920F931F93CF93B5
:10D09000DF933B014C01142F522EE601809163294E
:10D0A00090E027E1A22E21E0B22E8A9D60018B9DA7
:10D0B000D00C9A9DD00C112422E33FE2C20ED31E65
:10D0C00080E095E0A0E0B0E0F60180839183A28348
:10D0D000B38380E4848380E395E7A0E0B0E08583B8
:10D0E0009683A783B0870E94E461F6016187728707
:10D0F000838794878091632990E09C012A9DC001D9
:10D100002B9D900D3A9D900D1124FC01EE5CF04D8D
:10D1100028EE33E040E050E0258736874787508B84
:10D1200021E0208F728A618A138A148B558A068BBC
:10D13000278B8D5B9F4CB70146E050E00E9449BCB5
:10D14000F09063296F2D70E020E00DE110E06A9D02
:10D15000A0016B9D500D7A9D500D1124AFEFBFEFD4
:10D1600010C0822F90E0809FF001819FF00D909F72
:10D17000F00D1124E40FF51FEE5CF04DB2A7A1A74E
:10D180002F5F283070F39B0183E0220F331F8A95B5
:10D19000E1F7A901460F571FFA01E459F64D8885BA
:10D1A0008087E0E00BC0F0E0DA01AE0FBF1FA459AA
:10D1B000B64DEC0FFD1F80818C93E92F9E2F9F5F52
:10D1C0008885E81780F3E093FE20C7E1D1E06C9FEB
:10D1D000A0016D9F500D7C9F500D1124DA01AE5CB3
:10D1E000B04DAF5FBE4F9FEF9D9382E08D931D9238
:10D1F0001D921D921D921D921D921D921D921D92B7
:10D2000011E01D939D93F901E60FF71FE459F64DC8
:10D210008085E80FF11D339781918D9381918D93D6
:10D2200080818C93A051B140552009F45AC08EEFF3
:10D2300090E85A969C938E9359975C961C921E92F6
:10D240005B975E961C921E925D9790961C921E9222
:10D250005F9792961C921E92919794961C921E92A2
:10D26000939796961C921E92959798961C921E9252
:10D27000979769E0F69EB00111246459764DCA0172
:10D28000855B904D0E9409668091632990E0FC01C6
:10D29000EC9FC001ED9F900DFC9F900D1124FC01AF
:10D2A000EE5CF04D12A611A623E030E035AB24ABC6
:10D2B00013AB855B904D0E944B640E941563611413
:10D2C00071048104910469F08091632990E08C9F3E
:10D2D000F0018D9FF00D9C9FF00D1124EE5CF04D40
:10D2E000138B8091632940E452E46FE070E00E9468
:10D2F0006688DF91CF911F910F91FF90EF90DF90A3
:10D30000CF90BF90AF909F908F907F906F905F90E5
:10D31000089541E00E94608D0895CF93DF93EC0162
:10D320008881833319F48981833389F020E030E0E8
:10D33000FE01E20FF31FD901A459B64D90818C91E3
:10D34000981799F42F5F3F4F2630310589F78C8568
:10D350009D8586589D4D49F4109263296E5070400A
:10D36000CE010E9640E00E94608DDF91CF9108952E
:10D37000CF93DF9320916329E22FF0E0DF0124E0D7
:10D38000AA0FBB1F2A95E1F7A353B94CEC0180E12A
:10D3900009900D928150E1F784E0EE0FFF1F8A950E
:10D3A000E1F7E353F94C8FEF8787DF91CF91089531
:10D3B000FFCF0F931F93CF93DF93809164299091B8
:10D3C0006529009709F458C18150954008F045C17E
:10D3D0008091FB299091FC29892B59F58091FD2999
:10D3E0009091FE29892B29F58091FF299091002A9F
:10D3F000892BF9F48091012A9091022A892BC9F492
:10D400008091032A9091042A892B99F48091052A0E
:10D410009091062A892B69F48091072A9091082A15
:10D42000892B39F48091092A90910A2A892B09F4D1
:10D4300014C18091FB298F3F09F414C180916329A5
:10D44000813071F48091810390918203892B41F4A2
:10D450008BEF99E20E94AD83882311F41092632927
:10D460008BEF99E20E94AD83882331F08BEF99E234
:10D470000E947B84EC0114C080916329813041F4C7
:10D480008091810390918203892B11F4109263297A
:10D490000E94CD7FFC01009709F4DFC0C081D181DB
:10D4A000209739F08A8D9B8D8530910509F065C0F4
:10D4B0000BC08BEF99E260E070E040E020E030E0EC
:10D4C0000E94E084EC0102C01B8E1A8E88A988237A
:10D4D00029F0109264311092633118AA809163315F
:10D4E00090916431892BA9F427E631E33FA72EA759
:10D4F0004091642950916529409363315093643180
:10D50000E3EEF9E2C901BF010E94FEBB80916429EC
:10D5100088AB8BEE99E260E840E050E00E94B06397
:10D52000892B19F08BEE99E202C080E090E060E078
:10D5300070E0AE010E9401768091632990E027E1BE
:10D5400031E0829FF001839FF00D929FF00D112436
:10D55000EE5CF04D658576858785908928EE33E011
:10D5600040E050E00E9427B6AB01BC01CE0184969A
:10D570000E943B8781E08CA775C0009729F588A998
:10D58000882329F0109264311092633118AA809197
:10D59000633190916431892B09F06EC027E631E345
:10D5A0003FA72EA74091642950916529409363318C
:10D5B00050936431E3EEF9E2C901BF010E94FEBB62
:10D5C0008091642988AB58C0029761F483E090E0B1
:10D5D0009B8F8A8FCE014C9640E45BE46CE470E054
:10D5E0000E943B878091632990E027E131E0829F90
:10D5F000F001839FF00D929FF00D1124EE5CF04D31
:10D60000658576858785908928EE33E040E050E097
:10D610000E9427B6AB01BC01CE0184960E943B87D5
:10D620008E01005F1F4FC8010E948C8648A94423C9
:10D63000A1F0409364291092652923EE39E26EA58A
:10D640007FA5C90150E00E94FEBB10926431109288
:10D65000633118AAC8010E948C8610926529109225
:10D6600064290AC080E090E00E948C8610926529AF
:10D67000109264291092E820DF91CF911F910F91B1
:10D6800008950F931F93DF93CF93CDB7DEB76097C5
:10D690000FB6F894DEBF0FBECDBF8C0164367105A6
:10D6A00020F0FC01108280E035C0FB01E351F94C11
:10D6B0008081882319F4F80110822CC040918F30AA
:10D6C00050919030DE01119620E030E0413051055C
:10D6D00019F4EDE1F0E002C0E0E0F0E0C901880FEC
:10D6E000991FE80FF91FEE59FF4C808191818D93AE
:10D6F0009D932F5F3F4F2730310541F7CB010E94AB
:10D70000B156988B8F87C801BE016F5F7F4F0E9413
:10D710008C8C81E060960FB6F894DEBF0FBECDBF53
:10D72000CF91DF911F910F910895CF92DF92EF92E9
:10D73000FF920F931F93DF93CF9300D0CDB7DEB747
:10D74000109263290BEF19E28FEF92E09093FC297E
:10D750008093FB291092FE291092FD291092002A35
:10D760001092FF291092022A1092012A1092042A84
:10D770001092032A1092062A1092052A1092082A63
:10D780001092072A80E092E090930A2A8093092A57
:10D7900098EEE92E9FEFF92EE00EF11E89E0D701F9
:10D7A00097968C93C8014097B8010E94116510921A
:10D7B000E82080E68093E329F70111821382128228
:10D7C00081E186832FEF278380E1C82ED12CC00E04
:10D7D000D11E82E099E0D60113969C938E93129706
:10D7E00090930C2A80930B2A80E094E315969C93E7
:10D7F0008E93149717961C921E921697085E1F4FD1
:10D8000082E08093132A81E0F801818313821282DF
:10D81000278B158A148A168A8091632990E027E164
:10D8200031E0829FA001839F500D929F500D1124E3
:10D83000FA01EE5CF04D84A995A9892BB1F0D701CE
:10D84000D496FA01E55BF04D80E101900D92815094
:10D85000E1F781E0809363290E944680109263295A
:10D86000FC01B29681A181FD05C01092652910923C
:10D8700064292EC02BE23AE2AF0180E1DA010D907B
:10D88000AD01D9010D929D018150C1F78089F80148
:10D8900082A711A610A681E083A78CE590E0909363
:10D8A00065298093642984E390E09A8389838A813F
:10D8B000D70114968C931497898115968C930E94A6
:10D8C000D55580959095F601978386830E94D969F6
:10D8D0000F900F90CF91DF911F910F91FF90EF90DC
:10D8E000DF90CF9008950F931F930E94CD7F892BD7
:10D8F00059F580916329E82FF0E034E0EE0FFF1F27
:10D900003A95E1F7E353F94C87858823E9F01786C8
:10D91000CF0160E420E030E040E050E001E00E9410
:10D92000E4818091632990E024E0880F991F2A9573
:10D93000E1F78353994C60E420E030E040E050E0B0
:10D9400001E010E00E9454668091632990E007E1B5
:10D9500011E0809FF001819FF00D909FF00D112448
:10D96000EE5CF04D83898823A1F00E94CD7F892B46
:10D9700071F08091632990E0809FF001819FF00D0C
:10D98000909FF00D1124EE5CF04D128A118A0E94D6
:10D99000E6620E94A3671F910F9108958091632909
:10D9A000813071F480918F30909190308F5F9F4FD4
:10D9B00009F18FE790E30E94B0460E94590508954F
:10D9C00080915C308823B1F480918F3090919030B9
:10D9D0008F5F9F4F79F48091782F9091792F8F5F8F
:10D9E0009F4F41F08091472F882321F088E69FE2E6
:10D9F0000E94B04608958091AC29882359F087E8A9
:10DA000099E2909386298093852982E00E944D5760
:10DA10000E94D9698091D829882359F083EB99E233
:10DA2000909386298093852982E00E944D570E9419
:10DA3000D96908950F931F93DF93CF93CDB7DEB7C6
:10DA400069970FB6F894DEBF0FBECDBF8C01E62FED
:10DA5000623708F03DC080918F30909190300197EF
:10DA6000B9F58091653190916631892B89F5809166
:10DA70002921882369F5609365311092663129E682
:10DA800036E3C901BA014E2F50E00E94FEBB81E08F
:10DA90008093632980EF93EB9A8B898B9C8B8B8B84
:10DAA00080E48D8BDE011196EFE7F0E380E10190D9
:10DAB0000D928150E1F71F87088BCE01019690935C
:10DAC00082298093812985E00E944D570E94D9695F
:10DAD00069960FB6F894DEBF0FBECDBFCF91DF9130
:10DAE0001F910F91089580917E29883081F5E091F2
:10DAF0006531F0916631309709F44FC029E636E37D
:10DB00008091662990916729B901AF010E94FEBBFF
:10DB10008091653190916631E0916629F091672995
:10DB2000E80FF91F2DE020830196E0916629F0911E
:10DB30006729E80FF91F2AE0208301969093E62ECB
:10DB40008093E52E109266311092653108958230EF
:10DB500021F581E080932921E0916629F0916729E0
:10DB60008091642990916529E80FF91F108200D0F7
:10DB700000D082E398E0EDB7FEB792838183809175
:10DB8000662990916729948383830E9424BD109213
:10DB900029210F900F900F900F900895CF92DF9250
:10DBA000EF92FF920F931F93CF93DF93D82EC62E41
:10DBB00079018A011092E820ACE2B1E2EBEFF9E2E0
:10DBC00080E101900D928150E1F78091642990915C
:10DBD0006529C0969093652980936429815095406A
:10DBE00030F080E095E0909365298093642963EE9E
:10DBF00079E2409164295091652940535040CB010E
:10DC0000C0960E9407BC80E68093E3291092E42925
:10DC10001092E6291092E5298AE38093E929809100
:10DC2000632990E027E131E0829FF001839FF00DAE
:10DC3000929FF00D1124EE5CF04D84818093EA29CF
:10DC40008091EB299091EC29892B51F58091ED2958
:10DC50009091EE29892B21F58091EF299091F0295F
:10DC6000892BF1F48091F1299091F229892BC1F44B
:10DC70008091F3299091F429892B91F48091F529D1
:10DC80009091F629892B61F48091F7299091F829D8
:10DC9000892B31F48091F9299091FA29892BD1F0BF
:10DCA000EBEFF9E2DF01509780E10D900192815096
:10DCB000E1F780912C218F3F91F484E0D81651F444
:10DCC00022E0C21639F48BEE99E26CE271E20E9416
:10DCD00011650EC0109265291092642935C0ABEE13
:10DCE000B9E2ECE2F1E280E101900D928150E1F7BE
:10DCF000E091E820CE2FD0E0FE01E55FF54DD08227
:10DD0000C182C801B7010E94B556C15FD54D688375
:10DD100079838A839B838091642990916529889770
:10DD20009093E729889688528093E8298091E8208B
:10DD3000C82FD0E0C55FD54D1B821A820E94CD55F9
:10DD4000809590959B838A83DF91CF911F910F914E
:10DD5000FF90EF90DF90CF90089543EE59E28091CD
:10DD6000632990E027E131E0829FF001839FF00D6D
:10DD7000929FF00D1124EE5CF04D84818093EA298E
:10DD80008091FB298F3F81F4DA015896FA01389689
:10DD900080E101900D928150E1F78BEE99E26BEFFB
:10DDA00079E20E9411651BC0ACE2B1E2FA0138963B
:10DDB00080E101900D928150E1F7EBEEF9E2DF0195
:10DDC000509680E10D9001928150E1F7ABEFB9E2FE
:10DDD000ECE2F1E280E101900D928150E1F7609177
:10DDE000E820662301F18AE38093E92970E04091FD
:10DDF000642950916529461B570B50936529409320
:10DE00006429485250405093E729485D5F4F842F62
:10DE100088528093E829615F754D4C5250408FE0E5
:10DE20009AE20E9407BC1092E82081E880930B2AB6
:10DE300010920C2A10920E2A10920D2A0E94CD5593
:10DE40008095909590930E2A80930D2A08950F93B4
:10DE50001F93CF93DF9320E62093E3291092E429C8
:10DE60001092E6291092E5292AE32093E9292091CE
:10DE7000632930E047E151E0249FF001259FF00D38
:10DE8000349FF00D1124EE5CF04D24812093EA299B
:10DE9000ABEFB9E2FC0180E101900D928150E1F716
:10DEA0008BEE99E26BEF79E20E9411658AE3809331
:10DEB000E92980E390E0909365298093642980911B
:10DEC0002A2190912B21019690932B2180932A2136
:10DED0002091E820C22FD0E0C15FD54D1982188271
:10DEE0000E94B1569B838A838091E820482F50E09E
:10DEF0002091642930916529FA01E15FF54D81E6B1
:10DF0000848331968F5F8138D9F7C90180969093C9
:10DF1000652980936429285030403093E72988523E
:10DF20008093E8298A01055F154D80E8F801808318
:10DF30001182138212820E94CD5580959095F8012E
:10DF40009383828380912A2190912B21DF91CF911D
:10DF50001F910F910895FC0171A760A70895FC011E
:10DF6000768B658B0895A0918529B09186291097AD
:10DF700019F0FD01B89605C0E0918129F091822940
:10DF8000759680917E2986FF22C050962D913C91F6
:10DF9000519780913E2190913F218217930731F450
:10DFA0008091402190914121009769F48091422114
:10DFB000909143218217930751F4809144219091CD
:10DFC0004521009721F09183808313821282208162
:10DFD00031812115310521F082819381F901099563
:10DFE0000895009749F0909386298093852983E0CE
:10DFF0000E944D570E94D9690895009749F0909367
:10E0000082298093812985E00E944D570E94D96919
:10E010000895CF93DF93EC018091402190914121AD
:10E020008C179D0771F480913E2190913F210E94B1
:10E030005F5610923F2110923E2110924121109282
:10E04000402180914421909145218C179D0771F4C6
:10E0500080914221909143210E945F56109243216A
:10E06000109242211092452110924421ECEAF9E2EB
:10E07000838194818C179D0719F414821382108276
:10E08000BC96CF0185978F5D994290F3E7EEFEE253
:10E09000858996898C179D0711F4118A108A7996C3
:10E0A0008FE2E931F807A0F3DF91CF910895AC0139
:10E0B00010923D21EEE3F1E220E014C080819181D5
:10E0C0008417950769F4828193818617970741F435
:10E0D00020933D2111821082CA010E945F5608954B
:10E0E00034962F5F223050F320933D210895CF9333
:10E0F000DF93EA010E945A60FC01009711F0D68B71
:10E10000C58BCF01DF91CF910895EF92FF920F93CE
:10E110001F93DF93CF93CDB7DEB760970FB6F89418
:10E12000DEBF0FBECDBF8C017B018FEF92E09A83E3
:10E1300089831C821B821E821D8218861F821A867A
:10E1400019861C861B861E861D8680E091E0988BB2
:10E150008F87CE010196B8010E945A60FC0100979A
:10E1600021F0F68AE58A118B008BCF0160960FB6FD
:10E17000F894DEBF0FBECDBFCF91DF911F910F91FD
:10E18000FF90EF900895AC0110923C21EEE3F1E294
:10E1900020E012C0322F3F5F80819181892B51F4A2
:10E1A00020933C215183408373836283CA010E9480
:10E1B0007C5608953496232F223060F320933C211F
:10E1C00008950F931F93CF93DF938A010E94D9552F
:10E1D000EC01009721F019A708A70E94F16FCE016A
:10E1E000DF91CF911F910F9108959F92AF92BF92AF
:10E1F000CF92DF92EF92FF920F931F93CF93DF9313
:10E200008091632990E027E131E0829FE001839FC4
:10E21000D00D929FD00D1124CE5CD04D8F898823D4
:10E2200009F4C2C38091EA298F3F09F0B3C38091FA
:10E23000EB298E3F09F0AEC38091EC29803809F0BC
:10E24000A9C38091E820A82FB0E0FD01E55FF54D5E
:10E250008181882309F09EC3A15FB54D8C91811106
:10E260008C83E091E820F0E0E15FF54D2481358179
:10E2700046815781211531054105510509F448C0F2
:10E280008091632990E0C7E1D1E08C9FF0018D9FE0
:10E29000F00D9C9FF00D1124EE5CF04DE580F680B2
:10E2A00007811085CA01B9010E94B556E616F70626
:10E2B0000807190769F10091632910E0E091E8204F
:10E2C000F0E0E15FF54D64817581868197810E9460
:10E2D000B5560C9FF0010D9FF00D1C9FF00D112401
:10E2E000EE5CF04D65837683878390870091632988
:10E2F00010E00E94E4610C9FF0010D9FF00D1C9F47
:10E30000F00D1124EE5CF04D61877287838794874E
:10E31000E091E820F0E0E15FF54D60857185828550
:10E3200093856115710581059105A1F0009163291F
:10E3300010E00E94B55627E131E0029FF001039FF3
:10E34000F00D129FF00D1124EE5CF04D658776877D
:10E350008787908B10924A211092492110924C216C
:10E3600010924B2140E009C0E42FF0E0EE0FFF1FB8
:10E37000E35BFE4D118210824F5F4430A8F340935F
:10E380005D218CE08093482160916429709165291A
:10E390003AC0F901ED51F64D8181882309F4F8C2A4
:10E3A0008081833071F0853039F08130E1F4F09371
:10E3B0004A21E093492117C0F0934C21E0934B216F
:10E3C00012C040E0443079F0542F5F5FE42FF0E05A
:10E3D000EE0FFF1FE35BFE4D80819181892B09F4D5
:10E3E000DEC2452FEFCF80914821E091E820F0E098
:10E3F000ED51F64DE80FF11D95A5990F990F990F65
:10E40000980F909348219091E82080914821282FDF
:10E4100030E0290F311D245D3F4F2617370708F4E0
:10E42000B8CF40935D21E0914B21F0914C21309782
:10E43000C1F00091632910E0648175818681978124
:10E440000E94B55627E131E0029FF001039FF00DD5
:10E45000129FF00D1124EE5CF04D60837183828376
:10E46000938310925D219924939480C16481758176
:10E47000868197810E94B5567B018C01E0915D21D8
:10E48000F0E0EE0FFF1FE35BFE4D0190F081E02D09
:10E4900060857185828593850E94B556E616F706DC
:10E4A0000807190708F45DC1E0915D21F0E0EE0F67
:10E4B000FF1FE35BFE4D0190F081E02D80898E3FD0
:10E4C00021F48189803809F44CC1838187FF7CC0A5
:10E4D000CF0140960E944483EC0190935821809391
:10E4E0005721E0915D210097C1F5F0E0EE0FFF1F8D
:10E4F000E35BFE4D0190F081E02D648175818681A2
:10E500009781611571058105910509F45DC0EF01E1
:10E5100060966F3F2FEF72072FEF82072FEF920762
:10E5200071F012810E94B55620E432E44FE050E0D1
:10E530000E9427B69B01AC01CE01612F06C0CE011F
:10E54000628120E030E040E050E000E00E94E481A1
:10E55000909358218093572137C0F0E0EE0FFF1FB2
:10E56000E35BFE4D0190F081E02D64817581868131
:10E570009781611571058105910549F06F3FEFEFB6
:10E580007E07EFEF8E07EFEF9E0749F404C0CE0140
:10E590000E94418019C089A1816089A315C00E9491
:10E5A000B55620E432E44FE050E00E9427B6AB01BC
:10E5B000BC01CE0141960E943B87E0915721F0912A
:10E5C000582181A18E7F81A3E0915D21F0E0EE0FC3
:10E5D000FF1FE35BFE4D0190F081E02D838186FFFC
:10E5E000C0C084819581A681B7810097A105B1053E
:10E5F00009F4B7C0CF014096628141E050E00E942B
:10E60000B063DC0190935C2180935B21E0915D21FC
:10E61000009709F478C0F0E0EE0FFF1FE35BFE4DBA
:10E620000190F081E02D64817581868197816F3F33
:10E63000FFEF7F07FFEF8F07FFEF9F0709F460C031
:10E640000E94B55661527C418040904040F5E09177
:10E650005D21F0E0EE0FFF1FE35BFE4D0190F081C6
:10E66000E02D64817581868197810E94B5567B017A
:10E670008C0180915B2190915C2142960E94ED86F5
:10E680005B016C01C801B70120E432E44FE050E0C7
:10E690000E9427B6A616B706C806D90600F500914F
:10E6A0005B2110915C210E5E1F4FE0915D21F0E037
:10E6B000EE0FFF1FE35BFE4D0190F081E02D6481C2
:10E6C0007581868197810E94B55620E432E44FE03F
:10E6D00050E00E9427B6AB01BC01C80109C080917F
:10E6E0005B2190915C21429640E058E467E27DEA2C
:10E6F0000E943B87E0915B21F0915C21128E31C03A
:10E700005A969C922EC0F0E0EE0FFF1FE35BFE4D89
:10E710000190F081E02D6481758186819781EF0100
:10E7200060966F3F2FEF72072FEF82072FEF920750
:10E7300071F012810E94B55620E432E44FE050E0BF
:10E740000E9427B69B01AC01CE01612F06C0CE010D
:10E75000628120E030E040E050E001E010E00E9403
:10E76000546680915D218F5F80935D21E0915D21F2
:10E77000E43058F4F0E0EE0FFF1FE35BFE4D019034
:10E78000F081E02D309709F071CE8BEE99E20E9476
:10E790007B84FC01909356218093552160914921FF
:10E7A00070914A216115710509F461C0009771F4F7
:10E7B0006E5F7F4F8BEE99E241E022E030E00E94F5
:10E7C000E084909356218093552151C0828D938D82
:10E7D000892B21F482E090E0938F828F209163292E
:10E7E000822F90E0FC0133E0EE0FFF1F3A95E1F736
:10E7F000E80FF91FE459F64DA084213061F4E0914F
:10E800004921F0914A218181813019F098E0A92EA7
:10E8100002C082E0A82E0091492110914A210E5F8A
:10E820001F4FE0905521F0905621E7016096C801F6
:10E83000BE014A2D50E00E94F1BB009721F4F70180
:10E84000808DA81671F0CE01B8014A2D50E00E94CB
:10E85000FEBBE0915521F091562182E090E0938F2C
:10E86000828FE0915521F091562181E0818FE091D6
:10E87000E820F0E0E15FF54D82819381E091552140
:10E88000F0915621892B09F454C0309771F48BEE26
:10E8900099E260E070E041E025E030E00E94E08431
:10E8A000909356218093552102C081E0818F809101
:10E8B0005521909156210E947F7F8C0190935A217F
:10E8C00080935921E091E8200097D9F400915521D7
:10E8D00010915621F0E0E15FF54D828193810E9415
:10E8E000B156A0E0B0E0BC01CD0120E432E44FE03D
:10E8F00050E00E9427B6AB01BC01C8010E94BC8257
:10E9000025C0F0E0E15FF54D828193810E94B15610
:10E91000A0E0B0E0BC01CD0120E432E44FE050E0E3
:10E920000E9427B6AB01BC01C80102960E943B873A
:10E930000DC0309759F0CF010E947F7F90935A21EC
:10E9400080935921009711F00E943680E091552163
:10E95000F09156213097C9F040A94423B1F040937B
:10E9600064291092652923EE39E266A577A5C901CD
:10E9700050E00E94FEBB1092643110926331E0912E
:10E980005521F091562110AA0FC00E94CE6C02C0F2
:10E9900040935D21109265291092642905C02D5184
:10E9A000364D318320831FCDDF91CF911F910F9181
:10E9B000FF90EF90DF90CF90BF90AF909F90089521
:10E9C000EF92FF920F931F93DF93CF9300D0CDB7B9
:10E9D000DEB780916329282F30E087E191E0289FFE
:10E9E000F001299FF00D389FF00D1124EE5CF04DE1
:10E9F0008789882309F4FCC0F90183E0EE0FFF1F2B
:10EA00008A95E1F7E20FF31FE459F64D2085822F36
:10EA100090E00296022F0E5F87709070081B892B82
:10EA200009F0085F83EE99E220E62093E329109233
:10EA3000E4291092E6291092E5292AE32093E92996
:10EA40002FEF2093EA29FC0178962FEF32E03093E4
:10EA5000FC292093FB2913821282158214821782CB
:10EA6000168211861086138612861586148620E07B
:10EA700032E0378726870896BF010E9411652091F2
:10EA8000E820A22FB0E0FD01E55FF54D85E8808329
:10EA90001182FD01E15FF54D108211821282138215
:10EAA0001092E7298091EB299091EC29892B99F517
:10EAB0008091ED299091EE29892B69F58091EF29BC
:10EAC0009091F029892B39F58091F1299091F229C3
:10EAD000892B09F58091F3299091F429892BD9F498
:10EAE0008091F5299091F629892BA9F48091F72935
:10EAF0009091F829892B79F48091F9299091FA293C
:10EB0000892B49F488E08093E829D096B093652951
:10EB1000A09364295DC0E02EFF24822F90E0C09670
:10EB20008E0D9F1D9093652980936429085F009343
:10EB3000E8290850AD5EB54DB0934A21A093492114
:10EB400081E08C9306950695069511960C93119786
:10EB5000209163291296822F90E0FC0103E0EE0FD2
:10EB6000FF1F0A95E1F7E80FF91FE459F64D4085BC
:10EB700089E0289F900111242459364DCD01B90117
:10EB800050E00E94FEBB8091632990E0FC0113E0FD
:10EB9000EE0FFF1F1A95E1F7E80FF91FE459F64D44
:10EBA000808590E09701281B390B225030403A8332
:10EBB00029832091492130914A212E5F3F4F280F10
:10EBC000391FC90160E070E049815A810E9419BC77
:10EBD0008091E820082F10E0055F154DF8011382A1
:10EBE00012820E94CD5580959095F801938382837F
:10EBF0000F900F90CF91DF911F910F91FF90EF90A9
:10EC00000895FF920F931F93CF93DF938C01EA0136
:10EC100080916329282F30E087E191E0289FF0015F
:10EC2000299FF00D389FF00D1124EE5CF04D87897F
:10EC3000882309F413C1F90153E0EE0FFF1F5A9521
:10EC4000E1F7E20FF31FE459F64D2085822F90E0A3
:10EC5000029642E0F42EF20E87709070F81A892B1B
:10EC600011F088E0F80E1092E82080E68093E32906
:10EC70001092E4291092E6291092E5298AE3809304
:10EC8000E9299FEF9093EA29EBEFF9E2611571050D
:10EC9000B9F49093FB2982E081831382128215825A
:10ECA00014821782168211861086128681E083876D
:10ECB00094878D8585878E859F859787868707C0F2
:10ECC000DF01FB0180E101900D928150E1F787E8BF
:10ECD00080930B2A10920C2A10920F2A1092102A5D
:10ECE0001092112A1092122AA3E1BAE2FE0180E1E9
:10ECF00001900D928150E1F71092E729CE0160E872
:10ED000040E050E00E94B063892B09F070C001150B
:10ED1000110549F0ABEEB9E2F80180E101900D92E6
:10ED20008150E1F706C08BEE99E26BEF79E20E9429
:10ED3000116588E1F80EF092E82988EEF80E0F2DA3
:10ED400010E0005C1F4F1093652900936429005464
:10ED50001040A091E820B0E0AD5DB54DB0934A21E0
:10ED6000A093492181E08C93F694F694F694119641
:10ED7000FC921197209163291296822F90E0FC015A
:10ED800033E0EE0FFF1F3A95E1F7E80FF91FE45962
:10ED9000F64D408589E0289F900111242459364D75
:10EDA000CD01B90150E00E94FEBB8091632990E043
:10EDB000FC0123E0EE0FFF1F2A95E1F7E80FF91F92
:10EDC000E459F64D808590E0081B190B0250104065
:10EDD0002091492130914A212E5F3F4F280F391F42
:10EDE000C90160E070E0A8010E9419BC29C010921E
:10EDF000EC291092EB291092EE291092ED29109235
:10EE0000F0291092EF291092F2291092F129109214
:10EE1000F4291092F3291092F6291092F5291092F4
:10EE2000F8291092F7291092FA291092F92988E10D
:10EE30008093E82980E490E0909365298093642989
:10EE40008091E820C82FD0E0C55FD54D1B821A8283
:10EE50000E94CD55809590959B838A83DF91CF91B9
:10EE60001F910F91FF900895BF92CF92DF92EF9282
:10EE7000FF920F931F93DF93CF93CDB7DEB72B97FE
:10EE80000FB6F894DEBF0FBECDBF8091632990E02E
:10EE900027E131E0829FF001839FF00D929FF00DFA
:10EEA0001124EE5CF04D8789882309F4B1C190915B
:10EEB000E820E92FF0E0DF01A15FB54DDC90809103
:10EEC000EA298F3F09F0A0C1E55FF54D81818823D4
:10EED00009F09AC114968C9114978F3F09F494C14C
:10EEE000E0E4BE2EBD20D6FE05C08091FB298F3FF9
:10EEF00009F48AC184E18093482110924A2110923A
:10EF000049216091642970916529292F30E0245DA1
:10EF10003F4FA9014D51564D1AC0FC01ED51F64D20
:10EF20008181882309F470C18081823021F4F093BB
:10EF30004A21E093492180914821FA01E80FF11D0F
:10EF40009181990F990F990F980F90934821809173
:10EF50004821F901E80FF11DCF01E617F707E8F2A4
:10EF6000CD01049660E840E050E00E94B063FC01EF
:10EF700090935C2180935B21009769F0808991894F
:10EF8000892B09F041C18091E82090E08D5E954D7C
:10EF90000E941C6439C18091E82090E08D5E954DFF
:10EFA0000E947B849093562180935521892B09F4EC
:10EFB0002BC120916329822F90E0FC0173E0EE0FBA
:10EFC000FF1F7A95E1F7E80FF91FE459F64D008528
:10EFD000213051F4E0914921F0914A218181813021
:10EFE00011F008E001C002E02091492130914A214E
:10EFF0002E5F3F4FCE010196B901402F50E00E9495
:10F00000FEBB0987E0904921F0904A21E114F10408
:10F0100011F410E018C080915521909156219B87E2
:10F020008A87BC01605F7F4FC7010296402F50E086
:10F030000E94F1BB982FEA85FB85808D081711F09F
:10F0400011E001C0192F60E8C62ECD20E0915521B6
:10F05000F0915621828D938D009709F045C0E114FF
:10F06000F10409F4D1C09F01205F3F4FA7014E5F1B
:10F070005F4FC901BA01402F50E00E94FEBBE091F2
:10F080005521F0915621008FE0905521F0905621A6
:10F09000BB2021F181E090E0F701938F828F809176
:10F0A000632990E027E131E0829FF001839FF00D1A
:10F0B000929FF00D1124EE5CF04D61857285838581
:10F0C000948528EE33E040E050E00E9427B6AB0183
:10F0D000BC01C7014C960E943B8774C082E090E05F
:10F0E000F701938F828F6EC0D5FC0AC0112341F0C7
:10F0F000019709F089C082E090E0938F828F84C0ED
:10F10000E114F10489F09F01205F3F4FA7014E5F9A
:10F110005F4FC901BA01402F50E00E94FEBBE09151
:10F120005521F0915621008FBB2041F1E0905521EF
:10F13000F090562181E090E0F701938F828F8091CB
:10F14000632990E027E131E0829FF001839FF00D79
:10F15000929FF00D1124EE5CF04D618572858385E0
:10F16000948528EE33E040E050E00E9427B6AB01E2
:10F17000BC01C7014C960E943B8710C08091492179
:10F1800090914A21892B51F0112341F0E0915521B2
:10F19000F091562182E090E0938F828FE09155218B
:10F1A000F0915621818D882369F0CC2059F4CF014C
:10F1B0000E947F7F90935A2180935921009711F0EC
:10F1C0000E943680E0915521F0915621C18EE09148
:10F1D0005521F091562140A94423B1F04093642970
:10F1E0001092652923EE39E266A577A5C90150E0A2
:10F1F0000E94FEBB1092643110926331E091552160
:10F20000F091562110AA04C0109265291092642929
:10F210002B960FB6F894DEBF0FBECDBFCF91DF9116
:10F220001F910F91FF90EF90DF90CF90BF900895C6
:10F23000BF92CF92DF92EF92FF920F931F93DF93D3
:10F24000CF93CDB7DEB729970FB6F894DEBF0FBEC8
:10F25000CDBF50916329652F70E087E191E0689FF1
:10F26000F001699FF00D789FF00D1124EE5CF04DD8
:10F270008789882309F47EC28091EA298F3F09F0AB
:10F2800075C28091E820282F30E0F901E15FF54D4B
:10F2900084818F3F09F46AC2F901E55FF54D8181F0
:10F2A000882309F063C210924A211092492184E117
:10F2B00080934821009164291091652944E1F90166
:10F2C000BC9616C0DC01AD51B64D11968C911197CC
:10F2D000882309F449C28C91813021F4B0934A21EA
:10F2E000A093492111968C91880F880F880F480FA1
:10F2F000CF01840F911D8017910720F3409348217F
:10F30000A0914921B0914A21109709F499C08091A8
:10F31000EB299091EC29892B59F58091ED29909159
:10F32000EE29892B29F58091EF299091F029892BDD
:10F33000F9F48091F1299091F229892BC9F48091F7
:10F34000F3299091F429892B99F48091F5299091D2
:10F35000F629892B69F48091F7299091F829892B56
:10F3600039F48091F9299091FA29892B09F4FEC189
:10F37000FB0113E0EE0FFF1F1A95E1F7E60FF71FF1
:10F38000E459F64DB084513051F411968C91119797
:10F39000813019F078E0B72E02C062E0B62E9D01F0
:10F3A0002E5F3F4F8E010F5F1F4FC801B9014B2DDC
:10F3B00050E00E94FEBBB9868BEE99E20E947B84EE
:10F3C0007C019093562180935521009749F48BEE50
:10F3D00099E2B80140E022E030E00E94E08430C0D1
:10F3E0000091492110914A210E5F1F4F50E1C52E17
:10F3F000D12CC80ED91EC801B6014B2D50E00E9479
:10F40000F1BB009721F4F701808DB81681F0C60199
:10F41000B8014B2D50E00E94FEBBE0915521F091C8
:10F420005621B08EE0915521F091562105C0F7018B
:10F43000828D938D892B21F482E090E0938F828FCF
:10F440008091E82090E08D5E954D60E840E050E0CE
:10F450000E94B06390935C2180935B21892B09F417
:10F4600085C18091EB299091EC29892B09F074C01A
:10F470008091ED299091EE29892B09F06DC0809142
:10F48000EF299091F029892B09F066C08091F1292C
:10F490009091F229892B09F05FC08091F329909116
:10F4A000F429892B09F058C08091F5299091F6290B
:10F4B000892B09F051C08091F7299091F829892B67
:10F4C00009F04AC08091F9299091FA29892B09F015
:10F4D00043C08BEF99E20E942561882309F446C15D
:10F4E000E0915B21F0915C2180899189892B61F108
:10F4F0008FEF92E09093FC298093FB291092FE29D4
:10F500001092FD291092002A1092FF291092022ACF
:10F510001092012A1092042A1092032A1092062AAD
:10F520001092052A1092082A1092072A80E091E092
:10F5300090930A2A8093092A8BEE99E26BEF79E285
:10F540000E94116550E255C08091E82090E08D5EE8
:10F55000954D0E941C640AC18BEE99E260E840E080
:10F5600050E00E94B063892B09F000C18BEF99E253
:10F570000E9425618823B9F0EBEFF9E2DF01509793
:10F5800080E10D9001928150E1F78091E820E82F11
:10F59000F0E0ABEEB9E2ED5EF54D80E101900D9249
:10F5A0008150E1F725C08BEF99E260E840E050E040
:10F5B0000E94B06320915B2130915C2128173907AC
:10F5C00009F0D4C0EBEFF9E2DF01509780E10D9034
:10F5D00001928150E1F78091E820E82FF0E0ABEE56
:10F5E000B9E2ED5EF54D80E101900D928150E1F7B9
:10F5F00050E61092E82080916329282F30E087E1BF
:10F6000091E0289FF001299FF00D389FF00D112403
:10F61000EE5CF04D838981115068F90143E0EE0FF3
:10F62000FF1F4A95E1F7E20FF31FE459F64D2085DD
:10F63000822F90E00296422F4E5F87709070481B99
:10F64000892B09F0485F80E68093E3291092E42932
:10F650001092E6291092E5291092E729485E40931E
:10F66000E82948518AE38093E9298FEF8093EA29BA
:10F6700088E880930B2A10920C2A50930F2AA3E15A
:10F68000BAE220915B2130915C21C901FC0180E14B
:10F6900001900D928150E1F7042F10E0005C1F4FA4
:10F6A000109365290093642900541040A091E8202C
:10F6B000B0E0AD5DB54DB0934A21A093492182E001
:10F6C0008C9346954695469511964C9311972091AB
:10F6D00063291296822F90E0FC0133E0EE0FFF1FAA
:10F6E0003A95E1F7E80FF91FE459F64D408589E0B6
:10F6F000289F900111242459364DCD01B90150E0C5
:10F700000E94FEBB8091632990E0FC01A3E0EE0F14
:10F71000FF1FAA95E1F7E80FF91FE459F64D808520
:10F7200090E0081B190B02501040209149213091A4
:10F730004A212E5F3F4F280F391FC90160E070E05A
:10F74000A8010E9419BC8091E820082F10E0055FF5
:10F75000154DF801138212820E94CD558095909527
:10F76000F8019383828306C0409348211092652953
:10F770001092642929960FB6F894DEBF0FBECDBF54
:10F78000CF91DF911F910F91FF90EF90DF90CF907D
:10F79000BF9008956F927F928F929F92AF92BF9287
:10F7A000CF92DF92EF92FF920F931F93DF93CF934D
:10F7B00000D0CDB7DEB7AC0180916329282F30E0AF
:10F7C00087E191E0289FF001299FF00D389FF00D0F
:10F7D0001124EE5CF04D8789882309F420C2F901D9
:10F7E000A3E0EE0FFF1FAA95E1F7E20FF31FE45924
:10F7F000F64D2085822F90E00296E2E0DE2ED20EBA
:10F8000087709070D81A892B11F088E0D80E611596
:10F81000710529F58FEF92E09093FC298093FB29E5
:10F820001092FE291092FD291092002A1092FF29B1
:10F830001092022A1092012A1092042A1092032A8E
:10F840001092062A1092052A1092082A1092072A6E
:10F8500080E091E090930A2A8093092A08C0ABEFD8
:10F86000B9E2FB0180E101900D928150E1F7411571
:10F87000510549F0ABEEB9E2FA0180E101900D9239
:10F880008150E1F706C08BEE99E26BEF79E20E94BE
:10F8900011651092E82080E68093E3291092E42914
:10F8A0001092E6291092E5298AE38093E9298FEFE7
:10F8B0008093EA2986E880930B2AE3EEF9E211A609
:10F8C0008091632990E007E111E0809FF001819F22
:10F8D000F00D909FF00D1124EE5CF04D848180932B
:10F8E0000F2A818992890E94B1569093122A80939F
:10F8F000112A8091E820E82EFF24EFE0FAE2EE0ED4
:10F90000FF1E8091632990E0809FF001819FF00DA0
:10F91000909FF00D1124EE5CF04D6581768187811A
:10F9200090850E94B556F70164837583868397831B
:10F930008091E820E82EFF248FE09AE2E80EF91E7D
:10F940008091632990E0809FF001819FF00D909F4E
:10F95000F00D1124EE5CF04D6585768587859089E4
:10F960000E94B556F70160877187828793870D2DB6
:10F9700010E0085C1F4F1093652900936429085319
:10F980001040A091E820B0E0A55EB54DB0934A21AB
:10F99000A093492181E08C938D2D8695869586953F
:10F9A00011968C931197209163291296822F90E0E3
:10F9B000FC0133E0EE0FFF1F3A95E1F7E80FF91F66
:10F9C000E459F64D408589E0289F9001112424597F
:10F9D000364DCD01B90150E00E94FEBB80916329F4
:10F9E00090E0FC0123E0EE0FFF1F2A95E1F7E80FFE
:10F9F000F91FE459F64D808590E0081B190B025061
:10FA000010402091492130914A212E5F3F4F280F0D
:10FA1000391FC90160E070E0A8010E9419BCFCE038
:10FA2000DF0ED09248210E9446807C0110925D2119
:10FA3000B2E29B2EA3E06A2EF0EC7F2EE4E08E2E45
:10FA4000AA24AA94BA2C6501C8C0899DF00111248A
:10FA5000EE0DFF1D81A18670863009F0B9C080814E
:10FA60008E3F21F48181803809F4B2C08091E82072
:10FA7000082F10E0045D1F4F80914821482F50E06F
:10FA8000D801AD51B64DA40FB51F6C9213967C9260
:10FA9000139711968C92119720915D21822F90E0FF
:10FAA000FC0175E0EE0FFF1F7A95E1F7880F991FB3
:10FAB000E80FF91FEE0DFF1D808912968C931297A7
:10FAC000299DF0011124EE0DFF1D81A180FF0DC0C5
:10FAD0001496AD92BD92CD92DC9217971896AD9286
:10FAE000BD92CD92DC921B9743C0040F151F0D51A0
:10FAF000164D658976898789908D20E432E44FE040
:10FB000050E00E946DB6CA01B9010E94B556F801D5
:10FB100064837583868397838091E8209091482140
:10FB2000092F10E0080F111D015F154D80915D2117
:10FB300090E0FC0145E0EE0FFF1F4A95E1F7880FCA
:10FB4000991FE80FF91FEE0DFF1D658D768D878DCE
:10FB500090A120E432E44FE050E00E946DB6CA016B
:10FB6000B9010E94B556F801608771878287938733
:10FB7000E091E820F0E080914821E15FF54DE80F49
:10FB8000F11D148615861686178680915D2190E0FA
:10FB9000DC0125E0AA0FBB1F2A95E1F7880F991F0A
:10FBA000A80FB91F7096AE0DBF1D80E10D90019298
:10FBB0008150E1F780914821805E809348218091B7
:10FBC0006429909165298096909365298093642992
:10FBD00080915D218F5F80935D2180915D218430D4
:10FBE00008F433CF809164299091652988979A838E
:10FBF00089838A818093E72989818093E82980918C
:10FC0000E820082F10E0055F154DF80113821282DD
:10FC10000E94CD5580959095F801938382830F9033
:10FC20000F90CF91DF911F910F91FF90EF90DF9098
:10FC3000CF90BF90AF909F908F907F906F900895DE
:10FC4000BF92CF92DF92EF92FF920F931F93DF93B9
:10FC5000CF93CDB7DEB769970FB6F894DEBF0FBE6E
:10FC6000CDBF50916329052F10E087E191E0089FF7
:10FC7000F001099FF00D189FF00D1124EE5CF04D7E
:10FC80008789882309F4F8C08389882309F4F0C0A0
:10FC90008091EA298F3F09F0EBC08091E820682F1E
:10FCA00070E0FB01E55FF54D8181882309F0E0C03C
:10FCB00010924A211092492184E080934821E090DB
:10FCC0006429F090652920E030E044E0FB01BC9617
:10FCD00011C0DC01AD51B64D11969C91119799233D
:10FCE00009F4C0C08C91813009F49D01990F990FDE
:10FCF000990F490FCF01840F911D8E159F0548F371
:10FD00002093492130934A21409348212115310500
:10FD100009F493C08091EB299091EC29892B59F536
:10FD20008091ED299091EE29892B29F58091EF2979
:10FD30009091F029892BF9F48091F1299091F22981
:10FD4000892BC9F48091F3299091F429892B99F496
:10FD50008091F5299091F629892B69F48091F729F2
:10FD60009091F829892B39F48091F9299091FA29F9
:10FD7000892B09F47DC0F80183E0EE0FFF1F8A95FF
:10FD8000E1F7E00FF11FE459F64DB084513049F42A
:10FD9000F9018181813019F008E0B02E02C012E033
:10FDA000B12E2E5F3F4F8E010F5F1F4FC801B9016B
:10FDB0004B2D50E00E94FEBBB9868BEE99E20E946B
:10FDC0007B847C019093562180935521009749F4C0
:10FDD0008BEE99E2B80140E022E030E00E94E0843E
:10FDE0002CC00091492110914A210E5F1F4FB0E1B4
:10FDF000CB2ED12CC80ED91EC801B6014B2D50E018
:10FE00000E94F1BB009721F4F701808DB81661F0D4
:10FE1000C601B8014B2D50E00E94FEBBE091552178
:10FE2000F0915621B08E05C0F701828D938D892BFC
:10FE300021F482E090E0938F828F109265291092D6
:10FE40006429DE011A96EBEEF9E280E101900D9251
:10FE50008150E1F780E090E0BE01665F7F4F0E9435
:10FE600052620AC030934A2120934921409348218D
:10FE7000109265291092642969960FB6F894DEBF36
:10FE80000FBECDBFCF91DF911F910F91FF90EF90EB
:10FE9000DF90CF90BF9008952091632930E040E03B
:10FEA000ABE0B0E086E190E0289FB001299F700DA3
:10FEB000389F700D11240FC0842F90E08A9FF001AD
:10FEC0008B9FF00D9A9FF00D1124E60FF71FE2595A
:10FED000FB4D12864F5F423078F34093AA25089578
:10FEE00090E028E831E0A901849F9001859F300DC2
:10FEF000949F300D1124225A3E4DC9010895CF938D
:10FF0000DF93DC011092B0251092AF251092AA2544
:10FF100050916329252F30E040E0CBE0D0E086E12E
:10FF200090E0289FB001299F700D389F700D11241B
:10FF300029C0842F90E08C9FF0018D9FF00D9C9F35
:10FF4000F00D1124E60FF71FE259FB4D828588233F
:10FF5000C1F0808191818A179B0799F44093AA256B
:10FF60008BE0489FC001112426E1529F900111248B
:10FF7000820F931F82599B4D9093B0258093AF259C
:10FF800005C04F5F4230A8F24093AA258091AF256B
:10FF90009091B025DF91CF9108950F931F93CF9348
:10FFA000DF931092B0251092AF251092AA25909160
:10FFB0006329292F30E086E1989FD001112440E089
:10FFC00050E060E00BE010E086E190E0289FE00167
:10FFD000299FD00D389FD00D11242BE036C0862FDD
:10FFE00090E0809FF001819FF00D909FF00D112413
:10FFF000EC0FFD1FE259FB4D8285882329F101900A
:020000021000EC
:10000000F081E02D309701F1828D938D009711F0F2
:10001000059759F441155105B9F4629FA0011124C7
:100020004A0F5B1F42595B4D0FC06093AA258BE0BE
:10003000689FC00111248A0F9B1F82599B4D90938A
:10004000B0258093AF2509C06F5F623040F25093B6
:10005000B0254093AF256093AA258091AF2590915C
:10006000B025DF91CF911F910F910895FC01128669
:100070000190F081E02D828D938D059709F415A6EE
:100080000895FC0181A18D7F81A3089520916329AA
:1000900088E8289F9001112426563B4DC9010895F8
:1000A0007F928F929F92AF92BF92CF92DF92EF9208
:1000B000FF920F931F93CF93DF9390916329A92F02
:1000C000B0E086E1989FE001112420E030E040E0BC
:1000D0000BE010E086E190E0A89FB001A99F700DB1
:1000E000B89F700D11245BE018C0842F90E0809FB2
:1000F000F001819FF00D909FF00D1124E60FF71F86
:10010000E259FB4D8285813039F4459F90011124DD
:100110002C0F3D1F22593B4D4F5F423030F330933F
:10012000B0252093AF254093AA251092AE251092BA
:10013000AD2587E191E0A89FF001A99FF00DB89F40
:10014000F00D1124EE5CF04D8789882309F4DCC0A2
:100150001092AA2511E3812E912CB8E8AB2EB1E0C4
:10016000BB2EA1E37A2EF2E0CF2ED12CC7E1D1E055
:10017000E4E0EE2EF12CC3C08091632990E0242F9F
:1001800030E0289DD001299DB00D389DB00D11247F
:100190008A9D90018B9D300D9A9D300D1124A20FE8
:1001A000B31FA25ABE4D9D968C919D97813009F048
:1001B000A1C0479DF0011124E20FF31FE25AFE4D4A
:1001C000F093AE25E093AD25828D938D813091051E
:1001D00001F18130910538F08330910549F10497A0
:1001E00009F088C034C084A5833018F09D961C9215
:1001F00081C0CF0184960E941287892B09F47AC0AE
:100200004091AD255091AE2580E090E060E070E037
:1002100048C0CF014C960E941287892B09F46AC00E
:10022000E091AD25F091AE25D38EC28E14A662C0AA
:10023000CF014C960E941287892B09F45BC0E09194
:10024000AD25F091AE25F38EE28E14A623C084A5D1
:100250008330D0F014A6CF010E947F7FFC019093E1
:10026000B0258093AF25009749F012860190F08168
:10027000E02D828D938D059709F415A6E091AD25AB
:10028000F091AE2515A636C0CF0184960E94128744
:10029000892B81F14091AD255091AE2580E090E011
:1002A000BA010E9401760091AD251091AE25809192
:1002B000632990E08C9FF0018D9FF00D9C9FF00DC5
:1002C0001124EE5CF04D658576858785908928EE52
:1002D00033E040E050E00E9427B6AB01BC01C8010A
:1002E00084960E943B87E091AD25F091AE2584A5D0
:1002F0008F5F84A78091AA258F5F8093AA25409164
:10030000AA25483008F438CF1092AC251092AB25BE
:1003100081E08093AA25C8E8D0E002E218E841C055
:1003200050916329252F30E0842F90E0FC0175E087
:10033000EE0FFF1F7A95E1F7880F991FE80FF91F5D
:100340002C9FC0012D9F900D3C9F900D1124E80F14
:10035000F91FE554FB4D808181FF1EC0409FF001D5
:100360001124519FC0011124E80FF91FE656FB4DDF
:10037000F093AC25E093AB2581A180FD0DC0CF01AA
:1003800041960E941287892B39F0E091AB25F091BC
:10039000AC2581A18D7F81A38091AA258F5F809359
:1003A000AA254091AA25443008F4BACFDF91CF9115
:1003B0001F910F91FF90EF90DF90CF90BF90AF9083
:1003C0009F908F907F900895AF92BF92CF92DF92CF
:1003D000EF92FF920F931F93CF93DF93182FB92EB5
:1003E000A62E69017A011092AC251092AB2581E00E
:1003F0008093AA258091632990E041E028E830E0CD
:10040000829FB001839F700D929F700D112419C0BF
:10041000242F2F5F842F90E0FC0135E0EE0FFF1FAB
:100420003A95E1F7880F991FE80FF91FE60FF71FBC
:10043000E554FB4D808181FD03C04093AA2510C087
:10044000422F443028F34093AA25443049F40E94B7
:100450000AB863E070E00E945AB68F5F8093AA25C5
:100460009091AA2582E2989FF0011124809163293E
:1004700028E8829FC0011124E80FF91FE656FB4DC2
:10048000F093AC25E093AB25EF01212F3B2DC90163
:10049000DC0180E10D9009928150E1F7A08AC1143E
:1004A000D104E104F10469F0CF014196B701A6013E
:1004B0000E943B87E091AB25F091AC2581A18E7F16
:1004C00002C081A1816081A32091632930E0609105
:1004D000AA25862F90E0FC01A5E0EE0FFF1FAA954C
:1004E000E1F7880F991FE80FF91F88E890E0289F2F
:1004F000A001299F500D389F500D1124E40FF51FC6
:10050000E554FB4D80818260808300FF13C0862FFD
:1005100090E0FC0165E0EE0FFF1F6A95E1F7880FA0
:10052000991FE80FF91FE40FF51FE554FB4D80817B
:10053000846012C0862F90E0FC0125E0EE0FFF1FC3
:100540002A95E1F7880F991FE80FF91FE40FF51FAF
:10055000E554FB4D80818B7F80838091AB2590910A
:10056000AC25DF91CF911F910F91FF90EF90DF901D
:10057000CF90BF90AF900895EF92FF920F931F938B
:10058000CF93DF93EC017A018B011092B02510928A
:10059000AF251092AA252091632930E040E0ABE01E
:1005A000B0E086E190E0289FB001299F700D389F50
:1005B000700D112416C0242F2F5F842F90E08A9F86
:1005C000F0018B9FF00D9A9FF00D1124E60FF71F9D
:1005D000E259FB4D8285882319F44093AA250FC068
:1005E000422F423040F34093AA25423041F40E940A
:1005F0000AB862E070E00E945AB68093AA25E091A2
:10060000AA258BE0E89FF00111248091632926E15F
:10061000829FC0011124E80FF91FE259FB4DF093AE
:10062000B025E093AF25C193D193CF01B801A701C5
:100630000E943B872091AA2530E04091632950E039
:100640008BE090E0289FF001299FF00D389FF00D7E
:10065000112486E190E09C01429FC001439F900DD0
:10066000529F900D1124E80FF91FE259FB4D81E0D4
:1006700082878091AF259091B025DF91CF911F9116
:100680000F91FF90EF900895EF92FF920F931F93B9
:10069000CF93DF937C011092AC251092AB25109282
:1006A000AA2500916329202F30E088E890E0289F58
:1006B000E001299FD00D389FD00D11243EC0812F1D
:1006C00090E0FC0175E0EE0FFF1F7A95E1F7880FCF
:1006D000991FE80FF91FEC0FFD1FE554FB4D8081BA
:1006E00081FF28C0212F30E0C90155E0880F991FF4
:1006F0005A95E1F7220F331F820F931F8C0F9D1F16
:1007000086569B4DB70140E150E00E94F1BB009737
:1007100089F482E2189FC001112428E8029F900109
:100720001124820F931F86569B4D9093AC25809386
:10073000AB2508C01F5F1093AA251091AA2514307D
:1007400008F4BDCF8091AB259091AC25DF91CF917E
:100750001F910F91FF90EF900895EF92FF921F93DA
:10076000CF93DF937C011092AA258091632990E0BA
:1007700028E830E0829FE001839FD00D929FD00D4A
:10078000112442C0812F90E0FC0175E0EE0FFF1FA5
:100790007A95E1F7880F991FE80FF91FEC0FFD1FFD
:1007A000E554FB4D808181FF2CC0212F30E0C90131
:1007B00055E0880F991F5A95E1F7220F331F820FDA
:1007C000931F8C0F9D1F212F30E0F901B5E0EE0F34
:1007D000FF1FBA95E1F7220F331FE20FF31FEC0F53
:1007E000FD1FE656FB4D4089469546954695865633
:1007F0009B4DB70150E00E94F1BB009711F481E0DE
:1008000009C01F5F1093AA251091AA25143008F47F
:10081000B9CF80E0DF91CF911F91FF90EF900895C5
:10082000CF92DF92EF92FF920F931F93CF93DF93BC
:10083000EC011092AE251092AD251092AA250091E0
:100840006329202F30E0E1E3CE2ED12C88E891E01F
:10085000289F7001299FF00C389FF00C11243AC09A
:10086000812F90E08C9D90018D9D300D9C9D300DD1
:1008700011242E0D3F1DF901E25AFE4D85A5882356
:1008800031F1408D8885481711F5C90182599E4D77
:10089000BE0150E00E94F1BB0097C9F481E3189FAC
:1008A000C0011124402F50E028E831E0B901469FF3
:1008B0009001479F300D569F300D1124820F931FDA
:1008C000825A9E4D9093AE258093AD2507C01F5F41
:1008D0001093AA251091AA25183010F28091AD2509
:1008E0009091AE25DF91CF911F910F91FF90EF90E6
:1008F000DF90CF900895CF92DF92EF92FF920F9307
:100900001F93CF93DF937C011092AE251092AD25FB
:100910001092AA2500916329202F30E0F1E3CF2E19
:10092000D12C88E891E0289FE001299FD00D389FC5
:10093000D00D112434C0812F90E08C9DF0018D9D4D
:10094000F00D9C9DF00D1124EC0FFD1FE25AFE4DA1
:1009500085A5882309F1CF01B70140E150E00E944D
:10096000F1BB0097C9F481E3189FC0011124402F07
:1009700050E028E831E0B901469F9001479F300DD3
:10098000569F300D1124820F931F825A9E4D9093D3
:10099000AE258093AD2507C01F5F1093AA25109147
:1009A000AA25183040F28091AD259091AE25DF91B7
:1009B000CF911F910F91FF90EF90DF90CF9008950E
:1009C000BF92CF92DF92EF92FF920F931F93CF933C
:1009D000DF93D82EC92E8B01B42E79011092AE254B
:1009E0001092AD251092AA252091632930E040E0B5
:1009F000A1E3B0E088E891E0289FB001299F700D45
:100A0000389F700D112416C0242F2F5F842F90E083
:100A10008A9FF0018B9FF00D9A9FF00D1124E60F35
:100A2000F71FE25AFE4D85A5882319F44093AA25A5
:100A30000FC0422F483040F34093AA25483041F47C
:100A40000E940AB868E070E00E945AB68093AA2516
:100A5000409163299091AA2581E3989FE001112498
:100A6000242F30E088E891E0BC01269FC001279F39
:100A7000900D369F900D1124C80FD91FC25ADE4D1C
:100A8000D093AE25C093AD25DE012D2D3C2DC9019F
:100A9000FC0180E101900D928150E1F701151105F3
:100AA000C9F01092AA25E0E00AC0F0E0DE01AE0F26
:100AB000BF1FE00FF11F808150968C93E92FD80162
:100AC00018968C919E2F9F5FE81778F3E093AA25E4
:100AD000888F1BC0842F90E0FC01A3E0EE0FFF1F66
:100AE000AA95E1F7E80FF91FE459F64D40859E01FC
:100AF000205F3F4FC90160E070E050E00E9419BCE8
:100B0000E091AD25F091AE25108EE091AD25F091EC
:100B1000AE25B18EF38EE28ECF014C9640E050E0D0
:100B200060E070E00E943B878091AD259091AE25FA
:100B3000849640E050E060E070E00E943B87E091E6
:100B4000AD25F091AE2514A681E085A7CF01DF91F8
:100B5000CF911F910F91FF90EF90DF90CF90BF90BA
:100B600008951F9310916329412F50E020E0A1E3E5
:100B7000B0E088E891E0489FB001499F700D589F10
:100B8000700D11240FC0822F90E08A9FF0018B9F7F
:100B9000F00D9A9FF00D1124E60FF71FE25AFE4D5B
:100BA00015A62F5F283078F320E0ABE0B0E086E1B7
:100BB00090E0489FB001499F700D589F700D11241F
:100BC0000FC0822F90E08A9FF0018B9FF00D9A9FBB
:100BD000F00D1124E60FF71FE259FB4D12862F5F2F
:100BE000223078F320E088E890E0489FB001499FE8
:100BF000700D589F700D112414C0822F90E0FC01DD
:100C0000A5E0EE0FFF1FAA95E1F7880F991FE80FE7
:100C1000F91FE60FF71FE554FB4D80818D7F808320
:100C20002F5F243050F32093AA2587E191E0489F5D
:100C3000F001499FF00D589FF00D1124EE5CF04D2E
:100C40008589882309F464C088E890E0489F900172
:100C5000499F300D589F300D1124D901A656BB4D28
:100C60008EEF90E811969C938E9384E490E0489FD9
:100C7000F001499FF00D589FF00D1124EE0FFF1F5A
:100C8000E456FB4D11821082FA01EE0FFF1FCA01DC
:100C900075E0880F991F7A95E1F7E80FF91FEE0FBD
:100CA000FF1FEE0FFF1FE256FB4D118210821796B9
:100CB0001C921E921697FA0194E0EE0FFF1F9A9570
:100CC000E1F7E40FF51F83E0EE0FFF1F8A95E1F7D0
:100CD000EE55FB4D118210821B961C921E921A97A4
:100CE0001D961C921E921C971F961C921E921E9778
:100CF00080E450968C9325543B4DF90180818360AC
:100D00008083812F40EA56E861E070E00E94FC8811
:100D10001F910895FFCF0895CF92DF92EF92FF9237
:100D20000F931F93DF93CF93CDB7DEB729970FB6FD
:100D3000F894DEBF0FBECDBF8C018091632988235C
:100D400039F501151105A1F483E389838A83809124
:100D5000072A8B838091082A8C838091092A8D83AE
:100D600080910A2A8E8386E089878E010F5F1F4F4C
:100D7000E0906429F090652980E060E040E050E078
:100D800026E093EEC92E99E2D92E0E945D8F10C005
:100D9000813091F40115110541F48FEF89838A8325
:100DA00082E089878E010F5F1F4FC8010E944B4F61
:100DB000109265291092642980E090E029960FB680
:100DC000F894DEBF0FBECDBFCF91DF911F910F9181
:100DD000FF90EF90DF90CF9008950F931F93DF93D4
:100DE000CF9300D000D0CDB7DEB78C01CE010196F5
:100DF0000E94E312F801208131814281538189816F
:100E00009A81AB81BC81281B390B4A0B5B0BB90162
:100E1000CA010F900F900F900F90CF91DF911F910B
:100E20000F9108950F931F93DF93CF9300D000D0BD
:100E3000CDB7DEB78C01CE0101960E94E31260E0CF
:100E400070E0F801208131814281538189819A814A
:100E5000AB81BC81281739074A075B0710F461E0B2
:100E600070E0CB010F900F900F900F90CF91DF911A
:100E70001F910F910895CF92DF92EF92FF920F93FF
:100E80001F93DF93CF9300D000D0CDB7DEB76C01B6
:100E90007A018B01CE0101960E94E312F601E482F1
:100EA000F5820683178389819A81AB81BC818E0D7F
:100EB0009F1DA01FB11F80839183A283B3830F90D6
:100EC0000F900F900F90CF91DF911F910F91FF9096
:100ED000EF90DF90CF900895882321F48DE00E9459
:100EE00021140895813019F48CE00E942114089592
:100EF000882321F489E00E9421140895813019F497
:100F000088E00E942114089584E00E94211485E065
:100F10000E94211486E00E94211487E00E9421147F
:100F200088E00E94211489E00E9421148AE00E9436
:100F300021148BE00E9421148CE00E9421148DE08A
:100F40000E9421148EE00E9421148FE00E9421143F
:100F500080E10E94211481E10E9421140895AF9242
:100F6000BF92CF92DF92EF92FF920F931F935A019D
:100F70006B01813031F480E120E030E005EB19E8CD
:100F800005C081E120E030E00EEA19E8EE24FF24FC
:100F90000E942D158823B9F0A114B104C104D10415
:100FA00091F000D000D085E398E0EDB7FEB79283D2
:100FB00081838EEE91E0948383830E9424BD0F9001
:100FC0000F900F900F901F910F91FF90EF90DF9077
:100FD000CF90BF90AF900895AF92BF92CF92DF9223
:100FE000EF92FF920F931F935A016B01813031F4FE
:100FF0008EE020E030E004EC19E805C08FE020E04E
:1010000030E00DEB19E8EE24FF240E942D15882313
:10101000B9F0A114B104C104D10491F000D000D002
:1010200085E398E0EDB7FEB79283818388ED91E088
:10103000948383830E9424BD0F900F900F900F9094
:101040001F910F91FF90EF90DF90CF90BF90AF90E6
:101050000895AF92BF92CF92DF92EF92FF920F93DB
:101060001F935A016B01813031F48CE020E030E0B5
:1010700003ED19E805C08DE020E030E00CEC19E844
:10108000EE24FF240E942D158823B9F0A114B10489
:10109000C104D10491F000D000D085E398E0EDB711
:1010A000FEB79283818381EC91E0948383830E94D5
:1010B00024BD0F900F900F900F901F910F91FF90F4
:1010C000EF90DF90CF90BF90AF900895AF92BF9216
:1010D000CF92DF92EF92FF920F931F93282F5A0126
:1010E0006B01E82FF0E0411551056105710551F4E0
:1010F000EE0FFF1FEF54FA4D808191815C01CC24EB
:10110000DD2406C0EE0FFF1FEF54FA4D51834083DC
:10111000213041F48AE0B601A50120E030E009EE7B
:1011200019E807C08BE0B601A50120E030E00BED27
:1011300019E8EE24FF240E942D158823B9F0A1148C
:10114000B104C104D10491F000D000D085E398E04F
:10115000EDB7FEB7928381838AEA91E0948383831B
:101160000E9424BD0F900F900F900F901F910F9130
:10117000FF90EF90DF90CF90BF90AF900895AF9227
:10118000BF92CF92DF92EF92FF920F931F935A017B
:101190006B01813031F488E020E030E00EEF19E897
:1011A00005C089E020E030E007EF19E8EE24FF24D5
:1011B0000E942D158823B9F0A114B104C104D104F3
:1011C00091F000D000D085E398E0EDB7FEB79283B0
:1011D00081838DE891E0948383830E9424BD0F90E6
:1011E0000F900F900F901F910F91FF90EF90DF9055
:1011F000CF90BF90AF900895AF92BF92CF92DF9201
:10120000EF92FF920F931F93282F5A016B01E82F43
:10121000F0E0411551056105710551F4EE0FFF1F16
:10122000EB54FA4D808191815C01CC24DD2406C011
:10123000EE0FFF1FEB54FA4DB182A082213041F432
:1012400086E0B601A50120E030E004E11AE807C01D
:1012500087E0B601A50120E030E006E01AE8EE24C0
:10126000FF240E942D158823B9F0A114B104C104F4
:10127000D10491F000D000D085E398E0EDB7FEB73F
:101280009283818387E791E0948383830E9424BDC6
:101290000F900F900F900F901F910F91FF90EF9074
:1012A000DF90CF90BF90AF900895AF92BF92CF9252
:1012B000DF92EF92FF920F931F93282F5A016B0139
:1012C000E82FF0E0411551056105710551F4EE0F6D
:1012D000FF1FE754FA4D808191815C01CC24DD240D
:1012E00006C0EE0FFF1FE754FA4DB182A0822130F5
:1012F00041F484E0B601A50120E030E000E31AE803
:1013000007C085E0B601A50120E030E002E21AE85E
:10131000EE24FF240E942D158823B9F0A114B104F6
:10132000C104D10491F000D000D085E398E0EDB77E
:10133000FEB7928381838AE591E0948383830E9440
:1013400024BD0F900F900F900F901F910F91FF9061
:10135000EF90DF90CF90BF90AF90089510926329E7
:101360000E94B8610E94D969089581E08093632941
:101370000E94B8610E94D9690895109263290E9461
:10138000AF620E94D969089581E0809363290E9429
:10139000AF620E94D9690895109263290E94346354
:1013A0000E94D969089581E0809363290E94346383
:1013B0000E94D96908951092632980E040E050E0CE
:1013C00060E070E00E9466880E943F670E94D969D1
:1013D000089581E08093632940E050E060E070E090
:1013E0000E9466880E943F670E94D9690895109202
:1013F00063290E9476640E94D969089581E08093F0
:1014000063290E9476640E94D96908951092632925
:1014100080E040E050E060E070E00E94FC880E94C4
:1014200050800E94D969089581E08093632940E04B
:1014300050E060E070E00E94FC880E9450800E94B2
:10144000D96908951092632980E040E050E060E09F
:1014500070E00E9455890E94FB6C0E94D969089532
:1014600081E08093632940E050E060E070E00E94FA
:1014700055890E94FB6C0E94D96908950F931F93B0
:10148000DF93CF93CDB7DEB762970FB6F894DEBF88
:101490000FBECDBF9A8B898BFB0181E080936329BE
:1014A0008A898093603189898093613182E0809359
:1014B0007D298081809375298181809376298EEFA3
:1014C00090E89A8389831C821B821E821D82188663
:1014D0001F821A8619861C861B861E861D86188A00
:1014E0001F86CE01019660E420E030E040E050E04D
:1014F00001E010E00E94546662960FB6F894DEBFD9
:101500000FBECDBFCF91DF911F910F910895CF9264
:10151000DF92EF92FF920F93DF93CF93CDB7DEB7B9
:1015200029970FB6F894DEBF0FBECDBFAC01FE0108
:10153000319689E0DF011D928A95E9F786E0898777
:10154000109263294115510581F020E030E0BF0180
:10155000FB01E20FF31FDA01A20FB31F8C9180830E
:101560002F5F3F4F2630310599F786E0898783E664
:1015700098E00E94B86968E077E080E090E041E0A0
:1015800021E000E0BAE4EB2EB8E0FB2E6E010894F7
:10159000C11CD11C0E94DA6080E040E251EA67E0A1
:1015A00070E00E94558929960FB6F894DEBF0FBEF1
:1015B000CDBFCF91DF910F91FF90EF90DF90CF9053
:1015C0000895CF92DF92EF92FF920F936C0101E0AA
:1015D000009363298091810390918203892BC1F448
:1015E00083E598E00E94B8690093632968EE73E090
:1015F00080E090E041E021E000E05EE4E52E58E08C
:10160000F52E0E94DA6083E598E00E94B0460DC096
:1016100060E070E080E090E040E021E000E03EE447
:10162000E32E38E0F32E0E94DA6081E040E251EAD6
:1016300067E070E00E9455890F91FF90EF90DF9076
:10164000CF9008958DEB95E29093602980935F2968
:101650000E9484870E94B4460895FC0120E0908196
:101660008181808391832E5F32962031C1F7089566
:10167000992787FD90950E94B8BB8A3314F0875351
:10168000089580530895FF920F931F938C01FC01DE
:1016900080810E94388BF82EF29480EFF822F801B6
:1016A00081810E94388B8F0D1F910F91FF900895BB
:1016B000992787FD90950E94B0BB8833A1F18933AB
:1016C00084F4843341F185333CF4823301F1833374
:1016D00004F58133D1F417C0863309F187330CF553
:1016E0001CC0833641F184363CF4813601F18236E8
:1016F00004F5893351F419C0853609F18536ECF0CB
:10170000863619F41EC081E0089580E0089582E0D5
:10171000089583E0089584E0089585E0089586E0C3
:10172000089587E0089588E0089589E008958AE0A3
:1017300008958BE008958CE008958DE008958EE083
:1017400008958FE00895EF92FF921F93CF93DF9358
:101750007C01EC0110E001C01F5F8881992787FDA3
:1017600090950E9494BB892B19F4C0E0D0E022C070
:101770002196143089F7F9CFF70180810E94588BA8
:1017800090E0143029F4982F88279295907F0CC010
:10179000133019F4982F882707C0123029F424E059
:1017A000880F991F2A95E1F7C80FD91F1150089487
:1017B000E11CF11C112301F7CE01DF91CF911F91A4
:1017C000FF90EF9008955F926F927F928F929F9219
:1017D000AF92BF92CF92DF92EF92FF920F931F933F
:1017E000DF93CF9300D000D00F92CDB7DEB74C017E
:1017F0006B018C019C01A8E0EA2EFF24F8E05F2E2B
:101800005E010894A11CB11CE5E06E2E712C6C0EDB
:101810007D1E02C00F5F1F4FF80140814A3311F057
:101820004423C1F7C801821B930B059714F080E095
:101830005EC0F80182918F010F5F1F4F8A3319F04C
:10184000D501F9012FC0442319F0F40190E00EC036
:10185000EF2DF0E0EE0FFF1FEC0DFD1D1182108249
:10186000F39440C08A3309F49F5F319680818823C6
:10187000C9F7252D291B922F8F2D0AC0E82FF0E0E4
:10188000EE0FFF1FEC0DFD1D1182108291508F5F36
:101890009923A1F7F20EE21A0F5F1F4F98011FC0A4
:1018A0008D9331969E2F921B80818A3319F0A61555
:1018B000B705B1F7F501E90FF11D1082C5010E94CE
:1018C000A38BEF2DF0E0EE0FFF1FEC0DFD1D9183BC
:1018D000808398012F5F3F4FF394EA948901EE20B3
:1018E00009F09ACF80E0F8E0FF1609F481E00F904C
:1018F0000F900F900F900F90CF91DF911F910F914C
:10190000FF90EF90DF90CF90BF90AF909F908F901F
:101910007F906F905F900895AF92BF92CF92DF92C9
:10192000EF92FF920F931F93CF93DF938C01EB0104
:101930006115710509F46BC0EE24FF2433E7C32E53
:1019400038E0D32E20E3A22E9AE3B92E8881998124
:10195000009779F5EE2069F540E06F2D70E001C049
:101960004F5F242F30E0F901EE0FFF1FEC0FFD1F3A
:1019700080819181892B29F4260F371F283031056A
:101980007CF3413039F4D801AD928D01F394229665
:1019900040E030C08F2D90E0840F911D089709F42E
:1019A0004150842F90E0880F991FC80FD91FF40E63
:1019B00021C00E94B15600D000D000D0EDB7FEB7D4
:1019C0003196ADB7BEB712961C930E931197D38282
:1019D000C282958384830E9495BD080F191F2296A9
:1019E000F3944E2DEDB7FEB736960FB6F894FEBFC2
:1019F0000FBEEDBFF8E0FF1641F0D801BD928D019A
:101A0000B7E0BF1510F0E42EA1CFF8011082DF91EE
:101A1000CF911F910F91FF90EF90DF90CF90BF90EB
:101A2000AF900895AF92BF92CF92DF92EF92FF9264
:101A30000F931F93DF93CF9300D000D000D0CDB78A
:101A4000DEB77C0100E010E05E010894A11CB11C2F
:101A500046E7C42E48E0D42E00D000D000D0EDB729
:101A6000FEB73196ADB7BEB71296BC92AE92119743
:101A7000D382C282D701A00FB11F8C9184831582BB
:101A80000E9495BD0F5F1F4F8DB79EB706960FB68C
:101A9000F8949EBF0FBE8DBF00311105E9F6269662
:101AA0000FB6F894DEBF0FBECDBFCF91DF911F916F
:101AB0000F91FF90EF90DF90CF90BF90AF9008957F
:101AC0001F93CF93DF939C01EB01142F8091642926
:101AD00090916529892B19F02FEF3FEF13C083EE0A
:101AE00099E2B901AE010E9407BC10936329D0931B
:101AF0006529C093642981E00E944D570E94D969ED
:101B000020E030E0C901DF91CF911F910895DC0101
:101B10009C9111968C9111979F5F983728F090E0D7
:101B200003C06B9A639A08959817D9F38C91FD01BD
:101B3000E80FF11D62839C930895DC0111969C913E
:101B40001197FD01E90FF11D22818C918C9198175D
:101B500011F42FEF07C0892F8F5F883708F080E0DE
:101B600011968C93822F0895FC019081818120E051
:101B7000981321E0822F0895FC018081282F30E006
:101B80008181281B310937FF02C028583F4F822F1F
:101B900008951092543780915437809353371092A0
:101BA000CE378091CE378093CD3788E98093C100BE
:101BB00086E08093C2001092C50083E08093C40049
:101BC00010926D2608951092C1000895682F7894A0
:101BD0008DEC97E30E94878D8091C10085FD21C027
:101BE0008091C00085FFFCCF9091CE37E92FF0E0C7
:101BF000E353F84C22818091CD378091CD379817EF
:101C000011F42FEF07C0E92FEF5FE83708F0E0E0AD
